:020000040800F2
:1000000000A0002069C00008B995000841B10008AF
:10001000B7950008B5950008B395000800000000EA
:10002000000000000000000000000000B195000882
:10003000AF95000800000000AD95000831B1000840
:10004000B5C00008B5C00008B5C00008B5C00008BC
:10005000B5C00008B5C00008B5C00008B5C00008AC
:10006000B5C00008B5C00008B5C00008B5C000089C
:100070004196000801B1000889960008B5C0000843
:10008000B5C0000861960008B5C00008B5C00008FA
:100090006D8E0008B5C00008B5C00008B5C00008E6
:1000A000CD950008FD950008BB9500080D96000849
:1000B000ED950008DD950008B5C00008B5C0000842
:1000C000B5C00008B5C00008B5C00008B5C000083C
:1000D000B5C0000835960008299600081D9600084E
:1000E000B5C00008B5C000089D950008B5C000085F
:1000F000B5C00008B5C00008B5C00008B5C000080C
:10010000000000000000000000000000B5C0000872
:10011000B5C00008B5C00008B5C00008B5C00008EB
:10012000B5C00008B5C00008B5C00008B5C00008DB
:10013000B5C00008B5C000080000000000000000C5
:10014000B5C00008B5C00008B5C000080000000038
:10015000000000000000000000000000000000009F
:100160000000000000000000B5C00008B5C0000895
:10017000B5C0000800000000000000000000000002
:0801800000000000B5C00008FA
:100188002DE9F04F2DED068B5A4C5B4B23609DB04B
:100198000023636005F076FD18B907F0ADFD09F09E
:1001A800A7FE06F023FD554B554D4FF47002C3F8DA
:1001B80088200023059306932B6843F480332B6033
:1001C8002B6803F400330693059B01330593069BC4
:1001D8001BB9059BB3F5A04FF2D12B6813F400337C
:1001E80018BF01230693069B012B59D0434F454B5B
:1001F800FB606B6A43F080736B626B6943F4FC03CA
:100208001CAE6B6103238DF8223041F6FF7326F88C
:10021800503D4FF09040314604F07FFF4FF6FF739A
:100228003948ADF82030314604F077FF3748314679
:1002380004F073FF3648314604F06FFF3548314605
:1002480004F06BFF3146344804F067FF304604F091
:1002580093FD089B314AB3FBF2F3A360304B314A5C
:100268005A60F02287F82320072200279F60642025
:100278001A6007F0C3FC2C483946C8220DF0F5FC7B
:10028800EB6943F00303EB61AB6943F4A123AB6172
:100298006B6943F4C0236B61244B03F1DC0049E034
:1002A800234B12221A606B686B606B686B606B681B
:1002B80043F480636B606B6823F47C136B606B683A
:1002C80043F4E8136B602B6843F080732B602A6853
:1002D8000B4B9201FBD55A6822F003025A605A6808
:1002E80042F002025A606B6803F00C03082BFAD143
:1002F8007CE700BF080700209134000800ED00E00B
:10030800001002400005FA050004004800080048F3
:10031800000C0048001000480014004840420F003C
:1003280010E000E03F1901009C0F0020081B0108A5
:10033800002002401A7B93F80DE053F8147B02F07A
:100348000701D20807EB82028900176A4FF00F0CE9
:100358000EFA01FE0CFA01F127EA01011162176A8F
:1003680083424EEA07011162E4D10023DFF860936B
:1003780009F10C024FF0000803F8028001330B2B3F
:10038800F4D1DFF850A3C04FFF2389F8173089F85C
:10039800183089F8193089F81A3089F81B309AE82A
:1003A8000F0086E80F006B69089843F480236B619F
:1003B8006B6943F480236B61B44B10229A6120224D
:1003C8009A6109A904F0A9FE0A980BA904F0A5FEF0
:1003D8006B69C9F81C7043F400336B61EB6943F433
:1003E8008003EB612B6B23F020032B632B6B43F013
:1003F800805343F020032B634FF0904528466B6AE7
:1004080023F0F0036B626B6A43F040036B626B6A24
:1004180023F470636B626B6A43F480636B6202233C
:100428008DF8243003238DF8253031464FF40073BE
:1004380008938DF826808DF8278004F02FFE4FF45E
:10044800806328463146089304F028FE3B68904DA7
:1004580023F001033B603A688E4B13403B608E4BA0
:100468003B613B6843F001033B60C7F80880C7F86D
:100478000C80C7F80880BB6843F40043BB603B6846
:100488003B607B6823F0784323F400437B603B6840
:1004980043F001033B60B5F8E6305BB9B5F9E820F5
:1004A8003AB9B5F9EA80D8F1010838BF4FF0000829
:1004B80000E0984618F00108DFF81C926AD11BB2D8
:1004C80008EE903AB5F9E800B5F9EA10DFED737A6D
:1004D80089F80080F8EEE88A08EE100A0AEE901A09
:1004E80068EEA78AB8EEC88AF8EEEAAAB0EE680AFB
:1004F80028EE278A6AEEA7AA0DF0E6FDB0EE409A2C
:10050800B0EE680A0DF066FEF0EE409AB0EE480ACA
:100518000DF0DAFDF0EE408AB0EE480A0DF05AFE12
:10052800B0EE408AB0EE6A0A0DF0CEFDB0EE40AAF9
:10053800B0EE6A0A0DF04EFE20EE097A69EE8A7A6C
:10054800F0EE475AE7EE885A2AEE096A69EE806AA1
:10055800C4ED0B5AF0EE465AE6EEC85AE7EE087AB2
:10056800E6EE486A2AEE28AA28EEC00A69EEE89A5A
:1005780068EE898A84ED08AA84ED090A84ED0A8A5E
:10058800C4ED0C5AC4ED0D9AC4ED0E6AC4ED0F7A91
:10059800C4ED108AAB689B0318D5C82007F02EFB62
:1005A80008F0D6F8C82007F029FB3D4B3D486364A6
:1005B80000210C220DF059FB022384F84B3008F07F
:1005C80039F902F06DFE384B03442365374F38493B
:1005D8003B68B5F8EEB095F8ED8043F002033B6058
:1005E800344B1A68B2F85220039200220A706265EE
:1005F800029307F0FFFD8246002800F085812E4B0C
:100608002E4A1A602E4A5A60BBF1BB0F2D4ADA6097
:1006180001D9012312E0BBF1610F01D902230DE0DA
:10062800BBF1290F01D9032308E0BBF1130F01D94E
:10063800042303E0BBF1090F07D9052389F801302A
:100648003B6843F001033B6011E00623F6E7B8F18D
:100658000A0F13D0B8F1000F40D01B4B1B78002BAA
:1006680040F09580B8F1000F00F08D809846174B48
:100678000022B8F1080F1A70E9D12FE03B6823F087
:1006880002033B60E9E700BF00580040000400484F
:10069800041A0020FFE0CF007A25E00035FA8E3CEE
:1006A800141B002050070020404B4C00FC02002087
:1006B800B2040020980400209C0400201184000843
:1006C8001382000890C1793DF12000201A0500200E
:1006D8000807002064010108100000204FF0000BFB
:1006E800DFF83C92C4F854B007F084FD0028B4D079
:1006F80006213346D0200A4607F0BEFC9DF8233079
:100708009DF825C003F001035B000CF0010C43EADF
:100718008C0C9DF8213003F001035CEA030C09D02E
:10072800BCF1010F02D189F858B01CE0BCF1020FEE
:100738000FD115E007ABD0200C210122CDF808C05D
:1007480007F09AFC9DF81C30DDF808C013F00F0381
:1007580001D10520D9E0042B02D189F858C002E064
:10076800012389F858306A4B6A4A1A606A4A5A6003
:1007780094F85820002A14BF6E226F221A72674B11
:1007880008221A7069E73B6823F002033B600A20DD
:1007980007F034FA7720A021012207AB07F06CFCA0
:1007A80000285FD01E210122772009F02FF802F0DF
:1007B80077FD804602F074FDC8EB0000B0F52F6F9E
:1007C800F8D34FF00008A8F160014FF00009C9B252
:1007D8000222334677208DF820908DF8219007F07B
:1007E8004BFC9DF821309DF8201043EA01214C4B29
:1007F80003F15A0228F8021008F10208B8F1100FA4
:10080800E1D1B3F8686006F00F0006F47F46A3F85C
:10081800686001224B4623F001012144B1F85A10C7
:10082800002918BF002213F0010F04D0C9B289EAC9
:100838000109082102E089EA1129FAE719F4004FB1
:1008480018BF89F4C05901394FEA4909F6D1013373
:10085800102BE0D10643A4F868601AB9C9F303392C
:1008680048453ED03B6823F004033B6095F8E230EE
:100878000BB12C4A137095F8E3300BB12A4A137068
:1008880095F8E4300BB1294A13703B689E0702D5EE
:100898001F4B1B689847264E336898473B6813F0F0
:1008A800080FB0461AD0039B1AB2642392FBF3F1E7
:1008B80003FB11231BB207EE103AF8EEC76A07EEE6
:1008C800101AF8EEC77A9FED1B7AE6EE877AB2EE39
:1008D800047A67EE877AC4ED1B7A39E00023E36671
:1008E80036E0154B42F210721A805A80134A5A6049
:1008F800134A9A60134ADA60134A1A61134A5A6112
:10090800BAF1000FB2D1ADE7032009F0D3FA00BF66
:10091800080500204D5F0008BD810008F120002077
:1009280008070020B20400201A050020F220002049
:100938009C0400208988883C300300200784000834
:100948009D810008FD830008AD810008972C0008F0
:10095800A14B20221A8510229A614FF00A099E4E57
:10096800B38A9BB283F02003B382B38A9BB283F02D
:100978001003B382192007F041F909F1FF39192052
:1009880007F03CF919F0FF09E9D11023B3612023DE
:10099800B361924B9FED928A1B68924E93F90C308B
:1009A800DFF8749200EE103AB8EEC00A20EE080A9A
:1009B8000DF08AFB308807EE900AF8EEE77A27EE0A
:1009C800800A0DF0BDFB36889FED877A874B6979E1
:1009D800188007EE906AF8EEE77A854B854A8648D4
:1009E8001170C7EE277A00EBC101844E497CC4F828
:1009F80074909FED837AC7EE877AC3ED007AD8EDBD
:100A0800037A804B27EE888ADFED7F7A28EE278AE3
:100A180083ED008A7D4B23677D4B1960A968984652
:100A280011F0200F1CBF0123C8F8003005F0B8FEF4
:100A3800162206F17800FF210DF017F9002384F83B
:100A480078303B680122980784F88E2007D586F80D
:100A58007920032286F88E20022286F87A20590708
:100A680008D594F88E20511C224484F88E10032156
:100A780082F8781013F00A0F14D094F88E30E21828
:100A8800042182F878105A1C54FA82F2052182F85F
:100A98007810DA1C023354FA83F384F88E20062285
:100AA80083F87820AB689A0608D594F88E20511CF4
:100AB80084F88E101444072284F8782013F0800FED
:100AC8004E4C0ED094F88E20A118092081F8780099
:100AD800911C013254FA82F284F88E100A2182F8AD
:100AE80078106A79082A01D00E2A08D194F88E2045
:100AF800511C224484F88E100B2182F8781094F847
:100B08008E203E48A6180C27511CC9B286F878706A
:100B18005F0784F88E1006D50232014480F88E20D3
:100B2800102281F8782094F88E203448A6181227CD
:100B380086F8787095F84561511CC9B2002E0CBF33
:100B4800002603F0010684F88E1036B10232014403
:100B580080F88E20132281F878209E0508D594F815
:100B68008E305A1C234484F88E20152283F878206E
:100B78002848284E002198220DF077F806F19809A8
:100B880096F84A30EBB9D5F830219A4600270097F5
:100B98000120394603230AF04FF8834638B9BAF1E1
:100BA800000F11D14FF496424FF0010AEEE730469C
:100BB80039464C220DF059F80123C6F800B086F8E2
:100BC8004A304C364E45DBD10220666F02F0E2FA1D
:100BD80020B3416823E000BF00040048540500200A
:100BE80035FA8E3C000000200AE81C4178050020F8
:100BF8004C040020DA0500206401010808070020E1
:100C080000401C4650050020BD378635141A0020C8
:100C1800FC06002098070020301B00200146C4F87D
:100C2800281141B9009103230220B2680AF004F8A0
:100C3800C44BC3F8280108A8002114220DF015F8A8
:100C48006B790E2B01D0082B02D101238DF82A30A5
:100C5800BD4EBE48B368C3F34002C3F380418DF86C
:100C68002420C3F380128DF826208DF82510C3F3B5
:100C78004032D8F800108DF82020C3F3C03200317C
:100C88008DF82220C3F3C02218BF01218DF823203C
:100C9800C3F300428DF827208DF8281003F00102D5
:100CA80001688DF8212091F8B011B6F8E000ADF890
:100CB8002E00C1F380014FF47A70ADF830008DF842
:100CC8002910D804B6F8DE1044BFB6F8DA30ADF80B
:100CD8003030B1F5FA7F84BF0023ADF83030B6F874
:100CE8001A31ADF82C10ADF83230994996F8223106
:100CF80084F82C31002384F82D314B709DF82A306C
:100D0800002B14BF0223002302B10133914A02EBE6
:100D180083034FF00008D3F8C8300393C146039902
:100D280031F808004FF6FF7290424FEA10230AD1BB
:100D3800894B94F82D211A70884A1778162F40F09D
:100D48004181002531E1022B02D19DF8202003E0EA
:100D5800012B04D19DF82120002A00F0EC80C0B2BC
:100D68007F4A9DF828104FF0140C0CFB00FA02EB98
:100D78000A0551B19DF82A1039B9012805D852F849
:100D88000A10784FB94208BF04239DF8291031B1E1
:100D98009DF82A1019B90438032840F2B580012BB0
:100DA8003DD1FF230027E97B84F8743184F875313D
:100DB800AB68686884F87871C4F88451ADF81C3061
:100DC8008DF81E10022307A98DF81F3084F83071A2
:100DD800C4F83471C4F83871C4F83C71C4F870713F
:100DE80084F8767184F87771029204F096F9029A81
:100DF800297B52F80A003A4603F0C8FD284605F058
:100E080067F8594B5949C4F88831594BC4F88C31A3
:100E1800C4F8907128460A1D09F0CBFA8BE0022B22
:100E280039D154488DF81F305FFA89F11C2779436E
:100E380047184FF0010E4FF0000B87F8019087F824
:100E480002B087F80AB000F801E0E97BA868FD6005
:100E5800ADF81C008DF81E106868029207A904F00E
:100E68005CF9029A297B52F80A005A4603F08EFD73
:100E7800284605F02DF8404B3B61404B7B61C7F895
:100E880018B0284607F1100107F1140209F091FA89
:100E980009F101094FE0032B34D19DF82520BDF855
:100EA800303032B194F82E71284608214FF6FF727F
:100EB8001AE0BDF82C2094F82E71B2F5FA7F0DD9FE
:100EC8002F49B1FBF2F22846082192B209F0ACFB97
:100ED80004EB87072B4BC7F858020CE02A49B1FBF3
:100EE800F2F22846012192B209F09EFB04EB870733
:100EF800264BC7F85802C36094F82E31013384F8A2
:100F08002E3118E0042B16D1BDF82E301E4A94F865
:100F18002D7192FBF3F22846BDF83230012192B2CE
:100F280009F082FB94F82D3104EB87070133C7F8E9
:100F3800880284F82D3108F10208B8F1160F7FF401
:100F4800EEAEF5E608070020041A002098040020F9
:100F58003508002064010108B8060020DA050020E1
:100F6800041B0108004001409D2F00089008002044
:100F7800793000088008002065620008712F000899
:100F880000127A009930000840420F0089300008AA
:100F9800B54A05EB020E0FCB8EE80F00B34B1A785B
:100FA80010350132C02D1A7008D0236F2B44D3EDB1
:100FB800007AF5EE407AF1EE10FAE9D1B368DB0475
:100FC8001ED419E0AA4BA94A03EBC703D3F814802F
:100FD80093F810C082F800C0B8F1000FEED00025D9
:100FE8006545EBDAA04A2B0103EB020E43440FCB15
:100FF80001358EE80F00F3E7082F9E4D20D121E040
:101008009A4B19780129F7D99B4B00228A4203F1A0
:101018001003F1DA13ED047AF6EE007A27EE277A58
:10102800013203ED047A13ED057A27EE277A03EDF2
:10103800057A13ED037A67EE277A43ED037AE5E73D
:101048000E2F03D12B7843F0100302E02B7823F006
:1010580010032B7004F0D2FE88488949894B8A4ACC
:10106800C4F8AC3201600023B6F81A01C4F8A8121B
:10107800A4F8B23284F8B432C4F8B822C4F8BC2256
:10108800824958520233242BFAD1814B1A60B36833
:101098001F077CD57F4B93F818310022042B70D89A
:1010A800DFE803F003032A4C5B00012B4FF0030237
:1010B80008D184F8C022072284F8C23284F8C122F9
:1010C8000C2308E0022384F8C032002384F8C232DB
:1010D80084F8C122072384F8C33200230093102028
:1010E80001236D494FF4E13209F0A6FD6B4BC4F8BA
:1010F800C802C4F8CC3240E001230093684A694929
:101108000523102009F098FDB6F81A21DFED667A5C
:101118009FED667AC4F8D00206EE902AF8EEE66AE9
:101128000023E6EE877AFCEEE77A614A17EE901A1A
:1011380099500433402BF8D15E4B0AE0009201230A
:1011480010205D494FF4E13209F076FD5B4BC4F89D
:10115800D402C4F8CC3210230DE0009201231020F1
:1011680057494FF4E13209F067FD564BC4F8CC32C9
:10117800C4F8D802082384F8C332003018BF01200D
:1011880028B9082002F0D7FB0023C4F8CC32B36892
:10119800580405D5082284F8C3224B4AC4F8CC2247
:1011A80042F201021A4003F0010103F400505AB15F
:1011B800464AC4F8CC2218B1454A082082F8C3022E
:1011C80011B10C2284F8C32294F8C3221906A2F1A3
:1011D800040284F8C42240F199803D4B3D4AD6F878
:1011E8003811DFF80881C3F8DC2200233A4A02EB01
:1011F800031092464068884204D00133DBB2042BC6
:10120800F4D90023002739461522DFF8E490334843
:1012180088F80130C8F80470C8F808700CF025FD8B
:101228002F4BC9F80030384609F08AF82D4B98F84A
:1012380001201B68C8F80C30D9F800301B780097DB
:101248000AEB0212BB420CBF0123032320203946BC
:10125800526809F0F1FC244B186000284AD180201C
:1012680002F069FB49E000BFE0050020BC20002037
:101278006401010891040020E8050020EC01002029
:10128800141B00203C020108B4090020BA06002003
:10129800F0020020041A002085480008C947000809
:1012A800A0860100DD3200080000B0C4CDCCCC3FE0
:1012B8000C020020492B0008214900087548000845
:1012C800D548000861480008792B0008852B0008DC
:1012D80008070020301B00200C000108E809002046
:1012E8002C1B0020001A0020680400206C04002039
:1012F8008C040020012009F023F82B4B18682B4B95
:1013080000F5D97204301A6002F092FB01F0C8FFB0
:10131800274B18607379052B03D1264B4FF4C872FD
:101328001A80254B4FF47A721A80244BC8221A80EF
:101338002B7843F008032B70214B1A7822F0020215
:101348001A70B3689A071ED51E4BC4F8F8320825E0
:1013580003F0AAFF282006F051FC013DF8D196F8C9
:10136800051194F8FC020A460123904203D3013385
:10137800082B0A44F9D1144A137096F806215343EE
:10138800124AA2F8FE32B3689B0308D594F84B3092
:1013980043F0010384F84B30042384F84C301DB02B
:1013A800BDEC068BBDE8F08F98040020C405002032
:1013B800B00500201C050020E8200020E0200020C7
:1013C800F0200020081B0020500100200807002002
:1013D800A74B2DE9F04FB3F90600A64B1D682DED7C
:1013E800028B2B89984287B010DBB0F5FA6FAA7987
:1013F80008DAC11A4A43A3F5FA6392FBF3F364339C
:10140800009305E0C2F16402009201E064210091BA
:10141800994BB3F81A21029293F9EC30974A5B4240
:1014280016689BB20021039334460A46904B029FEC
:10143800CB5E0193DB1B03F2F31C40F2E637BC459D
:1014480003D8002BB8BF5B4201E04FF4FA73022ABD
:10145800DFF8348231D096F85D7127B1BB42CCBF3A
:10146800C7EB03030023642793FBF7FCDFF814A200
:101478006FF0630B3AF81C900BFB0C3B0CF1010C62
:101488003AF91CA00FFA89FCCCEB0A0C0CFB0BFCFC
:101498009CFBF7FCCC4428F801C095F804C003FB7A
:1014A8000CFC774B9CFBF3F33B44DDF800C09BB28C
:1014B8000CFB03F393FBF7F716E096F85E7127B180
:1014C800BB42CCBFC7EB03030023DDF80CC003FB12
:1014D8000CF7A8F804706F79002BB8BF5B427B4308
:1014E800674F93FBF7F76437B318DFF8BCC193F87D
:1014F8000480642307FB08F898FBF3F802F80C80D3
:1015080094F80E900CF1030807FB09F999FBF3F91D
:1015180002F8089094F818800CF1060C07FB08F7FD
:1015280097FBF3F302F80C30029F019BDFF858C1D8
:10153800BB4204DA3CF801305B422CF8013001323E
:10154800032A01F1020104F101047FF46FAF4A4D4F
:10155800B5F81C31984205DBB0F5FA6FA8BF4FF417
:10156800FA6000E01846C01A4FF47A725043C3F587
:10157800FA63B0FBF3F36426424C434F93FBF6F255
:1015880004EB42016FF0630000FB023304EB4202FC
:10159800098BB2F91A000AB2821A534393FBF6F682
:1015A80031443A4EACF8061033885A0634D5384BD5
:1015B800DFED387A1A88238ED31A1BB208EE903AD8
:1015C800F8EEE88A68EEA78AB0EE680A0CF07CFDAF
:1015D800B0EE408AB0EE680A0CF0FCFDB7F902C024
:1015E800B7F9000006EE90CA07EE900AF8EEE66A30
:1015F800F8EEE77A20EE667AA7EE887A67EE807AC8
:10160800BDEEC77AE6EE887A17EE103AFDEEE77A75
:101618003B8017EE903A7B80AA6840F6020313409D
:10162800002B7CD01C4B1F88636B1F4494F8383008
:1016380067630133DBB20621B3FBF1F084F838307D
:1016480001FB103313F0FF0869D1930731D503F07C
:101658002BFE124B1A78124B1B88934226D3114B40
:101668001B689B7893428CBF002301231FE000BFB7
:10167800BA060020D0050020041A00209804002093
:101688000CFEFFFF080A00201203002004030020BC
:101698009005002035FA8E3CAC050020040A002095
:1016A800060A0020000A0020160A0020434684F893
:1016B8003930AB68180530D5904A914B527BE16BB5
:1016C80033F81220082391FBF3F0091A11FA82F279
:1016D800E26392FBF3F292B240F6E4435A43894B39
:1016E80040F6FF71B2FBF1F21968C8888988121AAE
:1016F8004FF47A735A4392FBF1F2D4E9120157433B
:1017080097FBF3F3C01841EBE3712264C4E91201BB
:101718007D4A002309F026FD2065002363637B4989
:101728007B4A0B6894F8399013F4805318BF01234F
:1017380082F85430AB68774D13F4807F884627D001
:10174800754F28783B681B68C0F380005B68984732
:1017580058B1012384F855303B681B68DB6898470B
:1017680018B16B4B022283F855203B681B689B68B5
:10177800984728B12B7859075CBF022384F8553065
:101788003B681B689B69984710B1002384F8553063
:10179800624F3B689A060DD5D8F8003013F4C06F35
:1017A80005D05F4B1B789B0701D4012300E0002381
:1017B80084F8563094F85520554B022A02D14C2013
:1017C8004E211EE0012A06D153204D214C220B4602
:1017D80004F0F8FB28E093F85620012A03D153209F
:1017E80001464E2206E093F85420012A04D15320E2
:1017F800014602464D23EBE7B9F1000F04D0532010
:101808004D210A464423E3E73288160603D55320C0
:101818004D210246DBE7434A12781AB1192008F035
:1018280063FD01E083F857902A78500703D53E4BB3
:1018380010221A855BE0D8F80030D90703D435495F
:1018480042F001020A703A6812F0020202D03749E7
:101858000988A9B93649098801B12AB9354A1288CF
:10186800003218BF012200E001224AB12E4A918AB3
:1018780089B281F0100191822A7822F001022A703F
:10188800274A1278120703D42A7822F001022A7014
:10189800DB0203D52B7823F001032B702B78264A23
:1018A80013F0010F05D00023A3651F4B1021996188
:1018B8000BE0A16D136841B9154903F5F42303F54D
:1018C80090738B65184B10211985A36D126873B13D
:1018D800D21A002A0BDB144A918A89B281F01001CE
:1018E800918203F5F4230A4A03F590739365134B29
:1018F8001B782BB306F02DFE00F00EBE200C002046
:101908000C0B0020000A0020407E05000003002088
:10191800080A0020F0200020C4090020FC02002052
:10192800910400204A05002000040048E02000201F
:101938001C050020E8200020D8200020F4200020EA
:10194800C44C94F84A30012B40F0E185C24B226820
:10195800DC651A66C04E306E01F0F5FC374600288B
:1019680000F0CF85306E01F0E9FCF36D93F8482064
:10197800E2B9B0F124077A427A4183F84820002A74
:10198800E8D1B64B1B785E07E4D4232802D106F0D1
:10199800E0FDDFE7B24B1B681B7D8342DAD1B14B18
:1019A800B14A1A60B14BB24ADA60D3E7012A05D1CD
:1019B8004D2814BF0022022200F09FBD022A05D143
:1019C8003C2814BF0022032200F097BD032A0BD144
:1019D80040284FF0000200F290851A71DA715871B0
:1019E8009871042200F089BD042A07D19A7983F8F6
:1019F800490050409871052200F07FBD052AA9D101
:101A080059791A799142997906D941409971511CAD
:101A18001971134418729DE7814240F06B8593F861
:101A280049506A2D00F08F8400F28D80322D00F02D
:101A38002B8562D8242D00F00C852BD8202D00F0A2
:101A48006982222D00F0A183012D40F032852C20DF
:101A580001F0B2FC002001F080FC284601F07DFC7A
:101A6800002001F07AFC432001F077FC4C2001F0C3
:101A780074FC462001F071FC4C2001F06EFC2846F5
:101A880001F06BFC002001F068FC002001F065FC0F
:101A98000025B7E0282D00F0E48412D8262D40F068
:101AA8000885744D032001F087FCB5F9E60001F0C4
:101AB80086FCB5F9E80001F082FCB5F9EA0000F00F
:101AC800DABC2A2D00F0DA842C2D40F0F284694D1E
:101AD800072001F071FC95F8180101F03EFCB5F9FA
:101AE8001E0101F06CFCB5F91A0101F068FCB5F9AA
:101AF8001C0101F064FC00F0C7BC652D00F0E68015
:101B08000DD8402D00F0C784642D00F0CB80342D13
:101B180040F0CF84482001F04FFC002655E3672DA4
:101B280000F0C981C0F08E81682D00F00382692D14
:101B380040F0BF84504E3078400000F0FE0001F0C5
:101B48003BFC002502E2742D00F05C8321D86E2D49
:101B580000F040820DD86C2D00F0038240F2128410
:101B6800062001F029FC454B186801F049FC444B5C
:101B780004E2702D00F07482C0F05382722D00F0E0
:101B8800A783732D40F09584082001F015FC0125EA
:101B9800D2E3782D00F09B8109D8762D00F00284DD
:101BA80000F264832F2001F007FC364DE5E2A42DF6
:101BB80000F01E8411D8A02D40F07B840C2001F089
:101BC800FBFB314B186801F01BFC304B186801F027
:101BD80017FC2F4B186800F041BCF02D00F02C8446
:101BE800FE2D40F06684082001F0E6FB002001F09D
:101BF800E6FB002001F0E3FB002001F0E0FB002001
:101C080000F039BC234B1B68585D013501F0A5FB7A
:101C1800042DF7D1002001F0D2FB00251E4B585DA2
:101C2800013501F09AFB0B2DF8D100251B4B585DAF
:101C3800013501F092FB082DF8D1072001F08DFB4A
:101C48000025174B585D013501F087FB072DF8D1AA
:101C5800CCE300BF98070020080A0020F0200020ED
:101C68007C070020FC9F0020EFBEADDE00ED00E009
:101C78000400FA05041A0020CB0900200C030020F8
:101C8800540400200F070108ACF7FF1FB0F7FF1F2F
:101C9800B4F7FF1F54010020E01B0108EC1B0108EA
:101CA800F51B01080720B74D01F086FBE62001F07F
:101CB80054FB687901F051FB002001F04EFB95F8C8
:101CC8002631002B0CBF04200C20C7E30B2001F0A9
:101CD80073FBAD4BB3F9000001F071FBAB4B1A6815
:101CE800AB4B9A420CBFB6F86400B6F8660080B2F7
:101CF80000B201F064FBA74B1B68C3F3C000C3F339
:101D08008002800040EA4200C3F340021043C3F35C
:101D1800401240EAC20003F01003184301F04FFBE1
:101D28009D4B1A8812F0010F0CBF0021022112F0FE
:101D3800020F0CBF0023042312F0040F0CBF00276E
:101D4800102712F0400F0CBF4FF0000C4FF0200C82
:101D5800009312F0100F914B01970CBF00204FF425
:101D6800007012F0200F1B68CDF808C00CBF0027C8
:101D78004FF4806712F4807F0CBF4FF0000C4FF4D3
:101D8800006C03F4803E02F0080B03F4807A0390A1
:101D98000497CDF814C003F4003703F4004C03F49F
:101DA800805903F4005803F4802603F4002503F453
:101DB800801003F0C00343EA0B0343EA0A0343EA33
:101DC800090343EA080343EA0C0343EA0E033B43CF
:101DD8001E43734B029F93F800E0DDF80CC03543B7
:101DE8002843CEF3800E40EA0E0300980B43019976
:101DF80003430B43049805993B4343EA0C0303430D
:101E080012F4007F43EA01030CBF00224FF40012D2
:101E18001A43644B00201D780346AB420AD262493C
:101E28005E5C012101FA06F616421CBF9940084380
:101E38000133F2E701F0E4FA524B93F8940601F00B
:101E48008CFA52E3122001F0B7FA584B584D1B8810
:101E5800B3F5806F22D90026A85F082390FBF3F022
:101E6800023601F0ACFA062EF6D1524DB5F9000053
:101E780001F0A5FAB5F9020001F0A1FAB5F90400DC
:101E88004D4D01F09CFAB5F9000001F098FAB5F94A
:101E9800020001F094FAB5F90400ECE2B5F900008B
:101EA80001F08DFAB5F9020001F089FAB5F90400DC
:101EB80001F085FAD9E7102001F07EFA00253F4BA2
:101EC800585D013501F049FA102DF8D10DE338209D
:101ED80001F072FA00263A4F06F12C053B68ED0036
:101EE8002B440136B3F9060001F069FA3B682B442C
:101EF800B3F9080001F063FA3B682B44B3F90A0010
:101F080001F05DFA3B681D44287B01F026FA082E93
:101F1800E1D1EAE2082001F04FFA0025284B1B68BE
:101F280003EBC503013593F86D0101F016FA082D8E
:101F3800F4D1DAE2102001F03FFA0025214B585D78
:101F4800013501F00AFA102DF8D1CEE233789D421E
:101F580080F0CB821C4B33F9150001F030FA0135C3
:101F6800F4E71A4D062001F027FAB5F9000001F050
:101F780026FAB5F9020001F022FA154BB3F9000070
:101F880079E200BF041A0020AC05002024070020D5
:101F980000540040FC02002004030020000300203D
:101FA800F020002096070020800700200000002075
:101FB80064050020A4050020000700203801002047
:101FC80098040020BE200020BA0600205C040020EF
:101FD80090050020072001F0EFF9B24BB24F1878B6
:101FE80001F0BBF9306D4FF6FF75A842A8BF28462F
:101FF80020EAE07000B201F0E2F9AC4BB3F900005E
:1020080001F0DDF9AA4B386C93F80C310028B8BF01
:1020180040420BB10A235843A842A8BF284600B241
:1020280029E2A44D072001F0C7F92B68187801F0C0
:1020380094F92B68587801F090F92B68187901F019
:102048008CF92B68587901F088F92B68987901F098
:1020580084F92B68987801F080F92B68D878EEE637
:10206800954E1E2001F0A8F933681B78022B4FF01B
:1020780000056FD1336803EB850393ED090AB2EECF
:10208800048A20EE080A0CF05BF8FA28A8BFFA20A8
:1020980020EAE070C0B201F060F93368DFED877ABA
:1020A80003EB850393ED0C0A20EE270A0CF048F8A1
:1020B800FA28A8BFFA2020EAE070C0B201F04DF972
:1020C8003368DFED7F7A03EB850393ED0F0A20EE8B
:1020D800270A0CF035F86428A8BF642020EAE070CD
:1020E800C0B2013501F039F9032DC3D1072D33688A
:1020F8001ED193ED120A20EE080A0CF021F8FA28F6
:10210800A8BFFA2020EAE070C0B201F026F93368CF
:1021180093ED130A20EE080A0CF012F8FA28A8BF6B
:10212800FA2020EAE070C0B201F017F900200BE0B5
:102138002B44187901F011F933682B44987B01F08E
:102148000CF933682B44187E013501F006F90A2D85
:10215800CCD1CAE133682B44187901F0FEF8336812
:102168002B44987B01F0F9F833682B440135187E2D
:1021780001F0F3F80A2DEDD1B7E115F8010F0028A9
:1021880000F0B38101F0E9F8F7E7A02001F014F9B5
:102198000025494B1B6805F11C0203EB82035E1DF9
:1021A800484A5B790C2101FB03230135187A01F0B9
:1021B800D4F8707801F0D1F8B07801F0CEF8F07862
:1021C80001F0CBF8282DE4D18FE13B4B06271B68A3
:1021D800774307F588771F440136B87A01F0BDF8D0
:1021E800787901F0BAF8B87901F0B7F8F87901F020
:1021F800B4F8387A01F0B1F8787A01F0AEF80C2E1C
:10220800E3D172E14FF00008012500262E4B1B7820
:102218009E4222DA2D4BF15C00232A4A03EB020985
:102228009A5C8A4204D00C33B3F58A7FF5D112E068
:10223800D9F804000BF05AFD82460DB92F4601E08B
:10224800804408E0574506DAD9F80430D85D01F033
:1022580084F80137F6E70136D8E7002D00F045810C
:102268005FFA88F001F0A8F80025CEE7164E30781E
:1022780001F0A2F8002533789D4280F03681134B97
:10228800E85C00230F4A99189A5C824204D00C3308
:10229800B3F58A7FF6D102E0087A01F05EF80135DD
:1022A800E9E700BF040A0020080A0020060B002006
:1022B800041A0020D0050020980400200000C8421D
:1022C80000007A4440070108960700208007002094
:1022D800BB4DBC4E162001F06FF8002001F06FF8DE
:1022E800B5F9D00001F06BF8B5F9D20001F067F844
:1022F800B5F9D40001F063F83368B3F9A80101F027
:102308005EF8002001F05BF8002001F079F83368EE
:10231800B3F952000A2390FBF3F001F050F895F856
:10232800040101F01AF895F8060101F016F895F87D
:10233800050101F012F859E0E8B2013501F00DF895
:10234800092DF9D1D1E0102001F036F89E4B9F4DB0
:10235800187800F0020001F000F89D4B187800F0A2
:10236800FCFF286801F04CF8686801F049F8B6F9F4
:10237800680001F024F8B6F96A0001F020F8B6F90F
:102388006C0078E0052001F017F8B6F96E0001F04E
:1023980016F8B6F9700001F012F896F8720000F01D
:1023A80001004CE500F091FE0746122001F004F808
:1023B8000FB9884B02E0102F03D1874B1E685D6868
:1023C80001E000252E46384600F0C7FF304601F0F0
:1023D80017F8284601F014F8804B186801F010F837
:1023E800002000F0ECFF002000F0E9FF002026E5C7
:1023F80096F8730080000130C0B200F0DDFF96F857
:10240800730000F0AAFF002597F873309D426CD244
:10241800734E705D00F0A1FF06F11003585D00F0E7
:102428009CFF06F120033036585D00F096FF705D82
:1024380000F093FF0135E7E7624D042000F0BCFF90
:102448002B68B3F9560000F0BAFF2B68B3F95400B3
:1024580011E0042000F0B0FF594B986800F0D0FF5D
:1024680043E0574D042000F0A7FFB5F9080100F03C
:10247800A6FFB5F90A0100F0A2FF36E0012000F03E
:102488009BFF4F4B5879DAE4012000F095FF4C4B45
:1024980093F82001D3E4082000F08EFF0025484B74
:1024A8002B44013593F8100100F057FF082DF6D1A1
:1024B8001BE0C92D54D078D9D12D00F0918140F27C
:1024C800E680D42D00F0DD8200F2BB82D22D40F0F0
:1024D800B182444B1B7803F0040303F0FF05002B83
:1024E80000F09E82002000F067FF3F4BDB6D98797B
:1024F80000F033FF3C4BDB6D002283F84820FFF7E8
:1025080029BA96F8B63013B1384B394ADA603948E7
:102518004C3484427FF415AA374B1B689B0617D5A9
:10252800364B314A1B68D2F8B810591A00290FDB0C
:102538002749097804290BD903F5123303F5F873F1
:10254800C2F8B8302E4B9A8A92B282F020029A8250
:102558002C4B9B68002B00F0E0822B489847DCE26C
:1025680000F0B3FD184B1A7810B142F0020201E0F6
:1025780022F002021A7000F0A8FD154B134D1870D6
:1025880000F0B8FD286000F0B5FD686000F0A8FD17
:10259800A6F8680000F0A4FD96F87230A6F86A0064
:1025A80043F0020386F872309CE72B2D2ED10020D1
:1025B80000F002FF00F089FD014B587192E700BF5F
:1025C800041A00209804002091040020880B0020A1
:1025D80090040020740B0020800B002008030020CA
:1025E8007C0A0020F0200020080A002000ED00E00E
:1025F8000400FA0530080020FC020020D820002042
:10260800000400489C040020C40A002034D8252D6A
:102618000BD1C74D002000F0CFFE0023AB6000F0C7
:1026280069FDAB681843A8605CE759D8212D00F014
:102638006282232D40F06C8200F047FD272821D8C4
:10264800BC4B1B6800F11C0603EB860600F03DFD41
:10265800B94B751D03F58A72197A814203D00C3380
:102668009342F9D10EE01B78737100F02EFD68706B
:1026780000F02BFDA8702FE0352D70D100F025FD5E
:102688000B2850D90120002100F078FE2AE7CD2D33
:1026980000F0E08000F27B81CA2D00F0E580CC2DAF
:1026A80040F03682A54D2E6800F00FFD30702E6880
:1026B80000F00BFD70702E6800F007FD30712E6879
:1026C80000F003FD70712E6800F0FFFCB0712E68F9
:1026D80000F0FBFCB0702D6800F0F7FCE87001E733
:1026E800272D10D1002000F067FE00F0F9FC904D76
:1026F800A5F8E60000F0F4FCA5F8E80000F0F0FC0E
:10270800A5F8EA00EEE6292D40F00282002000F04C
:1027180053FE00F0E5FC864DA5F8080100F0E0FC4A
:10272800A5F80A01DEE6834B062670431E6800F50D
:102738008870064400F0C9FC0328A3D8B07200F0E2
:10274800C4FC707100F0C1FCB07100F0BEFCF07107
:1027580000F0BBFC307200F0B8FC7072C2E622D800
:102768002D2D14D1002000F027FE00F0AEFC704D96
:1027780085F8180100F0B4FCA5F81E0100F0B0FCC3
:10278800A5F81A0100F0ACFCA5F81C01AAE6332D47
:1027980040F0BE81002000F00FFE00F096FC644B74
:1027A80083F820019EE6442D06D1002000F004FEA7
:1027B800012386F8B63095E6C82D00F09181412DA9
:1027C80040F0A681002000F0F7FD002500F07DFC18
:1027D800574B2B440135082D83F81001F6D181E6BB
:1027E80000F073FC804600F085FC074600F082FC90
:1027F800064600F07FFC054600F072FC00F070FC15
:1028080000F063FCB8F1000F12D14D4B1F605E6001
:102818004C4B1A8822F010021A804B4B1A7842F05F
:1028280001021A70002D3FF45DAE484B1D6059E659
:10283800B8F1100F7FF456AE454B1F605E600DB1C6
:10284800424B1D604248434B0222011D1A7005F09D
:10285800FCFC47E6404B1B7858073FF543AE3F4B1F
:102868004FF4C8721A803DE6324E33681B78022B4B
:102878004FF0000578D1376800F027FC07EE100A02
:10288800F8EE477AB2EE048AC7EE887A07EB850736
:10289800C7ED097A376800F018FC07EE900AB8EE21
:1028A800677ADFED2F7AC7EE277A07EB8507C7ED42
:1028B8000C7A376800F009FC07EE900AB8EE677AE0
:1028C800DFED287AC7EE277A07EB85070135032D58
:1028D800C7ED0F7ACFD1072D376817D100F0F5FB78
:1028E80007EE100AF8EE477AC7EE887AC7ED127A33
:1028F800376800F0EAFB07EE100AF8EE477AC7EEF1
:10290800887AC7ED137A00F0E0FB0DE000F0DDFBFC
:102918002F443871376800F0D8FB2F44B8733768F4
:1029280000F0D3FB2F44387601350A2DD3D1D9E5F1
:10293800041A00209804002040070108D005002050
:10294800740B0020040300209104002008030020D9
:10295800800B00207C0B0020F02000201C050020AC
:102968000000C84200007A44376800F0AEFB2F44EC
:102978003871376800F0A9FB2F44B873376800F046
:10298800A4FB2F4401350A2D3876EDD1AAE5CF2DC9
:102998002FD100F0A5FB00F0A3FB624D624EA5F815
:1029A800D00000F09DFBA5F8D20000F099FB376835
:1029B800A5F8D40000F094FBA7F8A80100F090FB5C
:1029C80000F098FB366800F08BFB00EB80004000BD
:1029D800A6F8520000F079FB85F8040100F075FBB9
:1029E80085F8060100F071FB85F8050100F06DFB24
:1029F80078E54E4B0AD91B785D073FF573AD05F0B6
:102A08007BF907F075FA04F0F1F86BE51B785907C4
:102A18003FF568AD464B1A7842F004021A7061E53A
:102A280000F053FB3F4B022883F89406E9D983F85A
:102A38009456E6E7D32D6BD100F052FBA6F8B4000C
:102A480050E5EF2D0BD1384D2E6800F049FBA6F864
:102A580056002D6800F044FBA5F8540042E5FA2D15
:102A680004D1324B1B785A07CBD551E0D62D4FD124
:102A7800002500F035FB2F4B58530235102DF8D1A7
:102A880030E50026284D06F12C07D5F800904FEACE
:102A9800C70800F025FB09EB0803D5F80090D8809B
:102AA80000F01EFB09EB0803188100F019FB07284A
:102AB80002D82B6843445873A0F57A739BB2B3F5D8
:102AC8007A7F03D82B6803EBC70358812D6800F081
:102AD800FCFA05EBC7070136082E3873D2D101E599
:102AE800002500F0FDFA144B58530235102DF8D18B
:102AF8000122124B92E700250B4B1E6800F0E5FA05
:102B080006EBC5060135082D86F86D01F4D1E9E418
:102B18000120002100F032FCE7E407B0BDEC028B95
:102B2800BDE8F08F041A002098040020F02000204F
:102B380091040020E4060020BA060020EC020020E0
:102B4800094BDFED0A7A53F8213006EE903AF8EE99
:102B5800666AB6EE047AE6EE877AFCEEE77A17EE56
:102B6800900A80B2704700BF0C02002000005C444D
:102B7800014B33F811007047BA060020014B33F8B7
:102B880011007047A00D0020032810B50F4B0DD879
:102B98000F4A126894888C4208D2D2888A4205D992
:102BA800012202FA00F01A78104318701B780F2BD4
:102BB8000BD1064B00221A70064B998808B21428CC
:102BC80002DD1439998010BD9A8010BDC80A002012
:102BD800C80D0020B4090020024B9A8801329A805F
:102BE800704700BFB4090020074B1A68074B1178DB
:102BF800B3F9040053780B4403EB83039842D4BF22
:102C080000200120704700BFC80D0020B409002033
:102C1800064B074A1B68B2F904001B7803EB8303D1
:102C28009842D4BF00200120704700BFC80D002083
:102C3800B409002010B50446FFF7EAFF002814BFC6
:102C48002046002000F0010010BD024B01221A723C
:102C5800704700BFB4090020014B187A704700BFC5
:102C6800B4090020034BB3F90400D0F1010038BFC8
:102C780000207047B4090020014B00229A80704759
:102C8800B409002003685A1C0260197070472DE9C6
:102C9800F04F514A514E17687389B28885B08446FF
:102CA80030890391A7EB032787FB00011404C209AD
:102CB80042EA4162F08814EB020872884FEAE11395
:102CC80087FB00014FEAC2344FEA1022B0894FF067
:102CD800000545EB030942EA01620B1287FB00017C
:102CE80014EB020A4FEAD05242EA41224FF00005A3
:102CF80045EB030B12F5FA604FEAE15343F100018B
:102D0800CDE90001B0F5FA6F71F1000147DAA2FBD5
:102D1800024502FB03F1052605EB4105A4FB06016C
:102D280006FB05114D104FEA3004B8EB040869EBB7
:102D38000509840844EA81748D10BAEB040A6BEB28
:102D4800050BDDE9004526484FF0FF3184428D41EF
:102D580025DA40F6AC5012184FF0000143EB01039E
:102D680002FB03F1A2FB022303EB41036FF0060011
:102D7800544200FB0344A2FB000118EB0008214465
:102D88004FF00B0449EB0109A2FB040104FB0311FA
:102D980049104FEA3000BAEB000A6BEB010B114BFC
:102DA8001A68A2FB0A0102FB0B11420D42EAC1227A
:102DB8004B15B2EB080263EB0903D00B40EA434022
:102DC800BCF1000F01D0CCF80000039808B10099BD
:102DD800016005B0BDE8F08FE80E00206207002012
:102DE80024FAFFFFEC0E002021B9022834BF00208E
:102DF8000220704702207047074B1B681B7803F0BE
:102E08007F03212B06D100F0DF0002280CBF002031
:102E18000220704702207047880F002020B9034B1A
:102E28001B6808221A82704701487047880F0020E3
:102E38004400002020B9034B1B6808221A827047FF
:102E480001487047880F002044000020212810B551
:102E580008D1114B1B681B7803F07F03212B10D07E
:102E6800022010BD2028FBD10B4B0C4A1B681070A8
:102E78001B7803F07F03212B094B18BF00230BB9E4
:102E8800EEE7084B044A00241268204693615482F6
:102E98009847204610BD00BF880F0020F32000206F
:102EA8003D2E0008252E00087047034B1A78202A6B
:102EB80004BF00221A707047F3200020014B04223F
:102EC8001A607047F8200020034B9B7A13B1034B1C
:102ED80005221A60704700BF600F0020F82000200C
:102EE800014B00221A60704760110020014B1868DE
:102EF800C0B27047A40E0020012070477047704789
:102F0800016BC268034610B5406941B1196C541A87
:102F18000139005D18BF0A46C0B21A6410BD196AAB
:102F2800405C0131914228BF0021C0B2196210BD36
:102F3800036B13B15A68036C01E0C269036A9A42D1
:102F48003BBFC0688018C3EB0200C3EB0000C0B2EF
:102F58007047436B13B190F844007047826A436A24
:102F6800D31A58425841704710F80A3C0133DBB273
:102F78000A2B00F80A3C0AD910F8123C23B910F8B9
:102F8800131C034A22F81130002300F80A3C70474A
:102F9800A00D0020334A136C90681944081A40F6B3
:102FA8008C23984210B513469160D06051603CD98B
:102FB800127893F945108A420BD1111F082908D8B5
:102FC80093F84610182901D8013103E083F844200A
:102FD80002E0002183F8461093F944108A421CD17C
:102FE800204991F84710C1B1002191421E4806DAE4
:102FF80003EB8104246920F811400131F5E7511EE3
:1030080000EB41011630814203D0002421F8024F21
:10301800F9E7164908780130087083F8452000223E
:1030280001211A7083F8471010BD92F84710B9B102
:10303800A0F2EF2440F2DA518C4208D811780B291B
:1030480005D80B1D0131117042F8230010BD002274
:1030580083F84720991804320020302A0861F9D1F2
:1030680010BD00BF38080020A00D00201C0D002056
:10307800024B1A6C01321144196470473808002059
:10308800024B53F820301B68196070476009002014
:10309800064B53F820301A681B89A1F57A714B4307
:1030A8004FF47A7093FBF0F31360704760090020C7
:1030B80038B50C68054620460AF018FE2146024637
:1030C8002868BDE838400AF019BE044B1B68DA7955
:1030D800511CD9711344187A704700BF640A002044
:1030E80010B5FFF7F2FF0446FFF7EFFF04EB0020EF
:1030F80080B210BD10B5FFF7F3FF0446FFF7F0FFED
:1031080004EB004010BDF0B5137C032B2ED80C2621
:10311800174C5E4306EB040C9CF80850284203F158
:10312800010521D0335D3BB1012B05D0022B03D023
:10313800032B14BF042303230E4C4E7B04EB031410
:10314800277B3740B7420FD14F686668B7420BD329
:103158008F68A668B74207D813709460C2F804C095
:10316800D16015741046F0BDEBB2CEE70020F0BD7B
:10317800140000206008010800230549595C8142B9
:10318800DAB203D001330A2BF7D11A46104670473A
:103198002B1D0108094AA2F13003197A81420BD08C
:1031A8000C339342F9D1064B197A014004D10C3300
:1031B8009342F9D1084670471846704744000020EA
:1031C800140000202DE9F0478278C6781F4BC2F121
:1031D800640802EB820C54425FFA88F84FEA4C0C00
:1031E800C6F16409A4B203F11807A0B20FFA80FA75
:1031F800BAF1000F04DC002814BF1546012500E0D1
:10320800454610FB00F0704315FB05F590FBF5F5FE
:103218004D4405FB0AF50A2095FBF0F56544ADB26F
:103228005D800888B1F802A02DB2C0EB0A0A05FB40
:103238000AF54FF47A7A95FBFAF5284423F8020F39
:103248000A34BB42A4B2D0D1BDE8F0871E0A0020E0
:1032580010B544780078002303FB03F11939614362
:1032680001F6C411594340F6C412414391FBF2F1EF
:10327800034A22F813100133072BEDD110BD00BF0C
:10328800080A002010B5044C2068FFF7E1FF206809
:103298000249BDE8104095E7D0050020D41A002067
:1032A80010B5094A094913688C6812689342F8D125
:1032B800074A106811684FF47A725043001BB0FB3C
:1032C800F1F002FB030010BD001A002010E000E03E
:1032D8001007002038B50446FFF7E2FF0F4B5A6885
:1032E8005860821A40F6C4118A4284BF00221A72BA
:1032F8001A7A0AB90F2C0FD10948002101704AB176
:10330800084D1544182A05F8014C03D101221972F9
:10331800027038BD01321A7238BD00BFC80A0020D9
:10332800F1010020F201002008B503681B699847E5
:1033380008BD08B50368DB68984708BD08B5036889
:103348009B68984708BD08B503685B68984708BD3F
:1033580008B503681B68984708BD064B10B50446B6
:1033680021461868FFF7F4FF034B1B689A7954400D
:103378009C7110BD680A0020640A002038B5044614
:1033880024200D46FFF7E9FF4D20FFF7E6FF002C4C
:10339800084C0CBF3E202120FFF7DFFF23680022E6
:1033A80028469A71FFF7D9FF236893F84900BDE8CA
:1033B8003840D2E7640A002001460020DEE7F8B56D
:1033C8000C4E0D4C0D4DC1B2074630686172FFF7C7
:1033D800BFFF2B68617A9A7930684A409A71C7F3BF
:1033E80007216172FFF7B4FF2B68617A9A794A4026
:1033F8009A71F8BD680A0020C80A0020640A0020F3
:10340800F8B5174D174C184F0646C1B22868A17277
:10341800FFF79EFF3B68A17A9A7928684A409A711B
:10342800C6F30721A172FFF793FF3B68A17A9A7947
:1034380028684A409A71C6F30741A172FFF788FFCE
:103448003B68A17A9A7928684A409A71310EA1722C
:10345800FFF77EFF3B68A17A9A794A409A71F8BDD6
:10346800680A0020C80A0020640A002010B5441E1B
:1034780014F8011F21B1034B1868FFF769FFF7E73C
:1034880010BD00BF30080020014B186860E700BF7E
:10349800380F0020054B1B6803EBC00090F906307D
:1034A80019420CBF01204FF0FF307047A0060020E2
:1034B8000A4B1A6802EBC002D379FF2B07D00849E0
:1034C8000978994203D9074A32F8130004E007281B
:1034D800D4BF908840F2DC5000B27047A0060020AC
:1034E800CB090020BA06002038B52DED0A8B91EDE6
:1034F800008A90ED00AAD0ED01AA90ED029AB0EEF4
:10350800480A04460D460AF0DFFDF0EE409AB0EE98
:10351800480A0AF05FFE95ED018AB0EE40BAB0EEB7
:10352800480A0AF0D1FDF0EE408AB0EE480A0AF0E7
:1035380051FE95ED02CAB0EE408AB0EE4C0A0AF090
:10354800C3FDF0EE40BAB0EE4C0A0AF043FE6BEE53
:10355800005A2BEEA97AB0EE655AA7EE485AA5EEA6
:10356800C87A20EE296A6BEE2B7A2AEE877A28EE43
:10357800C00AF0EE466AE7EE886AAAEE007AE6EE3E
:10358800087A6BEEA8BAA9EE277A6BEE687A6AEE2B
:10359800A66A6AEEA77AEAEE2B6AEAEE087A68EE7D
:1035A800A98AE9EE056AE9EE287ABDEC0A8BC4ED32
:1035B800006A84ED017AC4ED027A38BD38B5294D28
:1035C8002DED048BD5ED008AB0EE680A04460AF0AA
:1035D8007BFDB0EE408AB0EE680A0AF0FBFD95ED7F
:1035E800019AF0EE408AB0EE490A0AF06DFDF0EE5D
:1035F800409AB0EE490A0AF0EDFDD4ED017AD4ED17
:10360800026A67EEA80AB0EE407A60EE870A28EEF2
:10361800E60A66EE876A94ED007AE7EE290AA7EED5
:10362800880AE6EE880A0AF071FEDFED0F7A9FED50
:103638000F7A0F4B20EE270A80EE070A93ED007AE7
:1036480030EE070AB2EE047A80EE070A0AF078FD37
:10365800BDEC048B83B21A0444BF00F5B4739BB26B
:1036680018B238BD7C0500200000E144DB0F49405A
:1036780074070020034B1A78510744BF22F0040254
:103688001A707047F020002070B5FFF7C1FA38B300
:10369800144C237A0BB9A38070BD134D2E78C6F352
:1036A8008000FFF7C7FA90B1104B1A68104B518988
:1036B80019805189598052899A800E4A1268528815
:1036C800DA80E38846F0020601332E70E380FFF7C4
:1036D8008BFA10B92B785B0702D4BDE87040C9E7B4
:1036E80070BD00BFB4090020F0200020B009002000
:1036F800BA060020C80D002010B50278202A03461B
:1037080000F10100F9D0092AF7D02D2A03D1034688
:10371800BFEE000A04E02B2A08BF0346B7EE000AF2
:103728009FED377A1A46134612F8011BA1F13000B3
:10373800C4B2092C0AD805EE900AF8EEE57AF2EE42
:10374800046AE7EE267AB0EE677AECE72E2915D1FF
:10375800F2EE047AF0EE676A134612F8011B30396C
:10376800C8B209280AD805EE901AB8EEE56A86EEBE
:10377800276A67EEA67A37EE067AEDE71A7802F03E
:10378800DF02452A34D15A782D2A02D10233012288
:1037980004E02B2A14BF013302330022013B00212D
:1037A80013F8010F3038C4B2092C03D80A2404FBDB
:1037B8000101F5E7B1F59A7F34BF0B464FF49A73D0
:1037C8001946F7EE007A072905D9DFED0E6A0839A0
:1037D80067EEA67AF7E703F007032BB1F2EE046A67
:1037E80067EEA67A013BF8E722B1C7EE277A03E035
:1037F800F7EE007A67EE277A20EE270A10BD00BFA1
:103808000000000020BCBE4CF0B50124B0FBF4F56C
:103818008D4201D34C43F9E70026DCB1B0FBF4F547
:1038280004FB1500B4FBF1F41EB9002D01DC002CDB
:10383800F3D1092D03F101075FFA85FC04DD002AA5
:103848000CBF5725372500E0302565441D7001362B
:103858003B46E2E71C70F0BDF0B50124B0FBF4F57F
:103868008D4201D34C43F9E70026DCB1B0FBF4F5F7
:1038780004FB1500B4FBF1F41EB9002D01DC002C8B
:10388800F3D1092D03F101075FFA85FC04DD002A55
:103898000CBF5725372500E0302565441D700136DB
:1038A8003B46E2E71C70F0BD70B50646B6FBF2F485
:1038B8000846154614B12046FFF7F6FF05FB1464C9
:1038C800024B1B5D00F8013B70BD00BFBB1C01082B
:1038D8002DE9F041069C002B06460F460CBF4FF021
:1038E80020084FF03008234613F8011B09B9154684
:1038F80003E0002AFBDD013AF6E7002D04DD30463F
:103908004146B847013DF8E714F8011B11B13046AC
:10391800B847F9E7BDE8F08180EAE073A3EBE0730C
:103928008B4206DB002801DD401A704702D00844AC
:10393800704700207047034B9A6822EA000098609D
:10394800704700BF041A002008B506480AF0CEF9EF
:10395800C0B2142805D8034A431C20211154D8B2F8
:10396800F7E708BD410F002010B5121A07EE902A9C
:103978005B1A2DED028BF8EEE78A07EE903A184BAA
:10398800059CB8EEE78AD3ED007A28EE278A28EE60
:10399800080AA8EEA80A0AF05FFEDFED127A049B77
:1039A80020EE270AF0EE480AFCEEC07AB1EE680A6B
:1039B800C3ED007A0AF0AAFCDFED0B7A9FED0B7AD3
:1039C800E0EE077ABDEC028BFDEEE77A17EE903A4F
:1039D800002BBCBF03F50C43A033236010BD00BF10
:1039E800D00000202C7D8E3F00A00C46A00CB345D3
:1039F80007EE100AF8EEC77A9FED0A0A9FED0A7AD9
:103A0800F5EEC07AF1EE10FAD8BFF1EE677A87EEDC
:103A1800800A08B520EE070A0AF056FB034B83ED2F
:103A2800000A08BD8096184B35FA8E3CD00000205D
:103A38000179DFED2A7A827B294B07EE101AB8EE5E
:103A4800477AF2EE046A87EE277A83ED007A07EE6A
:103A5800102AB8EE477A234ADA6087EE277A83ED90
:103A6800017A4179204B07EE101AB8EE477AC17BEC
:103A7800DA6087EE267A83ED007A07EE101AB8EE40
:103A8800477A417E87EE277A06EE101A83ED017A8F
:103A9800B8EE466A9FED157A86EE076A83ED026AEC
:103AA8008179134B06EE101AB8EE466A017C807EC7
:103AB800DA60C6EE266AC3ED006A06EE901AF8EEE2
:103AC800666AC6EEA77AC3ED017A07EE900AF8EEA9
:103AD800677A87EE877A83ED027A70470000C842DA
:103AE800600E00200000FA44700E002000007A44A6
:103AF800940E002044F25063984203DDA0F50C4078
:103B0800A0387047034B9842BCBF00F50C40A0306A
:103B1800704700BFB0B9FFFF013101EB420291428B
:103B28000BD0030F092B94BF3033373301F8013C16
:103B38000023000101F8023BF1E770472DE9F0414D
:103B48000369C76804460D461F40002F33D0B7FAF3
:103B580087F34FF00042DA40D2431B3B2261174003
:103B6800042BF2D8DFE803F0211E1B1803006B6A50
:103B780033B103F1FF3800231FFA88F86B6202E0C3
:103B8800E36A1FFA83F82E6A002EDED033683046C7
:103B9800414698477668F7E72868616B07E06868E8
:103BA800A16B04E0A868E16B01E0E868216C036898
:103BB80089B29847C9E7BDE8F0810E4B800A984260
:103BC80010D007D8B0F5801F12D04A3B98420DD1CB
:103BD80002207047084B984206D00233984205D11C
:103BE800042070470020704703207047FE2070476C
:103BF800012070474B00100050001000044B53F890
:103C080020301BB107289CBF1B681960704700BF94
:103C18009009002010B5054C00202188FFF7EEFF21
:103C280061880120BDE81040E8E700BF38010020A6
:103C3800054B98420CBF054B054B1A88013292B2CE
:103C48001A800020704700BF005400406C0A002012
:103C58006E0A0020A54AA64913682DE9F04F03F51E
:103C68009C43A44D20330B60AB6813F4807F85B070
:103C7800174604D0A04B1B681B681B699847AB68A4
:103C880042F201041C405CB99C4E337873B19A4BE4
:103C98001B681B681B68984702F018F8347005E029
:103CA800974B1A7801321A7002F010F8AB68DA04F0
:103CB80005D5944B1B68DB0701D4FFF7DBFC924B5F
:103CC80039681C68237CFBB1904A013B32F91330F8
:103CD800A3F57A73B3F57A7FA8BF4FF47A7323EA12
:103CE800E37307EE903AB8EEE77ADFED897A844B12
:103CF800C7EE277A9FED877A67EE877AFCEEE77A38
:103D080017EE902A5A803BE0AA68170438D57C4AF7
:103D18005068081A002833DB01F59C4020301689CA
:103D28005060607CB6B296FBF0F4107C013000F075
:103D38000F001074024454741A46714800F11104BB
:103D48001C5D01332244102B92B2F6D112B292FBC1
:103D5800F3F31BB2642BA8BF642323EAE37307EED3
:103D6800903AB8EEE77ADFED6C7AC7EE277A9FEDE6
:103D7800697A67EE877AFCEEE77A17EE903A438025
:103D8800AB68DE0510D5654B654C994208D92368A8
:103D98001B681B6A984718B923681B685B6A9847B1
:103DA80023681B685B699847AA68524BB5F8DC1012
:103DB800D4040AD55548B3F81A31B0F90620581A70
:103DC80082420ADD19448A4205E05049B3F81C31A1
:103DD800B1F906209A42C0F253840122002395F8D3
:103DE80023A195F82411B5F81C41B5F81E619B462E
:103DF800464FF85E4FEA9B0BA042C4BF6BF07F0BA7
:103E08005FFA8BFB0233B042B8BF4BF0400B082B74
:103E1800EED13B4C94F821305B4505D194F8223023
:103E2800F92B04D8013300E0002384F822303D4BFD
:103E380084F821B093F80080324F9946B8F1000F0A
:103E480014D13B68D80707D582B9374B1B78DB07F5
:103E58000CD506F011F809E0334B1B785E0705D541
:103E680011B1FFF707FC01E0002AFAD094F82230DC
:103E780023492E4E142B40F098802B4B1B781AF1B7
:103E8800000A03F0040318BF4FF0010A03F0FF0211
:103E980083B1B8F1000F00F08880BBF15F0F02D149
:103EA800FFF7E8FB81E0BAF1000F7ED0BBF17D0F90
:103EB8007BD1F5E7BBF1570F0BD11D4B4FF47A724D
:103EC8001A801C4B1B6813F008036ED11A4A138022
:103ED8006BE0AB68580741D5BBF15A0F3ED1174B81
:103EE800187878B31A700122154B4CE0D8200020BE
:103EF800F4020020041A0020F0020020E80100204B
:103F0800040B002000030020EC010020BA0600206A
:103F180000007A4400C07F440000C842404B4C0077
:103F2800C009002060000020F02000209804002034
:103F3800E8200020FC020020900500204905002010
:103F48004B05002091F82320AD4B82F0010281F847
:103F580023200AB1042216E0062214E0BBF15D0F0B
:103F680000F01083BBF15B0F00F00E83BBF15E0F16
:103F78000BD1032209E3BBF1A70F40F02683A14B25
:103F88001A7842F004021A700FE0BBF1560F01D103
:103F980002F0E6FF99F80030002B00F00D83BBF12A
:103FA8006F0F40F0028305F067FFAB685B0734D5FD
:103FB80094F82330ABB1944B1B78580711D593482C
:103FC800934BB0F90620B3F81C319A4209DD3B68DF
:103FD80013F0010305D18F4A322111808E4A82F8ED
:103FE80023303B68D9030AD58C4B1A782AB98C4AF6
:103FF800127812B9874A3221118001220CE0884BCD
:104008001A7852B1804A127802F0040202F0FF01D5
:104018001AB91970834B01221A70D6F80090002340
:1040280009F1750A3B6009F1770698460AF102031F
:1040380003EB080113F808204B7816F8010C9A4294
:104048000AD2314601F09AFF30B116F8023C01223B
:104058009A403B6813433B6008F10408B8F1A00F8D
:1040680006F10406E2D1704B1B7843B13B68DFF8D8
:10407800CC816E4E13F0020F40F0A28197E109F255
:104088001512019209F58B769846019A16F8010CDB
:10409800531C03EB080113F808204B789A4229D2E5
:1040A800314601F06BFF28B396F802C0604B3079B7
:1040B80096F803B00CF1FF3C0CEB4C0C9C44564BAF
:1040C8004FF00C0903F1240A09FB00F90AEB090176
:1040D8004A6862450ED000220AF809B08A600122B7
:1040E80002FA00F093F85420C1F804C022EA000054
:1040F80083F8540008F10608B8F1480F06F10606DF
:10410800C3D14C4B4C4A1E68D2F800A0DFF830816E
:104118004FF000099B46D8F80030002B00F03E8194
:104128001978002900F03A81D8F80420C2EB0A0275
:10413800002A0CDB0AF5FA7294F85400C8F8042037
:10414800012202FA09F220EA020284F8542018F83F
:10415800040C5A780430C0B2002A40F0E6802B4A9A
:1041680032F910000190B5F81A01019A00F1C80C53
:10417800624501DD9B7814E0019AC838824202DA70
:104188009B785B420DE094F85420012303FA09F36D
:1041980022EA030384F854300AF5FA73C8F80430A5
:1041A800FCE094F8542042FA09F2D20700F1F680B4
:1041B800002B134ACCBF02200120013910700A29B4
:1041C80000F2E480DFE801F0060F3E4B545D6F819A
:1041D800939DA70032781344FA2BA8BFFA2323EA49
:1041E800E373337007E072781344642BA8BF642329
:1041F80023EAE37373703046FFF72AF8C6E000BF7E
:104208004A05002091040020F0200020BA06002072
:10421800041A002030050020040B00204805002067
:10422800490500204B050020F4200020040300204D
:10423800A0080108D0050020001A0020FC02002078
:104248002C0B0020F2781344642BA8BF642323EAC4
:10425800E373F3703046A16DFEF7B4FF96E0327950
:104268001344642BA8BF642323EAE37333718DE0FE
:1042780072791344642BA8BF642323EAE373737130
:1042880084E0E16D4A781A44C82AA8BFC82222EA05
:10429800E2724A700A781344C82BA8BFC82323EADD
:1042A800E3730B7072E0E16DCA7A1A44C82AA8BF9A
:1042B800C82222EAE272CA728A7A1344C82BA8BFBB
:1042C800C82323EAE3738B7260E0E16D4A7D1A44E8
:1042D800C82AA8BFC82222EAE2724A750A7D134496
:1042E800C82BA8BFC82323EAE3730B754EE0E26D21
:1042F80091780B44C82BA8BFC82323EAE3739370B3
:1043080044E0E26D117B0B44C82BA8BFC82323EA05
:10431800E37313733AE0E26D917D0B44C82BA8BF99
:10432800C82323EAE373937530E0012A2ED19B78E2
:104338004FF4966292FBF3F3AE4A32F91000B0F5EF
:10434800617F05DB40F633029042B8BF024601E0C8
:104358004FF46172A2F5617292FBF3F3DBB2A64AE5
:10436800581C0C29107011D194F860209A420DD075
:10437800042BA24A28BF02230A2184F8603001FBDB
:1043880003230633CBF80030FEF77CFF94F8542063
:10439800012303FA09F3134384F8543009F101099E
:1043A800B9F1040F08F10C087FF4B5AE5EE6AB680E
:1043B800D80514D5924B1B681B689B68984770B149
:1043C800D8F800309B070AD5328812F001030CD1C7
:1043D8008C49636642F00102A3660A8006E03388CE
:1043E80023F001033380012300E000233A685107DA
:1043F80010D57BB1338823F0010103F0020389B2A1
:104408009BB2318053B96366A3667E4B41F00201CB
:10441800198003E0338823F00203338033887A4914
:1044280013F0030F4FF020000CBF88610885D8F8FF
:104438000010880640F1918074490978890753D59E
:104448007349097804294FD912F4007C11D0DA068F
:1044580053D4704823F0200343F010033380011D28
:10446800012384F86C3003F0F0FE022384F87830DE
:1044780043E023F0100189B25005318030D5664AF7
:1044880012685089654AB2F90080B8F1000FB8BFC8
:10449800C8F10008804509DAB2F90220002AB8BF3D
:1044A80052428242ACBF0022012200E06246D2079B
:1044B80016D59B0621D45A48D4F88430E36741F0D6
:1044C800200131804FF00108D4F8883084F86C80DE
:1044D800011DC4F8803003F0B8FE84F878800CE041
:1044E80023F03003338008E023F0300333800023C7
:1044F80084F87830012384F86C3094F86C3063B316
:1045080000210A464748484C00231352474804F103
:104518008C0C135246488C4413520020CCF80000EF
:10452800CCF80430CCF8080004F1B40C8C44023206
:10453800CCF80000CCF80430CCF8080004F1DC0C0E
:104548008C44042ACCF80000CCF80430CCF80800DD
:1045580001F11401D6D184F86C303B6813F4006F74
:10456800338814BF43F4807323F4807333806B79EA
:10457800082B02D00E2B40F09680338823F040039E
:10458800338090E0012200E002225FFA82F808F10D
:10459800FF3385F8943605F0ABFC02F027FB0220C8
:1045A8002821424605F046FCFFE4BAF1000F03D08B
:1045B800BBF17E0F3FF4F7ACBBF1970F7FF4DBAC98
:1045C8001C4B4FF4C8721A80EFE40023BBF1BB0FF9
:1045D800039301D1022304E0BBF1B70F04D14FF6D6
:1045E800FE73ADF80E302FE0BBF1BE0F24D10223CD
:1045F80028E000BFBA0600204A05002094200020C9
:10460800C009002004030020000400489104002091
:1046180090040020740B0020C40500201203002021
:10462800800B0020DC200020040B0020C80500209F
:10463800CC0500201C050020BBF1BD0F7FF4B5ACF4
:104648004FF6FE73ADF80C303368BDF80C10B3F8B4
:1046580054200A44A3F85420BDF80E10B3F856208D
:104668000A44A3F8562005F043FC02F0BFFA0F20D5
:104678001421012205F0DEFB002384F8223094E4A3
:104688000A4B002200215A669A66C3F80421C3F82F
:104698000821C3F80C21C3F81011C3F81411C3F88A
:1046A8001811FFF79BBB05B0BDE8F08F040B002085
:1046B800704730B5094B1A68D378042B0CD8084CCE
:1046C800518A04EBC30518B9AB88591A118230BD59
:1046D80054F83300084430BD002030BD880F002056
:1046E800B000002010B5214B18B91B6802221A82AD
:1046F80010BD1F4A1968002010800C7814F07F0440
:1047080013460DD14A7A910644BF0221197012F05E
:10471800400F1A7814BF42F0010222F0010215E09E
:10472800012C20D0022C1FD14A7912F0800F02F000
:104738000F024FEA820202F1804202F5B842126883
:1047480006D002F03002102A07D101221A7004E0C4
:1047580002F44052B2F5805FF6E7064B1B681B690E
:104768009847034810BD104610BD00BF880F0020B1
:10477800300C00208C0F002010B5064C18B92368A7
:1047880001221A8210BD044B1B689B689847206859
:104798000C3010BD880F00208C0F002010B5064C7F
:1047A80018B9236801221A8210BD044B1B681B68C4
:1047B800984720680A3010BD880F00208C0F002011
:1047C800204B1A782DE9F0471E4622B31E4B90F86D
:1047D80000C01F781D4B93F8008002231C4AD5188F
:1047E80003F1010AAC783C4104F00F0464450DD292
:1047F8000B2C0BD895F8029002EB0A0502EB840209
:10480800AD7809EA080405EB042454610233102B3F
:10481800E4D10023337003788B420FD90C4B93F803
:10482800440060B10B4A89000B441278586902B100
:10483800400800F5777080B2BDE8F0870020BDE839
:10484800F08700BFF0010020C8090020C909002036
:10485800300C0020CA09002007299ABF024B33F800
:1048680021000020704700BFCC020020024B53F803
:104878002100C0F3CF0070477402002038B5114CF6
:10488800012384F844300546FEF70AFDA36CA064B2
:10489800C31A41F288329342E36484BF002384F848
:1048A800503094F850301C44EDB20F2BA57003D152
:1048B800054B01221A7038BD024A013382F8503084
:1048C80038BD00BF300C0020F001002010B50446B0
:1048D800FEF7E6FC0D4B5A6D5865821A41F2883195
:1048E8008A429A6584BF002283F85C2093F85C3082
:1048F800074A142BD45403D1064B01221A7010BD59
:10490800024A013382F85C3010BD00BF300C002031
:10491800B5020020B402002010B50446FEF7C0FC22
:10492800164A136E1066C31AB3F57A6F84BF002354
:1049380082F8643092F8643023B9A82C1DD110494C
:104948000B7006E0022B02D10E490C7001E0242BFB
:1049580001D80D49CC540133DBB282F86430094ADE
:104968001178052202EB4102934206D1034B002243
:1049780083F86420024B01221A7010BD300C00200D
:104988004C020020720200204D0200203D4B1B7893
:10499800012B30B50CBF03230023B1B9016A21F004
:1049A800010101628469016A24F0F30444F00104FE
:1049B80021F00A0142F0010244EA03130A43836129
:1049C8000262836923F00C031BE00429046A1CD1EA
:1049D8004FF6EF71214001628169046A21F4734145
:1049E80041F48071120141EA033342F010024FF69C
:1049F8005F71214092B2114383610162836923F49C
:104A0800406383618369836130BD08291AD14FF6F9
:104A1800FF6121400162C469016A89B2A4B221F42C
:104A2800206124F0F30441F4807144F0010441EA68
:104A3800022244EA031392B2C3610262C2694FF6CA
:104A4800F37319E04EF6FF7121400162C569046AEB
:104A580040F6FF41294041F4807545F6FF71214039
:104A680041F4805444EA023245EA033392B2C36106
:104A78000262C2694FF2FF331340C361C369C36165
:104A880030BD00BF34080020084BDA68D10709D4CC
:104A9800DA68D20608D4DB6813F0040F0CBF0420D0
:104AA8000320704701207047022070470020024011
:104AB80002684FF6FE7313400360002303604360EF
:104AC8008360C3602A4B984222D02A4B984229D04F
:104AD800294B984230D0294B984237D0284B9842DE
:104AE8003ED0284B984206D153F8682C42F4700205
:104AF80043F8682C7047244B984206D153F87C2C15
:104B080042F0706243F87C2C7047204B984206D1E3
:104B180053F8042C42F00F0243F8042C70471C4B46
:104B2800984206D153F8182C42F0F00243F8182C9A
:104B38007047184B984206D153F82C2C42F47062F7
:104B480043F82C2C7047144B984206D153F8402C4C
:104B580042F4704243F8402C7047104B984205D1FC
:104B680053F8542C42F4702243F8542C704700BF79
:104B7800080002401C00024030000240440002408D
:104B8800580002406C0002408000024008040240C5
:104B98001C0402403004024044040240580402400D
:104BA8000D4B1B689BB203EBC0000C4B3E29034422
:104BB8004FEA430209D94B09C80604BF03F1FF3382
:104BC8009BB29B0243F4004304E04B08C90748BF6B
:104BD80001339B0213607047505C00400630002090
:104BE80010B5444B1B68187810F07F0004D15A7A2E
:104BF80022F020025A7210BD022878D15A88002A61
:104C080076D11A79002A73D15A7922F0800084006B
:104C180004F1804101F5B84112F0800F096814BF12
:104C280001F0300101F44051032860D800295ED01A
:104C38009B7A002B5BD004F1804404F5B84411063C
:104C4800236824D503F03003102B4AD102F07F03E8
:104C58009B0003F1804303F5B8431A68520608D550
:104C6800196840F60F720A4042F4004242F0C0024E
:104C78001A601A6822F4E04222F0400292B282F0EE
:104C8800300242F4004242F080021A6029E003F444
:104C98004053B3F5805F24D128B9174B93F82C10F3
:104CA800FFF77EFF10E0920002F1804202F5B84261
:104CB80013685B0408D5116840F60F730B4043F482
:104CC800404343F080031360236823F4804323F0B8
:104CD80070039BB283F4405343F4004343F08003D2
:104CE8002360064B1B685B699847002010BD0220B3
:104CF80010BD00BF880F0020E40000208C0F0020AA
:104D080008B50B4B002093F82C10FFF749FF094B0F
:104D18001B68187A082806D1074B4FF480521A806E
:104D2800064B10221A80B0F109035842584108BDB9
:104D3800E4000020880F0020820F0020840F00204C
:104D480030B5002303F1805202F5B852940043F4C1
:104D58000041256840F60F7241F080012A40013376
:104D68000A43042B2260EDD1024B40F0800018600A
:104D780030BD00BF4C5C0040AD4A516801F00C01E9
:104D880004292DE9F04305D0082906D0A94B036072
:104D9800B9B917E0A74B036013E053685468C3F32D
:104DA8008343E60303F1020301D4A34906E0D16A71
:104DB800A04C01F00F010131B4FBF1F1594301603E
:104DC80000E000215368DFF874C2C3F303131CF832
:104DD80003500368EDB223FA05F444605668C6F33D
:104DE80002261CF8067024FA07F787605668C6F38F
:104DF800C2261CF80660F6B2F440C460D2F82C90C3
:104E0800C9F3041909F00F080CEB480819F0100F42
:104E1800B8F810801FFA88F807D0B8F1000F04D04E
:104E2800B1FBF8F8C0F8108000E00361D2F82C80DC
:104E3800C8F3442808F00F090CEB490C18F0100FC0
:104E4800BCF810C01FFA8CFC07D0BCF1000F04D0CE
:104E5800B1FBFCFCC0F814C000E04361D2F830C0DC
:104E68001CF0100F06BFDFF8CCC1C0F818C0836172
:104E7800D2F830C01CF0200F06BFDFF8B8C1C0F868
:104E88001CC0C361D2F830C01CF0400F06BFDFF869
:104E9800A4C1C0F820C00362D2F830C01CF4807FDF
:104EA80008D08B4206D1AE4204D14FEA430CC0F879
:104EB80024C000E04462D2F830C01CF4805F08D0FF
:104EC8008B4206D1AE4204D14FEA430CC0F828C049
:104ED80000E08462D2F830C01CF4007F08D08B4216
:104EE80006D1AE4204D14FEA430CC0F82CC000E012
:104EF800C462D2F830C01CF4806F08D08B4206D14F
:104F0800AE4204D14FEA430CC0F844C000E0446408
:104F1800D2F830C01CF4006F08D08B4206D1AE42E4
:104F280004D14FEA430CC0F848C000E08464D2F8CA
:104F380030C01CF4005F06D08B4204D1AE4202D1CF
:104F48005900C16400E08464156B3949AD0701D18B
:104F5800046315E00C6B04F00304012C01D1036316
:104F68000EE00C6B04F00304022C02D14FF4004154
:104F780005E0096B01F00301032901D12D49016303
:104F8800146B2B4914F4403F01D1476318E00C6BB4
:104F980004F44034B4F5803F01D1436310E00C6B56
:104FA80004F44034B4F5003F02D14FF4004106E068
:104FB800096B01F44031B1F5403F01D11D4941630E
:104FC800146B1B4914F4402F01D1876318E00C6B54
:104FD80004F44024B4F5802F01D1836310E00C6BF6
:104FE80004F44024B4F5002F02D14FF4004106E048
:104FF800096B01F44021B1F5402F01D10D498163BE
:10500800146B0B4914F4401F01D1C76320E00C6BEB
:1050180004F44014B4F5801F01D1C36318E00C6B8D
:1050280004F44014B4F5001F0AD14FF400410EE017
:105038000010024000127A0000093D0062000020C2
:10504800096B01F44011B1F5401F01D11149C16349
:10505800126B114912F4400F02D10764BDE8F083C6
:105068000A6B02F44002B2F5800F0FD00B6B03F409
:105078004003B3F5000F02D14FF4004306E00B6B79
:1050880003F44003B3F5400F01D1024B0364BDE8BC
:10509800F08300BF00127A0000100240F0B5002330
:1050A8000E681A460125954005EA0604AC422ED141
:1050B8000D796F1E012F1AD887684FF0030C0CFA70
:1050C80003FC27EA0C07876091F805C087680CFA8B
:1050D80003FC4CEA070787608788BFB227EA040405
:1050E80084808C79878894403C43A4B284800324CC
:1050F80007689C40E4432740076007689D403D439C
:105108000560C5682C40CD799D402C43C4600132B0
:10511800102A03F10203C5D1F0BD73B506460D464A
:10512800002401232A88A34013421AD00093AB78A5
:1051380003F003028DF80420EA78022A03D0032A38
:105148000CBF032201228DF805203046C3F301125B
:105158006946C3F381038DF806208DF80730FFF701
:105168009DFF0134102CDCD102B070BD38B52DED97
:10517800048B4A4B0C460168C3F866108188A3F873
:105188006A10013A072A42D8DFE802F0040A101828
:1051980022292F35B3F866202280B3F8682013E05F
:1051A800B3F868202280B3F8662005E0B3F86620DB
:1051B80052422280B3F86820524205E0B3F86820D2
:1051C80052422280B3F866206280B3F86A301DE04C
:1051D800B3F8662052422280B3F8682012E0B3F890
:1051E80068202280B3F866200CE0B3F8662022809D
:1051F800B3F8682005E0B3F8682052422280B3F87B
:10520800662052426280B3F86A305B42A380244B26
:105218001B78002B3FD1B4F90210224DB4F90030AD
:1052280095ED030AD5ED007A09EE101A08EE903ACA
:10523800B8EEC99AB4F90430F8EEE88A29EE000A03
:1052480008EE103AA7EEA80AB8EEC88AD5ED067A95
:10525800A7EE880A08F074FF95ED040AD5ED017AE7
:10526800208029EE000AA7EEA80AD5ED077AA7EE56
:10527800880A08F065FF95ED050AD5ED027A608089
:1052880029EE000AA7EEA80AD5ED087AA7EE880A43
:1052980008F056FFA080BDEC048B38BD300C002010
:1052A80010000020280700201B4B1C4893F86C2096
:1052B8004078511C83F86C1002F00702184903EB80
:1052C800420331F81010A3F86E1000231A4615494E
:1052D800595A02330A44102B92B2F8D1D20806EE7A
:1052E800902ADFED117A9FED117A114BF8EEE66AFC
:1052F8001B6866EEA76A1B78C6EE876A07EE103A47
:10530800B8EEC77A0B4B66EE877AFCEEE77A17EEB3
:10531800902A1A70704700BF300C0020200C002023
:105328000C0B00209E0C00203333534000F07F45C7
:10533800000A0020040A00202DE9F04F8BB00893E2
:10534800864B0592B3F90220B3F900300090002B88
:10535800B8BF5B42002AB8BF52429A42B8BF1A4649
:105368007F4B01921B8803F00302049203F00202B0
:1053780003F0010392B20393002306929A461A4659
:105388001846029398461946049C002C3FD00229DF
:105398003DD0724C165B734CA45E022516FB054487
:1053A800059D6F42BC4203DB2F46BC42B8BF27466F
:1053B8006D4C165F009CBE1B089FBD5E009F2E446F
:1053C800E5796424754395FBF4F5FC7E6FF00407DA
:1053D80007FB04F8454505DB04EB8404A542B4BF8C
:1053E800A846A046614D049F5C59344442F21076A9
:1053F800B442A8BF34465E4EB442B8BF3446009E9D
:105408005C51757C6C432413012F02943ED0594D96
:10541800DDF800C0AD5E5148574C1CF80170805E45
:1054280053F804C085EAE576A6EBE576B6F5206F75
:105438001EDC022916D000EB8004240194FBF7F748
:10544800042495FBF4F57F1BBC444B4E4B4CBCF538
:105458007A5FA8BF4FF47A5CA445ACBF43F806C096
:105468009C5107E080EAE076A6EBE076642EE2DD68
:105478000025E550404C1D597D2495FBF4F5009C12
:105488000C44A47A6543402495FBF4FA069CBCB10D
:1054980002295FD0DDF804C0019E0CFB0AF7DDF895
:1054A80008C0C6F5FA7506FB00F405FB08444FF47E
:1054B800FA7605FB0C7594FBF6F495FBF6F506E019
:1054C800039C002C46D0022944D0029D4446294E14
:1054D800975B4FF004090FFA87FC9CFBF9F60996D5
:1054E800274E8E5D0796274E32F906B0975306F180
:1054F8000807CBEB0C0C14369CFBF9FC53F807900F
:1055080053F806B043F806901F4E43F807C08E5D67
:105518001E4FCB44E34406FB0BFB20269BFBF6FB0C
:10552800CBEB050BDDF824C0079D0CFB05F96FF0EC
:105538004F0599FBF5F9A1440131CB44032922F821
:1055480007B003F1040302F102027FF41DAF0BB0B0
:10555800BDE8F08F55460446B9E700BF12030020A6
:1055680004030020DC2000205C040020680B0020DD
:10557800F0D8FFFFA4050020080C002080C1FFFF21
:10558800160A0020B00C00201C0A0020D4050020B8
:105598002DE9F04F89B006460793564B0291B3F9AF
:1055A80004300393544B01921B8803F0010103F06C
:1055B80002039BB20493514B0691B3F800A04FF637
:1055C800FF714FEA1A13B1FBF3F1002305911D4651
:1055D8001946022D08D1029CDDF80CC067791B37EB
:1055E8000CFB07F77F1132E0424CDFF828C10C5B57
:1055F8003CF901C0019A4FF0020827B2C2F1000934
:1056080014FB08C44C4503DB91464C45B8BFA14682
:105618003B4CDDF81CC00C5F069AC4EB09093CF949
:105628000140A1447AB9029C049A94F804C00CF190
:105638001B0C07FB0CF73F114AB1447C04FB09F92A
:1056480007EB292703E0C77907FB09F73F112D4C22
:10565800DFF8C48031F904C096F80AB010F8059054
:1056680004249CFBF4FCCCEB070C0AFB0CF453F869
:105678000870E4120BFB0474234FB4F5001FA8BF95
:105688004FF40014BC42B8BF3C46204F43F80840D2
:10569800DA5943F807C0C2EB0C0809FB0CF9DDF82E
:1056A80014C00CFB08F807F10C0C183753F80CB0B1
:1056B800DA59934453F80C20DA514FEAA818377D89
:1056C80043F80C80C34407FB0BF73F1207EBE917BD
:1056D80007EB643401350E4F032DCC5306F1010658
:1056E80001F1020103F104037FF473AF09B0BDE8CF
:1056F800F08F00BF1203002004030020AC05002037
:105708005C040020A40500200000E0FFD00C00206D
:10571800D4050020DC200020080C0020F7B51E4B23
:105728001A680AB91C6800E001241C4A92F844501F
:105738000020C1B2A14200F1010007D2184F02AE09
:105748002F440E44795C06F8041CF2E71968091B1B
:10575800196092F844101D68214482F84410A5B9D4
:1057680003204021FFF71CFA0E4A136823F48043F4
:1057780023F070039BB283F4405343F4004343F097
:1057880080031360054B83F84450002CC7D09DF864
:10579800040003B0F0BD00BFA40E0020B00C002030
:1057A800A80E00200C5C0040436A8269D154436A09
:1057B80002690133934228BF00234362436B23B13C
:1057C8001B68DB0706D404F0C9BD036D1A6842F0F4
:1057D80080021A60704770B50E462021154608F001
:1057E80078FA0446B8B1441C204608F0D4FAB0F55B
:1057F800617F05DB40F634039842A8BF184601E0F4
:105808004FF461701923A0F5617090FBF3F03070CC
:105818002B7801332B702046202108F05AFA0446D1
:10582800B8B1441C204608F0B6FAB0F5617F05DB34
:1058380040F634039842A8BF184601E04FF461705F
:105848001923A0F5617090FBF3F070702B78013389
:105858002B70204670BDF0B587B0054608F046FAB3
:10586800C0B208BB0446464A06231268634303F5E0
:105878008873134419259F79DE799A7A4FF46170F9
:10588800591D15FB070715FB06005B79009701906A
:10589800C8780290097903913A482146013400F00A
:1058A800F9FD0C2CDFD168E0284608F074FA0B28C3
:1058B8005FDC334B062670431E6800F5887006448B
:1058C8000023681C20218DF8173008F002FA741D97
:1058D800054658B1451C284608F05DFA032805D846
:1058E8009DF81730607101338DF817302846202154
:1058F80008F0EFF9054658B1451C284608F04BFA60
:105908000D2805D870719DF8173001338DF81730C0
:105918002846611C0DF11702FFF75DFF202108F0F2
:10592800D8F9054658B1451C284608F034FA0C2821
:1059380005D89DF81730E07001338DF817302846E8
:10594800202108F0C6F950B1013008F024FA0D28DA
:1059580005D89DF81730207101338DF817309DF860
:105968001730062B09D020460021062208F07DF9C1
:1059780003E005480C2100F08DFD07B0F0BD00BF25
:1059880098040020E01C0108001D0108F0B585B04E
:10599800074608F0ABF9C0B2E0B90446324B1B68C1
:1059A80004F11C0203EB82021920D679157A531DE3
:1059B8004FF4617110FB061610FB051152795B78E4
:1059C8002A48019100962146013400F063FD282CF5
:1059D800E4D146E0384608F0DEF927283DDC224BC2
:1059E8001B6800F11C0603EB8606781C00232021A7
:1059F8008DF80F3008F06DF9751D044658B1441C38
:105A0800204608F0C8F9152805D870719DF80F30A0
:105A180001338DF80F302046202108F05AF904464A
:105A280058B1441C204608F0B6F90D2805D89DF851
:105A38000F30687001338DF80F302046A91C0DF126
:105A48000F02FFF7C8FE9DF80F30042B09D0284637
:105A58000021042208F009F903E00548282100F094
:105A680019FD05B0F0BD00BF98040020161D0108FF
:105A7800001D01082DE9F84F9B46714BDFED717A47
:105A88001B882DED028B08EE103AB8EE488AF7EE27
:105A9800008A28EE278A0024C8EE888A804689462C
:105AA8009246064625462746022F674B0ED199F89F
:105AB8000520B3F904309FED657A0A32534307EEA7
:105AC800903AF8EEE77AC7EE877A34E05A5F604B8F
:105AD800EB5ECAF100001344834203DB5345B4BFB5
:105AE800184650465B4BEB5EC01A3BF9053018442C
:105AF800594B07EE900A1B88B8EEE77AD907F2EE01
:105B0800047A87EE277A04D5D8ED117A67EE277ADA
:105B180011E099F80410DFED4D6A1431514307EE96
:105B2800901AF8EEE77A9B07C7EEA67A44BFD8ED3D
:105B3800126AE7EE267A494BD6ED085AEB5E07EE75
:105B4800103A474BB8EEC77AD3ED036A454B27EEB8
:105B5800267A234477EEC77AD6ED0B6A27EE886A51
:105B680067EEA55AD3ED007AE6EE267ADFED3E6AB7
:105B7800F4EEE67AF1EE10FA09D4DFED3C6AF4EEC1
:105B8800667AF1EE10FAC8BFF0EE667A01E0F0EE40
:105B9800667A3748C3ED007A0319D3ED006A83EDBE
:105BA800007A00F10C0218302244204492ED006A79
:105BB80077EE666A90ED007A80ED006A66EEA86A74
:105BC80036EE077AC2ED006A37EE267AF0EE086AFA
:105BD80087EE267AD6ED0E6A27EE260ADFED256ACD
:105BE800B4EEE60AF1EE10FA09D4DFED236AB4EE5A
:105BF800660AF1EE10FAC8BFB0EE660A01E0B0EE30
:105C0800660A75EEA77A013737EEC00A08F098FAE7
:105C18001A4BB0F57A7FA8BF4FF47A709842B8BF94
:105C28001846174B032FE85204F1040405F1020546
:105C380006F104067FF438AFBDEC028BBDE8F88F9F
:105C4800AC050020BD37863512030020000048420D
:105C5800DC2000205C04002004030020A4050020B0
:105C68009C040020140C002000007AC300007A4332
:105C7800F80C0020000096C30000964318FCFFFFB4
:105C8800D40500200F4B1A78562A17D15A88B2F536
:105C9800D76F13D11A79BE2A10D193F8B426EF2AF8
:105CA8004FF000000CD113F8012B5040064A9342E4
:105CB800F9D1D0F1010038BF0020704700207047AB
:105CC800704700BF00F80308B8FE0308434A91680C
:105CD8002DE9F84F40F201130B4040F201118B42BD
:105CE80093460CD13E4B93F86C2093F86D9083F853
:105CF8006D20B9EB020918BF4FF0010901E04FF020
:105D080001094FF00008374B1B785FFA88F4A3426B
:105D180061D9354B354E1B68354F23B93B685B89D4
:105D280026F8143054E03A682E48072C94BF12F82D
:105D380004A0A24651469847DBF80830DB05054623
:105D480009D5B9F1000F06D02A4B1B681B685046CD
:105D5800DB6929469847A5F2EE2240F2DC5392B25D
:105D68009A4288BF3B68DBF8082088BF5D8942F209
:105D78000103134053B3204B1978194B01F0030268
:105D880002EB840203EB420293F8CE00A2F86E50B5
:105D98001A4620B9032919D9012183F8CE1002EB3C
:105DA800C40302EB4402B3F87010B3F86E500D440C
:105DB800B3F87210B3F874300D441D44ADB2A2F8B4
:105DC800D05004232DB295FBF3F5ADB226F814504C
:105DD80008F1010897E7BDE8F88F00BF041A002012
:105DE800B00C0020CB090020D4090020BA060020FE
:105DF800EC010020F0020020040B0020094B30B514
:105E08009D68094B1868094B05F480551C680023E8
:105E18000DB1828800E0A28805495A520233182B36
:105E2800F6D130BD041A0020E0060020A4060020A8
:105E3800E4060020F8B500241F4B1F78E0B2B842F2
:105E48000CD21E4B33F810101D4B53F820301BB1E9
:105E58000B2801D8DB6898470134EDE7194B9B689C
:105E68005B0328D50025184E2B46EAB2BA4222D247
:105E7800726854689C4216D02046FDF79EFEEFF3E8
:105E88001283502282F312881049626A4FF0280C5C
:105E98000CFB001001324262626942F00102626149
:105EA800DBB283F3118856F8043F1B6800221A609E
:105EB80001352346D9E7F8BDBC200020BE200020CC
:105EC80060090020041A00205C0900209C0F0020B3
:105ED80013B5044600210068012204F057FB23682B
:105EE8001A8892B242F001021A80637B8DF804305E
:105EF8000022012301A88DF805308DF806208DF8C1
:105F0800073004F08FFC02B010BD0C4B1B6807B5BE
:105F1800196819B10A4A9069014391619A88ADF8E4
:105F2800042002228DF807209868002201A98DF824
:105F38000620FFF7F2F803B05DF804FB5C070020C9
:105F48000010024010B50A4C23681BB1FFF7DDFFB3
:105F580000232360074B1B7813B1012B03D010BD1E
:105F68004FF4006201E04FF48052034B1A8010BDD9
:105F78005C07002060070020000000200430104B60
:105F880033F91030B3F5617F10B505DB40F6330205
:105F98009342A8BF134601E04FF461730C781920AF
:105FA80040F2833210FB04249C4207DA497810FB44
:105FB80001209842B4BF0020012010BD002010BD70
:105FC800BA06002037B5214D8DF8073095F8E8302E
:105FD8008DF8062002AA1A448DF804008DF80510E1
:105FE80012F8042C443AD2B20F2A09D81849022BC5
:105FF80031F8124008D8A4B1204604F075F910E031
:10600800022B4FF0C804F7D9124B1A68D5F8EC30B8
:10601800121B934205D20D4A002382F8E8300E4A3B
:10602800137095F8E930012B00D064B995F8E83081
:10603800022B03D8054A013382F8E830074A0023C7
:1060480085F8E930137003B030BD00BFB00C0020F4
:10605800C4080108001A00204A0500205F0A002031
:10606800134B10B593E8140008331B68D01808D0F8
:1060780010490822FDF750FD20460F490422FDF77C
:106088004BFD0E4B1A68002393720D4A01211160D3
:106098000C4913604FF4E0500B6010600A480B6025
:1060A8004FF4364101801160084A136010BD00BFEB
:1060B800ACF7FF1F96000020A6000020880F0020E4
:1060C800405C0040445C00407E0F0020F820002027
:1060D8002DE9F04F064689B00F4615469B462978AC
:1060E800002900F0B880252902D001353046B0E0FB
:1060F8006C78302C03D002354FF0000903E0AC78FF
:106108004FF001090335A4F13003092B4FF00008C3
:106118001AD8A4F13003DAB2092A07D80A2B13DCFB
:106128000A2202FB083815F8014BF2E7A4F16103D3
:10613800052B02D8A4F15703F0E7A4F14103052B7E
:1061480002D8A4F13703E9E76C2C03BF2C780122AD
:1061580001350022632C66D006D8252C77D0582C20
:106168003FD0002C77D0BAE7732C63D002D8642CC8
:1061780011D0B4E7752C02D0782C32D0AFE70BF1F0
:10618800040A05ACDBF800000A2112B100222346FC
:1061980013E0234620E00BF1040A05ACDBF800000D
:1061A80072B1002806DA2D238DF8143040420DF123
:1061B800150300E023460A210022FDF74DFB0DE000
:1061C800002806DA2D238DF8143040420DF115030E
:1061D80000E023460A210022FDF716FBD34600946F
:1061E8001AE00BF1040303930DF1140ADBF8000025
:1061F800102132B1583C624262415346FDF72CFBF4
:1062080006E0B4F158035A425A415346FDF7FCFAE6
:10621800DDF80CB0CDF800A03046394642464B4672
:10622800FDF756FB5BE730469BF800100BF10404C2
:10623800B8470AE0DBF8003000933046394642465A
:1062480000230BF10404FDF743FBA34647E7304660
:106258002146B84743E709B0BDE8F08F38B510F8D4
:106268000E2C50F8043C04465AB9012200F80E2CB2
:1062780020F80C1C197B18680222BDE83840FEF78C
:1062880085BB30F80C2C20F80A1C891A89B220F832
:10629800081C084A10F80F0C002522F8101004F802
:1062A8000E5C1868197B2A46FEF770FB04F8065C3A
:1062B80038BD00BFA00D0020294BF0B51D68002295
:1062C8002848165CAB191418597801F0040101F03C
:1062D800FF0371B10132102AF2D10020F0BD1BB1C9
:1062E80003EB83035B00DBB210F8012B303A134455
:1062F800DBB2221A022AF2DC002184420AD919B13F
:1063080001EB81014900C9B210F8012B303A114460
:10631800C9B2F2E72E2E15D1601C0022042406789B
:10632800AF1902EB82027F7852007F0792B204D540
:10633800303A16FA82F2013092B2013C14F0FF04AE
:10634800EDD100E0002208484143642000FB02121E
:1063580006240648B2FBF4F200FB0320F0BD00BFA0
:106368007C0100206B11002040420F0080969800AD
:1063780030B5002213460D495C5C9CB12E2C04D12B
:10638800013378B11C1800250D55C95C0A246243F5
:10639800A1F13004092C9CBF303A52180E2B03D8B7
:1063A8000133E8E7104630BD002030BD6B110020F6
:1063B80070B50022064625491301585CB04204D046
:1063C8000132072AF7D1002070BD0B440FCB204DB6
:1063D800102E05F1180484E80F002B4616D007D8B4
:1063E800012E0DD0022E2ED11A4B1B689B680BE094
:1063F800202E22D0402E26D1164B1B681B6903E0A5
:10640800144B1B685B681BE0EB6119E0124A1268C9
:10641800127A042A17D8DFE802F0080803080800EF
:106428000E4AEA612A62032204E04FF4E132EA618B
:106438002A62012283F8252005E0064B1B68DB68E9
:106448002B62204670BD064870BD00BFE4080108F5
:10645800A00D00207C070020EC010020A086010090
:10646800B80D00200EB403B503AB084953F8042B4C
:1064780068468DE80A000649FFF72AFE009B0022BD
:106488001A7002B05DF804EB03B07047410F0020AA
:106498008D2C00080FB407B50A4904AB08680A49EF
:1064A80053F8042B09680193FFF712FE074B18688D
:1064B800FCF73AFF0028F9D003B05DF804EB04B00C
:1064C800704700BF0C07002008070020380F002085
:1064D80007B5064B0093064B06481968064A074B52
:1064E800FFF7D8FF03B05DF804FB00BFF51B0108F8
:1064F80074010020351D0108E01B0108EC1B010890
:1065080010B50748FCF7B2FF0024064B0648E158CF
:10651800E2180C345268FFF7BDFFE42CF5D110BD2A
:10652800511D0108BC0D0108671D0108F8B5074693
:1065380007F0DCFB044638B9194B1A485A791A4B4C
:10654800013A53F8221028E038461849224607F045
:10655800D5FB60B91648174CFCF788FF54F8041FA0
:1065680019B11548FFF796FFF8E7144805E000252C
:106578000D4B53F8256026B91148BDE8F840FCF7E3
:1065880075BF38463146224607F0B8FB013500286A
:10659800EED1034B0B485D713146BDE8F84079E711
:1065A800041A00206F1D0108B009010857260108C8
:1065B800831D0108AC090108961D0108B4240108CF
:1065C8009A1D0108AF1D010870B5044607F08EFB3F
:1065D80008B91E482EE020461D4907F001FC00249A
:1065E8002646254678B12CB1012C06D107F0D3FBFD
:1065F800064602E007F0CFFB0546154900200134A6
:1066080007F0EEFBEEE70B2D04D912480C21BDE88C
:1066180070403FE7012C07DC0F4B104833F9152079
:106628002946BDE8704035E7A6F57A73B3F57A7F59
:1066380003D90B48BDE870402CE70A482946324682
:10664800FFF728FF044B23F8156070BDC11D010832
:10665800EE210108FB1D0108E4060020211E0108A7
:10666800391E01085B1E010810B54F20FCF784FD98
:106678000C4C84F82C010020FCF77EFD4FF4E1332C
:10668800C4F83031C4F83431C4F83831C4F83C3176
:10669800522384F82D0184F82E0184F82F0184F800
:1066A800403110BD041A002010B5FEF7EDF94FF483
:1066B8003024012806D11CB1FEF7E6F9013CF8E7C1
:1066C800052010BD002C08BF052010BD70B505467B
:1066D800441E14F8011F61B1064E304607F0F9FA5E
:1066E8000028F6D0861B04483044631B80F810311C
:1066F800EFE770BD1D210108041A00207FB504468C
:1067080007F0F4FA082824D100231F49E25C09683D
:106718001144497801F00301022908BF203AE254E4
:106728000133082BF1D10025665D1848314607F082
:10673800D0FA28B101356019314607F0CAFA18B104
:106748001348FCF793FE1CE0082DEDD12046FFF717
:10675800BDFF1048FCF78AFE00230F4A1A4404A91B
:1067680092F810210A440949595C02F80C1C0133BB
:10677800082BF2D1002309488DF80C3001A9FFF746
:1067880089FE04B070BD00BF7C0100201D210108F6
:10679800741E0108941E0108041A00206A1D0108CD
:1067A800F0B500231946CEB200220C2505FB02F7EE
:1067B8000D483F5CB742D4B203D00132042AF4D169
:1067C8000BE0FF2C09D0094A1A4405FB040092F893
:1067D8002C21074CA25C027201330131052901D03A
:1067E800032BE0D9F0BD00BF14000020041A0020DC
:1067F8002B1D010830B52DED028B87B0B0EE408A15
:1068080000210C22044603A807F02FFAB5EEC08A2F
:10681800DFED2C7AF1EE10FACCBF38EE278A38EE8D
:10682800678ADFED297A28EE278A6946BDEEC88A8D
:106838000A2218EE105A85EAE570A0EBE570FDF71C
:1068480033F800239D420370ACBF20232D236846F4
:106858008DF80C3007F04AFA012807D130238DF85B
:106868000D308DF80E308DF80F300CE0022805D170
:1068780030238DF80D308DF80E3004E0032804BF66
:1068880030238DF80D30694603A807F015FA03A8E0
:1068980007F02CFA0338C5B22A4603A9204607F0A8
:1068A8004FFA002363552046084907F005FA03A963
:1068B8002046294407F000FA204607B0BDEC028BB9
:1068C80030BD00BF6F12033A00007A44A91E0108C8
:1068D8002DE9F04188B0044607F008FAC5B2002D4A
:1068E80072D19048904CFCF7C1FD54ED027AF5EE58
:1068F800407AF1EE10FA2CD0013529468B48FFF783
:10690800C9FD14ED020A04A8FFF774FF0146884880
:10691800FFF7C0FD14ED010A04A8FFF76BFF01465D
:106928008348FFF7B7FD94ED000A04A8FFF762FF5C
:1069380001467F48FFF7AEFD94ED010A04A8FFF772
:1069480059FF01467B48FFF7A5FD0C2D04F1100403
:10695800CBD1DFED797A794BB0EE677AF0EE676AE2
:106968000022AA4203F110030DDA13ED045A53ED85
:10697800035A13ED026A013276EE856A77EEA57A3C
:1069880037EE067AEDE76E48CDED016ACDED027A75
:106998008DED037AFCF76AFD002408AB234413ED60
:1069A800077ADFED687A684B6848B0EEC77AB4EECC
:1069B800E77AF1EE10FAD8BF18460434FCF756FD12
:1069C8000C2CEAD1624895E020466249052207F07E
:1069D80095F938B9604B034410300022C0281A6179
:1069E800F8D19CE020465D49042207F087F9064665
:1069F8002046002E40D1202107F06BF9002800F036
:106A08008E80451C284607F071F934468046544B61
:106A180053F824600EB953486CE0284631465FFAB3
:106A280088F207F06BF9671C20BB4B4BC21810307B
:106A38000021C02811619C46F7D14B4B03EBC702DC
:106A48009846D2F804E00024BEF1000F04D147486C
:106A58003146FFF71FFD5AE018F837309C42F6DA46
:106A680023010CEB030573440FCB103585E80F00A9
:106A78000134F1E73C46CAE707F08DF9461E0B2EB4
:106A8800074648DC2046202107F023F9054650B187
:106A9800451C2846FCF730FE2F4B03EB071787ED04
:106AA800000A012400E004462846202107F011F9D5
:106AB800054648B1451C2846FCF71EFE264B03EB4D
:106AC800061383ED050A01342846202107F001F951
:106AD800054648B1451C2846FCF70EFE1E4B03EB45
:106AE800061383ED060A01342846202107F0F1F841
:106AF80018B91F48FCF7BAFC11E00130FCF7FCFD9F
:106B0800154B032C03EB061686ED070AF1D119483D
:106B1800FFF7DEFE03E018480C21FFF7BBFC08B0C6
:106B2800BDE8F081B31E01081C1A0020DE1E010812
:106B3800E41E01086A1D010800000000181A002060
:106B4800E81E01080AD7233CAF1E0108AB1E010846
:106B5800B4240108F71E0108041A0020FD1E0108CC
:106B6800B00901089A1D010874010108021F0108F3
:106B7800121F01081F2201084C1F0108026D036B38
:106B880070B50446D5699BB9A90611D5C36A1BB16E
:106B9800908C80B298470BE0E169928C40694E1C5A
:106BA800D2B2E6614254E169E268914228BFE361EA
:106BB800616BA9B92A0613D5636AA26A9A42236D42
:106BC8000AD0501CA669A062B25CD2B21A852369A9
:106BD800984205D3A16203E01A6822F080021A6085
:106BE8002B0702D5236D08221A6270BD2DE9F041EA
:106BF800FFF748F810B90A2003F05CF9AE4CAF492A
:106C0800AF4E4FF4D762204607F026F894F8943632
:106C1800022B84BF002384F8943694F894364FF4FA
:106C2800E07202FB034303F5AA7393F85020336024
:106C3800022A84BF002283F85020A24A93F85030D9
:106C480013700A2202FB03439F4A03F29663136000
:106C5800A36842F201021A403AB944F208021A4003
:106C68001AB9954A43F400539360A368DB0703D528
:106C78004FF40050FCF75FFEA3685F0409D50820B5
:106C8800FCF759FE4FF40050FCF755FE0120FCF7C5
:106C980052FEA3681D0706D54FF40050FCF74BFEC3
:106CA8000120FCF748FEA368980402D54020FCF7B1
:106CB80042FE864B864D1D60FFF772FD854B05F140
:106CC8001C0201201A60FFF773FB0146012001F046
:106CD80005FB002849D00220FFF76AFB0146022085
:106CE80001F0FCFA002840D02020FFF761FB0146A4
:106CF800202001F0F3FAA368190601D5002834D042
:106D08001020FFF755FB0146102001F0E7FAA368B1
:106D18001A0700D548B30420FFF74AFB01460420B0
:106D280001F0DCFA30B90820FFF742FB01460820E1
:106D380001F0D4FAA3685B0503D400231A46194668
:106D480009E00028F9D110E079B90121C00708D479
:106D58000C33302B0BD060481844007A8707F5D5E0
:106D6800F2E70132D2B2022AF2D9FFF77DFCFCF732
:106D780089FA5A4B32685A4F1F605A4B101D1860D7
:106D880002F17501002311F803E0BEF1000F0BD1E9
:106D980001EB030C9CF802809CF803C0E04503D289
:106DA800514B83F800E002E00433A02BEBD14F4BAA
:106DB8004F49196011784F4B012903D0022903D09C
:106DC8004D4902E04D4900E04D4919604D4B02F52F
:106DD800D9721A60FCF72CFE33684B4A9FED4B7A48
:106DE80003F5D37111604A490020888049484A490F
:106DF80001604A4803F5B37606604948A1F12206C6
:106E0800066048480760484803F5D7760660474853
:106E18002E31016046490D60464903F5D870086077
:106E2800B4F8F01007EE901AB4F8F210F8EE677A9A
:106E38000432C2ED017A07EE901A93F858101170D7
:106E480093F874105170F8EE677A94F8251111735D
:106E58003949C2ED027A0A60384A191D1160384A68
:106E680003F160011160374A03F164011160364A89
:106E780003F25D111160354A1760B3F8622107EE1D
:106E8800902AF8EEE77A324AC7EE277A9FED317AF0
:106E980067EE877A93ED177AC2ED007ADFED2E7AE6
:106EA8002E4B67EE277AB6EE007AC7EE277AC3ED47
:106EB800007ABDE8F08100BF041A002000F803083A
:106EC80098040020640B0020D0050020EC0100206D
:106ED800141B00207C070020140000205C0B0020FD
:106EE800D41A0020600B002060000020B4040020A9
:106EF800F81A00204801002041530008995500085D
:106F08007D5A0008C4050020C80D00200000614417
:106F1800B409002020050020FC1A0020A00600204B
:106F2800E0060020A4060020DC050020A8060020BA
:106F3800AC060020B406002054050020640400209C
:106F4800A005002058030020B4050020BC0500203F
:106F5800C00500204C3D0F44DB0F49409C05002034
:106F680008B502F0C5FFFFF741FE0F2014210122EA
:106F7800BDE8084002F05EBF10B50446204606F0A2
:106F8800B5FE10F0FF0F07D10B4B0C4893F8941681
:106F9800BDE81040FFF77EBA204606F0FCFE022846
:106FA80008D8054B064C83F8940602F0A1FFFFF7BA
:106FB8001DFEE3E710BD00BF041A002048210108A8
:106FC8001F2201082DE9F0412DED048B824984B080
:106FD800054606F053FE8149002828460CBF0124C7
:106FE800072406F04BFE7E490028284608BF0224E5
:106FF80006F044FE002808BF0424E10740F1B780EA
:107008007848794FFFF746FA0020FFF761FA77488A
:10701800FFF740FA7648FFF73DFA7A79754B7648DC
:10702800013A53F82210FFF735FAD7ED047AF5EE56
:10703800407AF1EE10FA60D007F11805002615ED38
:10704800028AB5EE408AF1EE10FA52D001366B484A
:1070580055ED019A95ED009AD5ED018A3146FFF775
:1070680019FAB5EEC08AF1EE10FA02D56448FFF7B6
:1070780011FAB0EE480A6846FFF7BCFB01466148C2
:10708800FFF708FAF5EEC09AF1EE10FA02D55C485F
:10709800FFF700FAB0EE690A6846FFF7ABFB014656
:1070A8005848FFF7F7F9B5EEC09AF1EE10FA02D595
:1070B8005348FFF7EFF9B0EE490A6846FFF79AFB25
:1070C80001465048FFF7E6F9F5EEC08AF1EE10FAEE
:1070D80002D54B48FFF7DEF9B0EE680A6846FFF7BD
:1070E80089FB01464848FFF7D5F90C2E05F1100534
:1070F800A5D14648711CFFF7CDF94548454DFFF726
:10710800C9F9D7F8088055F8041F19B14248FFF7A4
:10711800C1F9F8E70D46414B53F8256056B10123F4
:10712800AB4013EA080F03D03D483146FFF7B2F9E8
:107138000135F0E73B48FFF7ADF931467B1804AA63
:1071480093F810311344384A8A5C03F8102C013143
:107158000829F3D1002335488DF808306946FFF730
:1071680099F93348FFF796F9402003F0EFF9A207A1
:107178001AD53048FFF78EF92F48FFF78BF92F48BB
:10718800FFF7FAFE2E48FFF785F92C48FEF7FEFBBD
:107198002C48FFF77FF92948FEF75DFB2448FFF7E5
:1071A80079F9802003F0D2F963070FD52648FFF755
:1071B80071F92648FFF76EF9204800F0F3FC1C48E7
:1071C800FFF768F94FF4807003F0C0F904B0BDEC24
:1071D800048BBDE8F08100BF741F01082F2D010842
:1071E8007B1F0108811F0108041A00208F1F010856
:1071F800A11F0108B0090108AD1F0108B81F010847
:10720800EE210108E22301086A1D0108C01F0108D8
:10721800D21F01089C0E0108E21F0108A00E0108F8
:10722800F01F0108FD1F01081D21010809200108A0
:10723800B424010812200108252001081F22010892
:10724800332001083D2001084C2001085D20010879
:107258002DE9F04FA44BDA682DED028B1A61A34A91
:107268001268DA60A24B1A6842F020021A60A14B39
:107278001A78012A0CBF002201221A709E4B1A7834
:1072880091078BB040F169839C490978042940F241
:1072980064839B49097801F0040101F0FF0011B9EA
:1072A80022F001021A701B78934E964C964D13F0FB
:1072B800010F10D178B19B070DD5944B20686268F7
:1072C80018605A60FCF794FB914B1B88AB823378AB
:1072D80043F001033370AB7D8E48039001334FF0C8
:1072E800050893FBF8F808EB8808C8EB03088A4BF5
:1072F80085F816801B780493831D03EB8808002308
:107308008048864A1E58864F9E5096FBF7F502F134
:1073180008071918DD51834F059107FB056742F2ED
:10732800107697FBF6F603991FFA86F902F1100A10
:1073380021F8029F03EB830B53F80A60039158F876
:107348000B1048F80B70C1EB060C0CEB0706049900
:10735800734F43F80A604FF0050C96FBFCF61832A1
:1073680007FB056501299D50074606D1A9F10202D0
:10737800B2F5797F9CBF059A15600433082BBFD1FD
:10738800614D5A4B6A6E19689FED677A1B686B6688
:107398008A1A07EE902AF8EE677A574BDFF8988139
:1073A8001B78624EC7EE877AB7EE008AF4EEC87A89
:1073B800F1EE10FA58BFF0EE487A13F00103C5ED6C
:1073C8001A7A13D007AA0092504B08AA01920CCB44
:1073D80097E80300FCF7C8FA079A6423B2FBF3F2B4
:1073E800A8F80020089A92FBF3F301E0A8F800300F
:1073F80095F86C203380444B002A39D0D3ED1A7AA3
:1074080021681A6FC8EE277A8A1A596F022007EE88
:10741800102AB8EEC77A626827EE277A511ABDEEAD
:10742800C77A434A17EE106A07EE101AD2ED006ABF
:10743800B3F97A20B8EEC77A27EE267A67EE277A6C
:10744800FDEEE77A17EE901A02FA81F1B3F9782087
:1074580002FA86F291FBF0F192FBF0F289B292B255
:10746800A3F87E10A3F87C20A3F87A10A3F878205C
:10747800012385F86C302F4B79681B883868224CBB
:10748800204E696703F030032867002B00F06582FF
:1074980004F18803009304F18C030193D4F880204D
:1074A800D4F88430FCF760FAD4F884207368D31ACF
:1074B80007EE903A1E4B326893ED007AD4F880308C
:1074C800F8EEE77A9B1A144AC4F8903067EE877A88
:1074D8001378FDEEE77A012BC4ED257A91462DD07D
:1074E800022B00F0DB8038E26C040020001A002038
:1074F800FC0200207A0A0020910400209004002059
:10750800F0200020880B0020C80D0020740B0020FC
:1075180090050020DE0D00207C0B00200C0E0020C2
:1075280080969800806967FF00007A44780A0020F6
:10753800D000002004030020760A002094ED2D7A64
:10754800C34B94ED266A1F68D4ED2A5AD4ED1A7AF3
:10755800D4ED2B4A94ED2C5ABE4BF1EE476AFDEE62
:10756800E66ABDEEC77A16EE906A17EE109A002208
:10757800B94951F8120007EE100AF8EEC76AA1F1EE
:10758800140466EE866A145BFDEEE66A283116EE90
:10759800905A2D1BADB255522DB207EE105AF8EE87
:1075A800C76A054466EEA56A07EE105AFDEEE66A5C
:1075B80016EE908AF8EEC76A93ED007A66EEA46A32
:1075C8001FFA88F8A6EEA77ABDEEC77A17EE105A0A
:1075D800B54203DB4D45A8BF4D4600E0354606EEF3
:1075E800905A5D68DFEDA53A451BB8EEE67A06EEDF
:1075F800905AF8EEE66A83ED007AC6EEA76A31344F
:10760800A4B2622CBDEEC77AC3ED046AB97858609B
:1076180004EE101AB8EE444A17EE10CA24EE234AB4
:1076280093ED027A88EE044AC4441FFA8CFC76EE85
:10763800C76A34EE274A87EE844AA4EE267A83ED99
:10764800047A83ED027A0FD965EE076A8348FDEE66
:10765800E66A16EE901AB1F5FA6FA8BF4FF4FA6110
:107668008142B8BF014600E00021614440F6B830CD
:1076780009B28142A8BF014679488142B8BF014694
:107688007848115278490A2000FB0211023253F857
:10769800140B0860042A7FF46BAF5EE16C4BD4F8DE
:1076A80088701E68B6F808807B08984528BF9846F9
:1076B800B4F8BC301AB2904502DC1FFA88F80EE024
:1076C80094ED1A7ADFED697A67EE277AFDEEE77AAC
:1076D80017EE908A98441FFA88F8A4F8BC80D5F869
:1076E800C030D5F88C40C3EB040A5046FCF702FAC8
:1076F800002841F2931201DD904201E04342934297
:10770800CCBF00230123DFED5A8A7BB305EE10AA14
:10771800B8EEC50A20EE280A06F05CFD06EE907A5F
:10772800F8EE667A40F6B83220EE270ABDEEC00AB7
:1077380010EE103A9BB2A5F8C4301BB29342A8BF12
:107748001346474A9342ACBFE318A31848F6A04231
:10775800934203DDA3F50C43A03B04E0002BBCBF20
:1077680003F50C43A033C5F8C83001E0C5F8C8409C
:10777800D5F8C840C4F50C53283307EE103AF8EE94
:10778800C77A67EEA88AB0EE680A06F09DFC8DED10
:10779800090AB0EE680A06F01DFD95ED367A95EDFA
:1077A800334AD5ED1A7AD5ED343AD5ED355A2E4B04
:1077B8008DED080AF1EE476AFDEEE66ABDEEC77A7E
:1077C80016EE90AA17EE10BA0022DFF8ACC032F914
:1077D8000C0005EE108A07EE100A0AA800EB420119
:1077E80011ED026A2348F8EEC56AB8EEC77A0CF1C3
:1077F8003C0C96EE267ABDEEC77A17EE101A09B23F
:10780800B1F57A7FA8BF4FF47A718142B8BF0146BB
:1078180088B222F80C0000B206EE900AB8EEE67ABA
:1078280067EE046AFDEEE66A16EE90CA67EE236A12
:1078380093ED007AA6EEA77A1FFA8CFCBDEEC77A04
:1078480017EE100A50451BDB5845A8BF584618E0EC
:10785800C4050020B80B0020580E002030F8FFFFA8
:1078680048F4FFFFCC050020E00B00200000C842D0
:10787800D302373918FCFFFF440E0020DB0FC94044
:10788800504605EE100A58685FED044AD3ED026AC7
:10789800081A06EE100AB8EEC66AB8EEC57A86EE81
:1078A800276A143303ED057A03ED016AB07843F8CB
:1078B800101C05EE100AB8EE455A36EE666A25EE3B
:1078C800245A40F6B83088EE055A35EE275A87EE26
:1078D800855AE5EE066ABDEEC75A43ED016A43EDE7
:1078E800036A65EEA66AFDEEE66A16EE901A8C4407
:1078F80015EE101A614409B28142A8BF0146194821
:107908008142B8BF01461848115218490A2000FBA5
:1079180002110232042A81ED007A7FF456AF3379DE
:1079280023B1642394FBF3F4114B1C8033889F42EA
:107938000DD9D5F8C030D5F88C00C01AFCF7DAF8A4
:1079480042F210730028B8BF4042984205DD012377
:1079580089F80030064BAA8A1A800BB0BDEC028B5E
:10796800BDE8F08F48F4FFFFCC050020B80B0020DD
:10797800BC0A00200D4B1A680D4B92B213445B00F1
:1079880010B51A680B4BC2F309021A6019680A4A43
:1079980089B20131491000238B4206D0074852F8BA
:1079A800044B20F813400133F6E710BD505C00404B
:1079B8001E300020A40E002020620040A80E0020E7
:1079C800054B06491A68538A18B98988CB1A138255
:1079D8007047086818447047880F0020D4000020BA
:1079E800054B06491A68538A18B98989CB1A138234
:1079F8007047886818447047880F0020D40000201A
:107A08002DE9F8435D4B5E4E1B685E4D00274FF035
:107A1800C0099F7283F80990DF7237602B6823F4DE
:107A2800EC4323F0700343F400739BB22B602B6884
:107A380023F4E04323F040039BB248F2800483F030
:107A4800100323432B6032684F4B13FA82F35B0019
:107A58004FF04008C3F8008033689BB203F100532D
:107A680003F540535B0080221A602B6823F4F873F7
:107A78001B051B0D23432B60444B384693F82C10F1
:107A8800FDF78EF82B6823F4804323F070039BB234
:107A980083F4405323432B603D4B1A6822F4EC4295
:107AA80022F0700292B21A6031683A4A12FA81F2F0
:107AB80052000320C2F800901A6822F4E04222F033
:107AC800400292B282F0200222431A601A6822F41D
:107AD800804222F07002224392B21A605A6822F45D
:107AE800EC4222F0700242F4C06292B25A603168ED
:107AF800294A12FA81F252004FF4807111605A68D3
:107B080022F4804222F07002224392B25A605A68EC
:107B180022F4E04222F0400292B282F02002224394
:107B28005A60EB6823F4EC4323F070039BB2EB60DC
:107B380032681A4B13FA82F35B004FF488721A60AA
:107B48004146FDF72DF8EB6823F4804323F07003DA
:107B58009BB283F440532343EB60EB6823F4E04388
:107B680023F0400323439BB2EB603846FDF7E8F867
:107B78000B4B01221A60BDE8F88300BF880F002074
:107B8800505C0040005C004004300020E40000200D
:107B9800045C004008300020103000201C30002019
:107BA800F820002010B50446204606F09FF810F093
:107BB800FF0F06D10C4B0D481978BDE81040FEF7B1
:107BC80069BC204606F0E7F802280CD8064B084C9A
:107BD8001870084B0A2202FB0030074B0630186069
:107BE800FBF750FBE0E710BD640B002044210108BF
:107BF8001F22010894200020D005002038B5044633
:107C080054B1FBF74DFB0546FBF74AFB401BB0F5AB
:107C18007A7FF9D3013CF3E738BD314A2DE9F047C3
:107C28001468238A257A9046ABB9042D13D12D48C0
:107C38002D490278012A0AD12C4A14682C4AA4B288
:107C480022445200136030220A80037043E010235C
:107C58000B8007253FE0A78ABB428CBF022504257D
:107C68009F4228BF1F46BEB2A369304698471F49A6
:107C78000B689BB203F1005303F540535B0007F117
:107C8800010C1B8803F1005303F540534FEA6C0CB9
:107C98005B000022624500F1020009D010F801AC37
:107CA80010F8029C49EA0A2923F822900132F1E7E8
:107CB8000A680F4B92B213445B0030221F60238A7C
:107CC8009B1B2382638A1E44074B66821A80094BDA
:107CD8004FF440521A80D8F800301D72BDE8F08782
:107CE800880F0020F6200020840F0020505C004000
:107CF80002300020820F00202DE9F04FD04AD14CED
:107D080010685168DFF85493DFF854B387B004ABB8
:107D180003C34FF4D7620021204605F0A6FF04F5FF
:107D2800AA73C9F80030C84B00261E7004F2966387
:107D3800CBF800305623237003236371A3604FF4FC
:107D48001673A4F8F03040F27E45FA23A4F8F23016
:107D5800A4F8D0502A2340F23A75A4F8EE30A4F8DB
:107D6800D2504FF4FA734FF47A75A4F8F630A4F8A9
:107D7800D450202340F27E5584F8F43040F24C4031
:107D88006E23A4F8D65040F2EA5584F80431A4F8DA
:107D98001C012B2340F26C70A4F8D85040F2B45563
:107DA8000127212240F2DC514FF01E0A84F80531E8
:107DB800A4F81E014FF4C8731920A4F8DA5032252C
:107DC80084F80621A4F80831A4F81A1184F82501CA
:107DD800A4F8DE3084F8EC7084F821A184F82471CA
:107DE80084F82771A4F8DC50A4F8E05084F82A71CC
:107DF800019002910392FEF737FC40F6AC53A38141
:107E0800D9F80030A6734FF00F0C83F808C04FF074
:107E1800170E4FF0220C83F818E083F819E083F866
:107E280009C04FF0550E4FF00E0C4FF0280883F89C
:107E380006E083F813C04FF02D0E4FF0350C83F891
:107E48000EA083F80FA083F810E0DD7183F81DC041
:107E58001E7083F8048083F805809E765E74DE7653
:107E68009E741E7701989872039A1A7553229A770E
:107E780064225A20DA7783F817E04FF00A0ADFF80D
:107E8800E4E1D87278225A7383F815A083F80C803D
:107E980083F82170C3F83CE0C3F840E04FF0824E0D
:107EA800C3F82CE04FF07C5EC3F838E0DFF8B8C1C7
:107EB800DFF8B8E1C3F824C0C3F828C0C3F844E029
:107EC800624ADFF8ACE1DFF8ACC102991A635A6381
:107ED800C3F848E0C3F84CC084F89606412084F8FB
:107EE800970684F89856A4F89E1684F89A6684F83B
:107EF8009B6684F8996684F89C6604219A66544ABD
:107F080083F85810DA661521524A83F87470A3F87A
:107F18005460A3F85660A3F85260C3F85CE083F895
:107F2800608083F8618083F864101A674A48FEF716
:107F3800CDFBD9F800504FF44873A5F86231C82337
:107F480085F8A7314FF49663A5F8A83140F2D933E4
:107F5800A5F8AA3140F6430385F86071A5F8AC315D
:107F680085F85D6185F85E6185F85F8185F86461F3
:107F780085F8A6A12B465F464FF47F72A3F86621C9
:107F880004A94FF4FA62A3F8682140F2DC52A3F87E
:107F98006A218A5D83F86C210136FF22082E83F856
:107FA8006D2103F10803E7D10123C82285F8AE311A
:107FB80085F8AF3185F8B03185F8B6316423A5F876
:107FC800B221A5F8B83114224FF4967385F8B4217C
:107FD800A5F8BA311E222823A5F8BC3185F8B521A9
:107FE8000023E21810330021C02B164E1161F8D17E
:107FF800294606F545704FF4E07205F02DFE294636
:1080080006F2D4404FF4E07205F026FE3B6859684A
:10801800186806F5D46203C2198922F8021B196888
:10802800C6F8AA16596851601B891381012386F87E
:108038006433022386F8243507B0BDE8F08F00BF0B
:108048000C0A0108041A0020640B00209A99193FB1
:10805800F6287C3F3D0A773F552101089804002007
:10806800D00500208FC2753D00002040CDCC4C3D8E
:108078000000A04000004040F8B5394E394C054694
:108088004FF4204730682760D0F818C01CF4004F20
:1080980011D1D0F804C0344F0CEA070747F49037E1
:1080A8002F4347604FF420472760D0F818C01CF0D2
:1080B800020F3FD00EE007F1FF3C0FB16746E3E740
:1080C800C4F800C000E02760FBF7B2FD003018BF1D
:1080D8000120F8BD012A01D941F0800181624FF4E5
:1080E8002041216087697F062AD5476821601E499B
:1080F800394041F0007141F41051294341EA0241ED
:1081080041600025E9B28A424FF42041216030687D
:1081180007D087697F0718D52160416A595501350D
:10812800F0E70B468269920614D523602023C361C9
:108138000120F8BD07F1FF3C002FC1D06746B4E726
:108148004F1E0029BFD03946CCE74F1E0029BAD0B0
:108158003946DEE75A1E0BB92260B5E71346E1E758
:108168002407002064110020009800FC07B50021B6
:1081780001AB03227720FFF77FFF9DF805009DF8EC
:108188000430000240EA03409DF80630184303B06B
:108198005DF804FB08B5FFF7E9FF014B586408BD1B
:1081A800A40E002008B5FFF7E1FF014B986408BD55
:1081B800A40E002013B5062204463B21D0206B46AE
:1081C800FFF75AFFA0B19DF800209DF8013043EA5F
:1081D800022323809DF802209DF8033043EA0223FE
:1081E80063809DF804209DF8053043EA0223A380AC
:1081F80002B010BD07B5752101220DF10703D0208B
:10820800FFF73AFF03B05DF804FB13B506220446F6
:108218004321D0206B46FFF72FFFA0B19DF8002027
:108228009DF8013043EA022323809DF802209DF83F
:10823800033043EA022363809DF804209DF805304B
:1082480043EA0223A38002B010BD73B5194C03683A
:1082580023600B686360184D0068184EFBF7C8FB75
:10826800174B009395E8030094E80C000196FBF780
:108278007BFB60686968134A33681360411A07EE2C
:10828800901A1149206891ED007A29680F4AF8EE92
:10829800E77A411A67EE877A1160FDEEE77AC2ED58
:1082A800017A0B4A13600B4B1B68DA880A4B1A8059
:1082B80002B070BD480E0020880B0020540E00202C
:1082C800500E0020900E0020D0000020580E0020F4
:1082D800880E0020C4050020840E00202DE9F043FC
:1082E800142285B0814688461B48002105F0BDFC54
:1082F80003261A4B0027B74224DA13F8042C00216E
:10830800C8B2013112B1501E0240F9E71C7AD1B24D
:10831800013214B1611E0C40F9E7421A002A0EDD41
:10832800A3F10C0595E8070001AC84E8070093E881
:10833800070085E8070094E8070083E8070001378D
:108348000C33D8E7013ED4D1034A4846414605B02C
:10835800BDE8F043FAF7D7BEF00E00202000002059
:1083680010B50848FBF782F8074B1C682046FAF757
:10837800DBFF18B90A20FFF741FCF7E7034B044A73
:10838800DA6010BD5E2101083008002000ED00E031
:108398000400FA0508B50548FBF768F8FFF7ACFCD8
:1083A80001F0A6FDBDE80840FFF7DABF6A21010821
:1083B80008B50748FBF75AF8064A002313701363F9
:1083C800054A1370FDF71AFDBDE80840FFF7C8BF5E
:1083D80080210108040F0020F420002008B504487B
:1083E800FBF744F801F084FDBDE80840FFF7B8BF8B
:1083F800AC21010877204821012201F007BA772033
:108408005821012201F002BA10B5184C23681BB19B
:10841800FDF77BFD002323606B218022D02001F033
:10842800F5F96420FFF7EAFB19210022D02001F0BA
:10843800EDF96B210322D02001F0E8F9372102225F
:10844800D02001F0E3F90A4B1A211A78D02001F064
:10845800DDF91B211822D02001F0D8F9D0201C21E9
:108468001022BDE8104001F0D1B900BF5C07002020
:108478001100002070B50A4E00EB8000064400246D
:108488003319013413F8A00C064B1D78684001F02D
:1084980023FA052CF4D12846BDE8704001F01CBA37
:1084A800570A0108F5200020642928BF6421F8B57F
:1084B80010FB01F7642497FBF4F40546E4B20026A8
:1084C800F3B2A34204D29F20FFF7D4FF0136F7E7A7
:1084D800AC420BD2142097FBF0F0C4EB841366383F
:1084E800C4EB83031844C0B2FFF7C4FF0134E4B2FD
:1084F800AC4238BF9A20F7D3F8BD0F4B10B50446ED
:10850800185CFFF7B7FF0D4B33F91430B3F57A7FDA
:1085180005DBB3F5FA6FA8BF4FF4FA6301E04FF437
:108528007A73A3F57A730A2293FBF2F10920C9B290
:10853800BDE81040FFF7B8BF1D210108BA060020AA
:1085480010B5441E14F8010F10B1FFF793FFF9E7B7
:1085580010BD2DE9F047704ADFF8D081137886B056
:108568009146BBB90122D8F8001089F800206B4A5F
:108578001A445068884203D00C33302BF7D10022BC
:1085880002235372664B67485963FAF76FFF6648D0
:10859800FAF76CFFD8F80000FAF7D5FE002800F0CB
:1085A800B780624B5E4C1868FAF7C8FE0928014686
:1085B80001D03F284CD14FF0000A256B5C4F56463E
:1085C8002DB1574839682A4605F098FB10B9BA46C4
:1085D80006B93E46574B0C379F42F1D3B6B13768C0
:1085E800DAF800E02B46F85C1EF80310814201D04F
:1085F80023630BE05A1C31B92D2B04D82020E054FA
:108608002263A15402E0E0541346ECE7236B0BB15C
:10861800564512D04848FAF729FF564509D856F862
:108628000C0BFAF723FFD8F800000921FAF790FE9F
:10863800F3E73D48FAF71AFF0025236B9D42A9D2BC
:10864800374BD8F80000595DFAF782FE0135F4E798
:10865800236B2BB9042839D12046FFF7A9FE57E030
:108668000C2801D1354890E70A2901D00D2947D1B6
:1086780033482B4EFAF7FAFE226B0023A3542278D4
:10868800232A16D004932F4B009303A82849039656
:1086980013220C2305F083FB054638B1006805F06A
:1086A80025FB0130AB683044984702E02648FAF7CA
:1086B800DDFE1B480021302205F0D7FA0023236392
:1086C80099F80030002B7FF462AF21E00C28C9D064
:1086D8007F2903D15EE72F2B3FF65CAFA1F1200283
:1086E800D2B25E2A3FF656AF13B920293FF452AFF3
:1086F8005A1CD8F800002263E154FAF729FE49E72A
:108708007F29E8D1013B00222363E2540F483FE769
:1087180006B0BDE8F08700BFF42000201400002058
:10872800040F0020B3210108EB21010830080020C4
:10873800BC0D0108A00E0108F0210108F52101086F
:10874800B4240108B9300008002201081C220108DD
:1087580010B5AE2001F0C4F8D42001F0C1F8802093
:1087680001F0BEF8A82001F0BBF83F2001F0B8F8EE
:10877800D32001F0B5F8002001F0B2F8402001F054
:10878800AFF88D2001F0ACF8142001F0A9F8A12071
:1087980001F0A6F8C82001F0A3F8DA2001F0A0F84B
:1087A800122001F09DF8812001F09AF8CF2001F005
:1087B80097F8D92001F094F8F12001F091F8DB2026
:1087C80001F08EF8402001F08BF8A42001F088F821
:1087D800A62001F085F8AF2001F082F8A62001F06C
:1087E8007FF8AE2001F07CF8202001F079F8002015
:1087F80001F076F8B02001F073F8402001F070F82D
:10880800002001F06DF8102001F06AF84FF4806440
:10881800013C0020A4B201F05FF8002CF8D18120BF
:1088280001F05EF8C82001F05BF8AF20BDE8104009
:1088380001F056B82DE9F341B54DFAF731FDAB6BB0
:10884800C31A002B0746C0F2898200F5C333A03350
:10885800AB63B04B95F83C201E78C6F38006B21A7D
:1088680018BF012285F83C604EB1002A00F07682DC
:10887800A94B5A789A7001225A701A702DE0A64BAB
:108888002AB1DA7842F00202DA709A785A70D97806
:1088980001F0020000F0FF0238B99F488068381ADA
:1088A800002803DB01F0010200E0012202F00100D0
:1088B8001870994A88B1C8070FD511790131C9B222
:1088C8000523B1FBF3F303EB8303CB1A9349DBB224
:1088D80013710B4493F8A33253708F4C23784BB326
:1088E800FFF736FFB02000F0FBFF402000F0F8FF54
:1088F800002000F0F5FF102000F0F2FF4FF4806830
:1089080008F1FF3800201FFA88F800F0E5FFB8F1F9
:10891800000FF5D1404600F0E7FF814B627853F82D
:108928002200FFF70DFEE37823F00203E3707D4B8E
:108938003B44A3606378062B00F2FB81DFE813F069
:108948000900F9011C00950007001E0174010024AC
:10895800D8E07549754A7648FDF784FD012000F096
:10896800C3FF7348FFF7ECFD724B714872491A68F0
:10897800FDF778FD022051E1704B9A6812F0020F62
:1089880098462ED06E4C6F4F217869480A23B1FB68
:10899800F3F203FB121339780091DBB26A49FDF751
:1089A80061FDFAF7D1FF012000F09EFF6048FFF754
:1089B800C7FD664B3A78186824788378642103FBEE
:1089C80012444C434178CB1A5A43B4FBF2F4E4B254
:1089D800022000F089FF21461520FFF765FD0324DA
:1089E80000E00124D8F80830190540F1A281584B5D
:1089F800584FD3F800E03968009164239EFBF3F2E6
:108A080003FB12E354494A48FDF72CFDFAF79CFF93
:108A1800204600F069FF4648FFF792FD4B4B3A6845
:108A28001B689FED4E7A5B8982F310029A1A07EE53
:108A3800902A06EE903AF8EEE77A601C67EE877A9D
:108A4800B8EEE67AC7EE877AFDEEE77A17EE901A67
:108A58006429A8BF642121EAE171CFB200F044FF84
:108A680015203946FFF720FD63E1012000F03CFFA7
:108A78003B48FFF765FD3B4B1A6812F0020F1F4693
:108A880015D039492A48B1F90020B1F90230B1F9B5
:108A9800041000913549FDF7E5FCFAF755FF02206F
:108AA80000F022FF2248FFF74BFD032400E00224D8
:108AB8003B68DA0740F13D812D491D48B1F9002096
:108AC800B1F90230B1F9041000912A49FDF7CAFC46
:108AD800FAF73AFF2046A1E00E2C00F02A81600840
:108AE800013000F001FF2046FFF707FD3B78A34265
:108AF80006D92020FFF7BEFC601CC0B2FFF7FDFCC2
:108B08000234E4B21C4F3B78A342E5D811E100BF20
:108B1800040F0020F020002050070020570A010809
:108B280058010020404B4C0020220108F51B010889
:108B3800410F00207401002028220108041A002097
:108B4800040A00205001002033220108000A0020F6
:108B5800480A0020580A00204B2201080000C84299
:108B680060220108FC02002064050020762201082A
:108B7800AC04002086220108CB090020794C7A49F0
:108B880094F894267948FDF76DFC012000F0ACFEBE
:108B98007648FFF7D5FC764B76491F7873483A46F6
:108BA800FDF760FC022000F09FFE7048FFF7C8FC4C
:108BB8000A2303FB0747704997F897266B48FDF788
:108BC80051FCFAF7C1FE032000F08EFE6748FFF75C
:108BD800B7FC6A4997F896266448FDF743FCFAF70C
:108BE800B3FE042000F080FE6048FFF7A9FC64494A
:108BF80097F89A265D48FDF735FCFAF7A5FE05209B
:108C080000F072FE5948FFF79BFC58485D4997F8F9
:108C18009B26FDF727FCFAF797FE062000F064FE76
:108C28005248FFF78DFC84E04E4B9B681B067CD5B1
:108C3800B12000F055FE0C2000F052FE102000F08C
:108C48004FFE0024504B1B5D3622C3EBC30393FB3E
:108C5800F2F0C0B2062828BF06206038C0B201343E
:108C6800FFF708FC102CEDD1484B49491B783F48C9
:108C780013F0020F474B1A780CBF4E235923FDF708
:108C8800F1FBFAF761FE022000F02EFE3748FFF7ED
:108C980057FC4149414B4C680A683448404992FBAB
:108CA800F3F294FBF3F3FDF7DDFBFAF74DFE032037
:108CB80000F01AFE2D483B4CFFF742FC3A4B3B496B
:108CC8001A883B4B29481B88FDF7CCFBFAF73CFE7A
:108CD800042000F009FE2548FFF732FCE768236905
:108CE80034496A6D2148FB1AFDF7BCFBFAF72CFEE4
:108CF800052000F0F9FD1D48FFF722FCA3682E4966
:108D080062681A48FDF7AEFBFAF71EFE062000F06F
:108D1800EBFD1648FFF714FC28491448152205F006
:108D28000FF8FAF711FE072078E7E37843F002031B
:108D3800E3709EB9B02000F0D3FD082000F0D0FD0C
:108D4800172000F0CDFD95F858401D4B185D0134F3
:108D580004F00304FFF78EFB85F8584002B0BDE825
:108D6800F08100BF041A002096220108410F00205C
:108D7800640B0020A2220108B3220108BF220108C7
:108D8800CB220108D8220108AC0A00209104002057
:108D9800E522010890040020880B002080969800A6
:108DA800FC2201086C040020720A00200C23010830
:108DB800740A00202023010831230108E809002053
:108DC80042230108154AD2F8883043F47003C2F8E8
:108DD8008830134B196841F001011960586811492E
:108DE80001405960196821F0847121F480311960BB
:108DF800196821F480211960596821F4FE0159602D
:108E0800D96A21F00F01D962186B0749014019632B
:108E1800002199604FF000639360704700ED00E017
:108E2800001002400CC07FF8CCFC00FF0A4B10B5C4
:108E380019684FF6FB720A401A60084A917A084A84
:108E48001C4609B1052300E001231360FFF7BAFFB0
:108E58004FF43643236010BD405C0040600F002093
:108E6800F82000202DE9F341A14EA24C33689BB2B3
:108E7800A383A28BE38B1A40950507D54FF6FF52C3
:108E880032609D4A11780131C9B21170A28B13402A
:108E9800180440F1EF820023ADF802303368954D95
:108EA8009AB21F04A28340F1E582AA8B02F00F0256
:108EB80085F82020002A40F0AE82904B1A6892B2C2
:108EC8006A846A8C02F03002AA846A8C02F44052E6
:108ED8006A8419684BF6BF720A4082F4005282F025
:108EE800200242F4004242F080021A60AA8BD106A6
:108EF8001FD4196848F60F720A401A60AB6A1A7ACA
:108F0800022A01D0042A02D1FEF787FE4AE2062A85
:108F180040F05B825A78052A08D11A78520605D1A2
:108F2800D878FBF70DFFEB6A1B6A9847236B9B68A1
:108F38004AE21A6892B2ADF80220BDF8022017057D
:108F480040F1C68119686E4F40F68F720A401A6068
:108F58003A686C4B92B213445B001A68AB6A197A90
:108F6800092917D092B2520002F1804202F5C0429C
:108F780011781970517859709188C8B2090A41EA74
:108F8800002159801189C8B2090A41EA0021998053
:108F98009289DA8001221A72DA885D78002A40F014
:108FA800D7801A7812F07F0248D1092D0AD1DA78D1
:108FB800012A20D89978F1B99988E1B99A72E36AB7
:108FC8005B6829E0052D11D193F90320002AC0F22E
:108FD800FC819A78002A40F0F8819A88002A40F0AB
:108FE800F4819B7A002B00F0A680EEE1032D15D1C9
:108FF800DA78012A07D0236B28465B69984703284B
:1090080040F09680A2E09A88002AF4D15A7A42F079
:1090180020025A72E36ADB6998478CE0012DEAD195
:10902800DA78012AE7D19A88002AE4D15B7A98068F
:10903800E1D5FBF7D5FD00287DD0DCE7012A1FD15B
:109048000B2DD8D1226B58799269D978DFF8A48092
:109058009047A36A9A7A002ACDD00028CBD11A79F2
:10906800002AC8D19B78002BC5D1D8F82C30DB68F2
:109078009847D8F828305A79DA72DA781A735AE0A9
:10908800022AB8D1012DD4D0032DB4D1597921F0B9
:10909800800E4FEA8E0202F1804000F5B84011F0D0
:1090A800800F006814BF00F0300000F44050BEF19B
:1090B800030FA0D8B3F802E0BEF1000F9BD100283F
:1090C80099D09B7A002B96D009061DD502F18042D3
:1090D80002F5B842136823F4E04323F040039BB23F
:1090E80083F0100343F4004343F0800313601CE053
:1090F800445C0040600F0020F7200020005C004026
:10910800505C00400430002002F1804303F5B8436E
:109118001A6822F4804222F0700292B282F48052DD
:1091280042F4004242F080021A60E36A9B6973E7E6
:10913800002840F04A813A689C4B92B213445B0085
:1091480000221A603023A38406233FE109233DE16E
:10915800062D12D11A78520677D19B78012B02D1AD
:10916800236BDB6968E0022B02D1236B1B6A63E087
:10917800032B6AD1236B5B6A5EE0002D3CD15988D2
:10918800002962D15A6822F47F42B2F5003F5CD1CF
:109198001A7812F07F0204D19B88002B00F0E0813E
:1091A80053E0012A0CD1226B587992699047002824
:1091B8004BD17F4B9B6A9B7A002B40F0D18144E0D6
:1091C800022A42D15B7903F00F010AB2920002F140
:1091D800804202F5B84213F0800F126814BF02F003
:1091E800300202F4405203292FD813F0700F2CD10B
:1091F800002A40F0B58128E0082D04D11B785F06CD
:1092080000F0B08121E00A2D1FD11A7802F07F0208
:10921800012A1AD19A7AC2B15988B1B95A6822F486
:109228007F42B2F5803F10D1226B587992699047FE
:10923800002800F0998108E03BB1A26A0025558218
:10924800936128469847284609E0226BA36A126969
:1092580058789047032802D1554B9B6A06E0A36AC9
:1092680053491A8A4FF6FF75AA4201D1092203E031
:10927800022800D012B908221A72A9E093F9000056
:1092880000281FDAD8880190019DAA4202D9019AC4
:109298001A8210E082420ED2096B91F82C108A4291
:1092A80001D2002105E092FBF1F001FB102212B976
:1092B8000121404A1170226B92F82C209A82FEF705
:1092C800ACFC85E003221A724FF440534B847FE0D4
:1092D800BDF8022012B2002ABFF6E0AD1968AD6AE7
:1092E80040F68F720A401A602B7A022B6DD0042B3D
:1092F8006BD0032B01D0052B62D1AB692A8A83B9C5
:109308002B8A002B37D04FF4405262842A4A1168C6
:10931800264A89B20A445200002111603022A284F0
:1093280029E0002AECD0B5F81480904528BF904673
:109338001FFA88F7384698472B8ADB1B2B826B8AE3
:109348001F441D4B6F821A681C4B92B213445B007A
:1093580008F101081B8803F1005303F54053590035
:109368004FEA680800234345CAD051F8232020F863
:1093780013200133F7E7AA8A9A4202D8A36A032284
:1093880002E01BB1A36A05221A720BE0A26A062149
:109398001172094A1168054A89B20A4452001360D9
:1093A8003023A384A36A1B7A10E000BF0230002098
:1093B800600F0020F6200020505C004004300020A0
:1093C800072B02D1236BDB6898470823A26A137224
:1093D800FBF796FC674B1A684BF6BF731340628C19
:1093E800D504628C48BF83F480539004A28C48BF94
:1093F80083F40053D106A28C48BF83F01003920671
:1094080048BF83F0200343F4004343F08003594AE4
:109418009BB213602EE0930003F1804303F5B84339
:10942800196889B2ADF80210BDF8021009B2002916
:1094380009DA186840F68F7101401960013A4E4BFD
:1094480053F822309847BDF802301B067FF526AD49
:1094580094F820108B0003F1804303F5B84348F6D5
:109468000F72186802401A60434B03EB81018B6945
:10947800984713E5A28BE38B1340580505D54FF6A3
:10948800FF3333603D4B5B689847A38BE28B1340F7
:10949800990444BF4DF6FF733360A18B384B0A40E3
:1094A800D20463D54EF6FF723260002283F834206E
:1094B80093F83430052B4FD8DFE803F0030E161B62
:1094C8002A37A36B2E4D1BB9FFF7B0FC062300E02B
:1094D800052385F8343049E0FFF7A8FC042384F815
:1094E80034300123A36341E0022384F83530032399
:1094F80033E094F83530013BDBB284F8353094F82A
:109508003530002B32D11E4B042283F834202DE055
:109518001C4B1A6892B242F010021A60052384F8B4
:1095280034300A2384F8353020E094F83530144A72
:10953800013BDBB284F8353094F8353003F0FF0096
:10954800A3B910490C684FF6EF7323400B6006234C
:1095580082F83430906309E0062384F8343005E05B
:10956800094B6AE6094B68E6094B66E602B0BDE8B6
:10957800F08100BF005C0040000D0108E4000020FD
:10958800600F0020405C0040ED460008A547000839
:1095980081470008024B4FF480221A60704700BFD1
:1095A80014040140704770477047FEE7FEE7FEE786
:1095B800704702480249FAF7C1BA00BF00480140A3
:1095C8003C10002001480249FAF7B8BA00400140AF
:1095D8001410002001480249FAF7B0BA000400400C
:1095E800EC0F00204FF080400149FAF7A7BA00BFFE
:1095F800C40F002001480249FAF7A0BA002C014024
:109608009C0F002001480249FAF798BA002C014043
:109618009C0F00200148FDF7B1BA00BF641000207C
:109628000148FDF7ABBA00BFB81000200148FDF7AC
:10963800A5BA00BF0C110020054B064820225A602D
:10964800DA6922F001021204120CDA6100F09FBEFE
:109658000000024064100020074B08484FF00072D9
:109668005A60D3F8802022F001021204120CC3F8C9
:10967800802000F08CBE00BF00000240B81000201F
:10968800064B07484FF400525A605A6C22F0010208
:109698001204120C5A6400F07ABE00BF00000240A7
:1096A8000C11002082B01B4A1B4B8DF80710116863
:1096B800186860B31B68052B29D1184B186820B1AE
:1096C80013685B1A312BF8D921E09DF808109DF832
:1096D800072042EA0121124A1180A2F5A662116808
:1096E800104A89B20A445200012111601A680A44DA
:1096F8001A600D4A136823F4E04323F040039BB239
:1097080083F0300343F4004343F08003136002B056
:10971800704700BF001A0020F820002060110020C8
:10972800806100400A300020045C0040244B25483A
:10973800196870B54FF47A73B1FBF3F1224B234DDE
:109748001A78234B1B78FCF7A5FE22482E6848217F
:10975800FCF7A0FE0024E2B21F4B53F8221049B1D7
:10976800012303FA02F2324202D01C48FCF792FEAF
:109778000134F0E72A6892070DD5194A194812787A
:1097880003EB8203196AFCF785FE174B197A11B1AE
:109798001648FCF77FFE1648F9F768FE154B164881
:1097A8001A68164B9A420CBF154B164B1A88164B63
:1097B80092B21988BDE870404FF4D763FCF76ABECF
:1097C800001A00207F230108040A0020FC02002060
:1097D80050010020BD2301083C0D0108961D010819
:1097E800F1200020DB23010808050020E5230108FB
:1097F800B424010824070020E9230108005400408C
:109808006C0A00206E0A0020AC05002070B50546E1
:109818002E482F4B00684FF420445C60866936045C
:1098280016D446682B4C344044F0807444F4903489
:109838002C4344604FF420445C608669B6071BD50E
:109848004FF4204481625C6081690E0619D51EE0E0
:10985800661E0CB13446E1E75E6007E02146846984
:10986800A40721D44C1E0029F8D15C60FAF7E0F96E
:10987800003018BF012070BD661E002CECD03446A5
:10988800DBE7611E0CB10C46DEE75960EEE7446881
:109898001049214041F0007141F480312943416071
:1098A8004FF420415960DAE782624FF420425A604F
:1098B8008169890604D55A602023C361012070BDDF
:1098C800511E002AE1D00A46F2E700BF2407002013
:1098D80060110020009800FC024640213C2095E7DA
:1098E800024680213C2091E708B55038C0B2FFF706
:1098F800F7FF0020FFF7F4FF1020BDE80840EFE76E
:10990800F8B5A44B1B680446187818B1012800F074
:10991800FD806BE2242CA04D0CD006D80A2C00F058
:109928008F800D2C00F08C80DCE02A2C06D02C2CAB
:1099380004D0D7E028726872A872E4E06A7A2E7AB6
:10994800954B2A440021D172EEB9DA7A9E76472ADD
:1099580019D11A7B502A16D15A7B472A07D19A7BEC
:10996800472A04D1DA7B412A01D101229A766A7BFF
:10997800894B522A07D19A7B4D2A04D1DA7B432A94
:1099880004BF02229A76AB7E834F012B02D0022BB2
:1099980037D04AE0B31E072B47D8DFE803F00408A6
:1099A80010141C27462DFCF787FCE8613DE0EA7A95
:1099B800794B532A39D1DA695242DA6135E0FCF73A
:1099C8007BFC286231E0EA7A734B572A2DD11A6A58
:1099D80052421A6229E0EB7A302B704B1A788CBF0E
:1099E80042F0020222F002021A701EE00020FCF788
:1099F800BFFC85F8240018E00020FCF7B9FCE884D7
:109A080013E0072E06D0082E0FD10120FCF7B0FC7A
:109A180078850AE00120FCF7ABFC41F21843584373
:109A28004FF47A72B0FBF2F33B85013600202A2C02
:109A3800594B2E72687261D1012283F82C2062E0A2
:109A480095F82C00002849D01423554A013B991851
:109A5800985C4870002BF8D1EB7A402B04D9A3F11D
:109A680037010901C9B202E01B0103F0F0012B7BA9
:109A7800A87A402B8CBF373B303BDBB21944C9B2C4
:109A88008842454B27D121201070464A4449106826
:109A980001301060987E01280AD002281DD1722258
:109AA8000A70414A198D11805A8D404B1A8014E072
:109AB80067220A70394A127896070FD53C4AD96945
:109AC8001160196A51603B4A93F824101170DA8CBE
:109AD800394B1A8002E03F2313700020002385F8D9
:109AE8002C3010E06B7A2C4A0E2B03D8591C1344E7
:109AF8005172DC7295F82C00274B18B99A7A5440A9
:109B08009C7200E0002000F00100F8BD224B93F8A1
:109B18002D100022082900F26981DFE801F0050C08
:109B2800101A2B4F7392A300B52C40F05F8183F875
:109B38002E20012282E0622C08BF02227EE003224E
:109B480083F82D2083F82F4083F8304083F8314084
:109B58004CE1042283F82D2093F8302093F831103B
:109B680083F832402244D2B283F830200A4483F882
:109B780031203BE1052283F82D2093F8302093F81B
:109B880031109C862244D2B283F830200A4483F8EC
:109B980031202BE18C04002060110020910400206A
:109BA800E8090020580F0020720A0020740A0020DB
:109BB800880B002090040020700A00200622988E4E
:109BC80083F82D2093F8302093F83110224400EBCD
:109BD8000420D2B280B283F83020B0F5AC7F0A44BA
:109BE80083F83120988603D9814A012182F82E1002
:109BF8000022DA86002840F0F9807D4B072283F89E
:109C08002D20F8BD93F8302093F831102244D2B2B9
:109C180083F830200A4483F83120DA8EB2F5AC7F1D
:109C280003D27349114481F83840013292B2DA867E
:109C38009B8E934200F2DA806D4B072283F82D2029
:109C4800D4E0082283F82D2093F83030A34200F0A6
:109C5800CD80674B012283F82E20664B5A6801326B
:109C68005A60C3E083F82D20142063490138421854
:109C7800455C55700028F8D193F831505C4AA542EC
:109C880006D03F230B705B4B5A6801325A60F8BD0F
:109C98005A4C25680135256092F82E4014B13E23B0
:109CA8000B70F8BD21240C7092F83240062C4CD071
:109CB80004D8022C14D0032C30D097E0122C62D098
:109CC800302C40F093804920087092F83C104C4AA0
:109CD800102988BF1021117010784A49002262E0CB
:109CE800502008704849D06B4860106C0860916C2F
:109CF8004FF47A7091FBF0F14448018092F890118A
:109D0800434A19B1117841F0020102E0117821F0BB
:109D180002011170012283F8912159E053240C703B
:109D280092F83D10CD0704D592F83C00C41E60425D
:109D3800604100F0010083F89001002848D1344ABE
:109D4800117821F00201117042E04F240C7092F852
:109D58004310C90704D592F84200C21E5042504130
:109D680000F0010083F8900120B9294A117821F008
:109D780002011170274A93F867101170264AB3F848
:109D88006410118024E0562008702448D16C0180AA
:109D9800116D42F2107091FBF0F121480180012110
:109DA80082F8921114E0824201F10C0110D21D4C8C
:109DB80011F8045C15551C4C11F8035C15551B4C27
:109DC80011F8015C15551A4C0D7815550132EAE762
:109DD80093F89131064A4BB192F8923133B100238E
:109DE80082F8913182F892310120F8BD0020F8BD47
:109DF800601100206C040020E8090020580F0020A2
:109E08007B0A002098110020880B0020700A00208F
:109E1800910400209004002078010020720A00209C
:109E2800740A00207C0A00208C0A00209C0A00206A
:109E3800AC0A00202DE9F04106460F469046002561
:109E4800EBB2434513D20024E3B2B3420AD2094B22
:109E58009A8A92B282F010029A823846FDF7CEFEB4
:109E68000134F1E73C20FDF7C9FE0135E8E7BDE81C
:109E7800F08100BF000400480B490B7813F0010F74
:109E880003F004020AD072B9980707D443F0040318
:109E98000B70064B1A88064B1A8070471AB90220B5
:109EA800FF210122C6E77047F0200020900500201E
:109EB800380A002008B50D4B202240F2DB141A8521
:109EC800604310229A61841E084B9A8A92B282F0EB
:109ED80020029A829A8A92B282F0100220469A82CE
:109EE800FDF78CFE1920FDF789FEEDE70004004818
:109EF800454B56222DE9F3411A704FF4D7625A8028
:109F0800BE221A71EF2283F8B426002283F8B52600
:109F180011461E46B35C0132B2F5D76F81EA0301E0
:109F2800F8D1394B83F8B516384B1A69120604D59F
:109F3800374A5A6002F188325A6004270020013FEC
:109F480017F0FF074FD0314B3422DA60002444B1B8
:109F5800002356F804800193FCF7A6FB0428EED1F1
:109F680017E0FCF7A1FB0428E9D1284D2B6943F041
:109F780002032B61274B6B612B6943F040032B6174
:109F8800FCF792FB2B69042823F002032B61DFD036
:109F9800D5E71E4D2B6904F1006243F0010302F579
:109FA8007E322B611FFA88F31380FCF77DFB0428AF
:109FB80010D1194A22440192019B4FEA1848A3F88C
:109FC8000080FCF771FB2B69042823F001032B6147
:109FD80005D0B4E72B6923F001032B61AFE7043404
:109FE800B4F5D76FB3D1094B1A69042842F080023F
:109FF8001A6102D1FBF746FE10B90A20FFF75AFF93
:10A0080002B0BDE8F08100BF041A00200020024021
:10A018002301674500F8030802F8030837B582886A
:10A028008368044610060D4606D52B4991F8941608
:10A038004FF4E07000FB0133D10505D527490978B5
:10A0480001EB810103EB410302F03F02042A12D025
:10A0580006D8012A0DD0022A32D193F9001030E037
:10A06800102A0AD0202A0AD0082A29D1B3F90010C8
:10A0780027E0197825E0198823E0196821E093ED95
:10A08800000A6846FCF7B6FB01461548FCF702FAD9
:10A0980005B3D4ED037A6846B8EEE70AFCF7AAFBE5
:10A0A80001461048FCF7F6F994ED040A6846B8EE44
:10A0B800C00AFCF79FFB01460A48FCF7EBF909E0E8
:10A0C80000210948FCF7E6F925B10848E16822694A
:10A0D800FCF7E0F903B030BD041A0020640B00203F
:10A0E800E2230108E12301081D2301088324010854
:10A0F8002DE9F041002407462546114BE65839461C
:10A10800304604EB030803F02DFE58B10D483146E4
:10A11800FCF7C0F940460021FFF780FF0A48FCF72A
:10A12800B9F90135143440F618339C42E5D125B904
:10A138000648BDE8F041F9F799B9BDE8F08100BFDC
:10A14800F00E0108E6240108B42401088A24010855
:10A158002DE9F0472DED028B044603F0C7FD0546B7
:10A1680020B1012819D123782A2B16D15548F9F79F
:10A178007DF90024544B5548E158E618FCF78AF954
:10A1880030462946FFF74AFF5148F9F76FF914346A
:10A1980040F618339C42EDD18FE020463D2103F074
:10A1A80098FD002800F08380034613F8012C202A2C
:10A1B80001D1013BF9E7451C2846C4EB030903F02C
:10A1C800EAFD82462846F9F797FA0025B0EE408A5C
:10A1D80014226A433C4BD7583846D61803F086FDFC
:10A1E800804639462046424603F088FD002854D16F
:10A1F8005FFA89F3434550D196ED037AF8EEC77AB2
:10A20800B4EEE78AF1EE10FA45DB96ED047AF8EE43
:10A21800C77AB4EEE78AF1EE10FA3CD8B388B28870
:10A2280013F0200F08BF08EE10AA140618EE101A33
:10A23800B36806D5274890F894064FF4E07404FBF9
:10A248000033D00505D52448007800EB800003EBE7
:10A25800400302F03F02042A0BD004D8013A012A35
:10A268000DD819700BE0102A05D0202A05D0082A2D
:10A2780005D1198003E0196001E083ED008A3946B1
:10A288001648FCF707F9BDEC028B30460021BDE803
:10A29800F047FFF7C3BE124803E001358E2D97D172
:10A2A8001048BDEC028BBDE8F047F9F7DFB8BDEC0C
:10A2B800028B2046BDE8F0471AE7BDEC028BBDE8EB
:10A2C800F08700BFA2240108F00E0108E624010867
:10A2D800B4240108041A0020640B0020B7240108E4
:10A2E800C22401088A24010830B51049104A0C78A4
:10A2F800104B8CB11C6815680444A54215D312682C
:10A308001A600D4B1A78002008700AB1013A1A70C9
:10A318000A4B01221A7030BD18681468C83084428C
:10A3280003D30120126808701A6030BD5F0A00204C
:10A33800001A00209C0D00204A050020990D0020DD
:10A348000449054B0968187000225A6199611A7707
:10A35800704700BF001A00206C040020826A8169DF
:10A36800436B1144D960416A914203D98A1A5A60F1
:10A37800816204E001698A1A5A600022826200221E
:10A3880080F844201A6842F001021A607047416B55
:10A3980010B50C684FF6FE7222400A60416A826A64
:10A3A800914202D0BDE81040D8E7012280F844204D
:10A3B80010BDF8B50468054620460E461746F9F75D
:10A3C800FCFB042843D82B7B9B089AB246B94FF074
:10A3D800020C0CFA03F3E168DB439BB20B40E36029
:10A3E8000A211B4B01FB002143F82160043143F88B
:10A3F800217046B12A7BE1689208022505FA02F22B
:10A4080092B20A43E260282202FB003000F12002E7
:10A41800EFF31286502383F312880023C1180D69C5
:10A4280015B115600A6904320433102BF6D10023E4
:10A438001360F3B283F31188036A1BB1E36843F036
:10A44800010303E0E2684FF6FE731340E360F8BDD2
:10A458009C0F002070B5046D427923688568064614
:10A4680023F0010302F0040094B0236000F0FF0120
:10A4780020B14FF480614FF4005000E0084612F01C
:10A48800010F14BF0423002312F0020F18BF43F07A
:10A49800080312F0080F226822F0010222606268A5
:10A4A80022F4405240EA02006060226822F4B0526E
:10A4B80022F00C0218BF0C230A4313432360A3683D
:10A4C80023F44073A3606846FAF756FC194B9C4284
:10A4D80001D10C9A0EE0184B9C4201D10D9A09E06B
:10A4E800164B9C4201D10E9A04E0154B9C420CBFBE
:10A4F8000F9A109A2368190448BF5200B2FBF5F36B
:10A5080005FB1322B2EB550F226828BF0133120452
:10A5180006D54FF6F072C3F342011A4041EA02032E
:10A528009BB2A381336D1A6842F001021A6014B01D
:10A5380070BD00BF003801400044004000480040A2
:10A54800004C0040417185E7816083E770B506469D
:10A5580000240B4BE518AA8816420AD0E15809488E
:10A56800FBF798FF28460021FFF758FD0648F8F743
:10A578007DFF143440F618339C42EAD170BD00BF09
:10A58800F00E0108E2240108B4240108224B5343C9
:10A59800224A10B5224CB2FBF3F20388013AA042DA
:10A5A80001F1FF3192B29BB20ED004F50064A042D3
:10A5B8000AD0B0F1804F07D0A4F59834A04203D058
:10A5C80004F58064A04202D123F070039BB2154CBD
:10A5D800A04206D004F58064A0421CBF23F4407357
:10A5E8009BB203800E4BC162984202850FD003F5DF
:10A5F800006398420BD003F54063984207D003F5F7
:10A608008063984203D003F58063984201D1002308
:10A6180003860123436110BD40420F0000A24A0493
:10A62800002C0140001000402DE9F3477B4E37789D
:10A6380005460C46006811469246984622467B1C01
:10A6480006F8043BFFF7A2FFAB68ADF80430686872
:10A65800022301A98DF806308DF80730FAF75DFD61
:10A668002B7B2C683F0106EB07090C2B00F2AB8013
:10A67800DFE803F007A9A9A93BA9A9A964A9A9A981
:10A688008A00236A664823F001032362216A63680B
:10A69800A26922F4803222F07302844242F07002EE
:10A6A80012D000F5006084420ED000F5406084426C
:10A6B8000AD000F58060844206D000F580608442AC
:10A6C80002D041F0030107E021F00E0123F44073AA
:10A6D80041F0030143F480736360A261C4F83480DD
:10A6E8002162A36943F0080326E0236A4C4823F05B
:10A6F80010032362216A6368A26922F0807222F43F
:10A70800E642844242F4E04206D000F5006084420A
:10A7180002D041F0300107E021F0E00123F440636A
:10A7280041F0300143F480636360A261C4F838806B
:10A738002162A36943F40063A36144E0236A3848B3
:10A7480023F480732362226A6368E169844221F0FA
:10A75800730141F0700106D000F50060844202D018
:10A7680042F4407207E022F4606223F4405342F45A
:10A77800407243F480536360E161C4F83C80226214
:10A78800E36943F008031DE0236A254823F4805356
:10A798002362226A6368E169844221F4E64141F454
:10A7A800E04142F4405203D000F50060844201D1F8
:10A7B80043F480436360E161C4F840802262E36946
:10A7C80043F40063E361AB7B1BB1636C43F4004368
:10A7D800636423889BB243F0010323802B7B0C2BFB
:10A7E80014D8DFE803F0071313130A1313130D1318
:10A7F8001313100004F1340307E004F1380304E0F4
:10A8080004F13C0301E004F14003F3514846A9F880
:10A8180008A0C9F8044002B0BDE8F087F41200208F
:10A82800002C01400D4B0278D9684378C943C1F325
:10A838000221C1F1040103FA01F1094B09011A448B
:10A84800C9B282F8001302780120510902F01F02F0
:10A8580000FA02F243F82120704700BF00ED00E043
:10A8680000E100E02DE9FF411D46714B98420F467B
:10A87800164672D16F4B704A1A60704A5A6102F5D7
:10A8880080729A614FF48072DA601A616C4A1A63B6
:10A89800143A5A63A2F54842203ADA6404329A64B8
:10A8A8009E601865674B9A6942F480429A615A69BA
:10A8B80042F001025A6102238DF80C3003238DF80F
:10A8C8000D3000238DF80E30AA074FF001038DF8E4
:10A8D8000F300ED504A9402341F8083D5A48036AB1
:10A8E80023F070630362036A43F0E0630362FAF7DC
:10A8F800D5FBEB070ED504A9802341F8083D524843
:10A90800036A23F070430362036A43F0E04303627F
:10A91800FAF7C4FB2C0710D54B48402302930123B8
:10A928008DF80E30036A23F070630362036A43F004
:10A93800E063036202A9FAF7B1FB0E238DF8043035
:10A948000022012301A88DF805308DF806208DF826
:10A958000730384CFFF766FFE8E03C4B98427BD164
:10A968003B4B354A1A604FF48072DA601A61394AF3
:10A978005A6102F580729A6118659E60314BDA69F6
:10A9880042F40032DA6102238DF80C3003238DF88B
:10A998000D3000238DF80E30A8074FF001038DF815
:10A9A8000F300FD504A9042341F8083D4FF090401B
:10A9B800036A23F470630362036A43F4E063036287
:10A9C800FAF76CFBE9070FD504A9082341F8083DFD
:10A9D8004FF09040036A23F470430362036A43F420
:10A9E800E0430362FAF75AFB2A0711D54FF090406B
:10A9F8000423029301238DF80E30036A23F4706355
:10AA08000362036A43F4E063036202A9FAF746FBB0
:10AA180026238DF804300022012301A88DF8053083
:10AA28008DF806208DF80730094CFFF7FBFE7DE016
:10AA3800003801400C1100208C0D0108B8130020CB
:10AA48005800024000100240000400480044004042
:10AA5800B8100020B8150020714B984240F0DB80F8
:10AA6800704B714A1A604FF48072DA601A616F4A4B
:10AA78005A6102F580729A619E6018656C4BDA69BA
:10AA880042F48022DA6102238DF80C3003238DF81A
:10AA98000D3000238DF80E3001238DF80F30AB07F1
:10AAA8000FD504A94FF4806341F8083D6148436A13
:10AAB80023F470634362436A43F4E0634362FAF742
:10AAC800EDFAEC070FD504A94FF4006341F8083DEF
:10AAD8005848436A23F470434362436A43F4E043AB
:10AAE8004362FAF7DBFA280711D552484FF480631E
:10AAF800029301238DF80E30436A23F47063436296
:10AB0800436A43F4E063436202A9FAF7C7FA2723CA
:10AB18008DF804300022012301A88DF805308DF846
:10AB280006208DF80730FFF77DFE3E4C012384F8A0
:10AB3800443000232362E361A3626362E7626571C4
:10AB4800A660A3712046FFF785FC15F0090F29D0F0
:10AB5800206B00B3E76CD4F80C806669F9F7A8FF9E
:10AB6800236B1A6822F4FF4222F0700242F48552E5
:10AB78001A601FFA88F25A609F60DE601A6842F015
:10AB880001021A60226D916841F0400191605B6892
:10AB98009BB2236406E0236D20221A621A6842F0F1
:10ABA80020021A6015F00A0F26D0606BF8B1A66C67
:10ABB8002769F9F77DFF636B1A6822F4FF4222F0D8
:10ABC800700242F4845242F010021A60BFB20022AE
:10ABD8005F609E60DA60196841F0020119605A608E
:10ABE8005A60236D9A6842F080029A6004E0236DEF
:10ABF8001A6842F080021A60236D1A6842F0010256
:10AC08001A609A6829074CBF42F0080222F008022D
:10AC18009A60204600E0002004B0BDE8F08100BF43
:10AC280000480040641000208C0D0108B81700206F
:10AC380000100240000400482DE9F04F8DB01E4678
:10AC480083460D4614469DF85890FBF7B1FB0DF16D
:10AC5800200E0746034600F1100C18685968724622
:10AC680003C2083363459646F7D13B7B0BB9099479
:10AC78000A94584608A9FDF731FB074610B94FF06A
:10AC8800000813E14368D3F80480B8F1000F05D039
:10AC9800584608A93A46F8F736FAEEE703780593D6
:10ACA80083681B780493032B00F20081DFE813F01C
:10ACB8000400D400D800DC007E4DAB6943F00103EA
:10ACC800AB616B694FF0904643F400336B6101242C
:10ACD8004FF0000903224FF4805A06A94FF0904024
:10ACE8008DF81D200392CDF818A08DF81C408DF822
:10ACF8001E408DF81F90FAF7D1F9A6F828A0C820B1
:10AD0800FCF77CFFC6F818A06B69039A43F400337C
:10AD18006B6130464FF4C0538DF81D2006A90222FE
:10AD280006938DF81C2003928DF81E908DF81F90C5
:10AD3800FAF7B4F9736A039A23F470437362736A77
:10AD480043F460437362736A23F470237362736A13
:10AD580043F460237362584B584E4FF480211960B6
:10AD680012233363082386F83530554B86F836406E
:10AD7800196821F480211960596821F480215960EB
:10AD880096F8343003F1804303F58233196841F4AF
:10AD980080211960306B4B4B20F01F0100F01F0021
:10ADA80051F803E004FA00F02EEA0000C850D6F883
:10ADB80030E045492EF01F000EF01F0E50F801C07C
:10ADC80004FA0EFE2CEA0E0E40F801E0306B20F07B
:10ADD8001F0100F01F0051F803E004FA00F04EEAEA
:10ADE8000000C850394B3A49C3F80090EB6943F466
:10ADF8000003EB61374B06A8D96014238DF818308F
:10AE08008DF819208DF81A908DF81B40FFF70AFD70
:10AE18002A238DF818309DF81B308DF819408DF8CD
:10AE28001A901BB106A8FFF7FDFC04E02A4B4FF46B
:10AE38008062C3F88420294A294B136002221A72BF
:10AE4800284A294B1360294A29491B6811609847E9
:10AE5800284B3360194812E0CDF80090264806E0E8
:10AE6800CDF80090254802E02548CDF80090294605
:10AE780022463346FFF7F6FC00283FF400AF049A59
:10AE880002710E4B059A03EB820398637B68586046
:10AE980000231C4A1A445168814203D00C33302BDA
:10AEA800F7D100E0904688F809B0804640460DB0DA
:10AEB800BDE8F08F0010024014040140B8190020CA
:10AEC80000040140080401400C040140D80042423B
:10AED8000005FA0500ED00E000E100E0880F002021
:10AEE800600F0020900F0020E40000208C0F00204D
:10AEF80014010020A40D010800380140004400405E
:10AF080000480040140000202DE9F3414020F8F7E4
:10AF180041F980B1446874B12046F8F705FA18B9C8
:10AF28000A20FCF76BFEF7E72E4B1B6820461969D1
:10AF3800F8F7FFF90BE02B4B00211B6800911A6909
:10AF480040200323FFF778FE0446002843D0254B12
:10AF5800254D1B682868D968F8F7EBF92868417906
:10AF68008A0704D4036841F002015B6998471F4BC4
:10AF780010229A6120229A612868F8F7E4F990B1C2
:10AF88001A4E10233385184B1868F8F7D7F9074677
:10AF9800FEF7B6FC08B1FCF75BF920463946F8F72E
:10AFA800D7F91023B3612046F8F7CDF960B10F4EF9
:10AFB800D5F80080202737852046F8F7BFF90146E5
:10AFC8004046F8F7C5F9B761094B9B689B03D3D591
:10AFD800FDF730FCD0E7074802B0BDE8F041F8F7CC
:10AFE80045BA00BFE40900206804002000040048B6
:10AFF800041A0020EC2401082DE9F047054602F068
:10B0080075FE304B0446D3F808809A4690B92E480E
:10B01800F8F72CFA2D4B53F8241049B10123A3401B
:10B0280013EA080F02D02A48FBF734FA0134F1E793
:10B03800284821E028462849224602F05FFE58B9F0
:10B048002648274CF8F712FA54F8041F0029EFD0C5
:10B058001F48FBF71FFAF7E72B782D2B03BF0135A5
:10B0680004F1FF344FF001094FF000090026174B97
:10B0780053F8267027B91B48BDE8F047F8F7F6B92A
:10B0880028463946224602F039FEC8B90120B040A8
:10B09800830501D51448EFE7B9F1000F03D0F8F79D
:10B0A8004AFC124804E040EA0800CAF808001048C0
:10B0B800F8F7DCF939460F48BDE8F047FBF7EAB97D
:10B0C8000136D4E7041A0020E2260108A00E010880
:10B0D800961D0108B424010857260108F526010821
:10B0E8009C0E01080A2701082127010835270108B5
:10B0F8003F2701086A1D0108084A13689B050BD5FC
:10B10800074B00211970074908684FF6FE73034082
:10B118000B604FF400735360704700BF000002409B
:10B12800FC20002030000240024B1A6801321A60ED
:10B13800704700BF001A002008B5084BB3F8D800C4
:10B1480093F8BC260023D9B2914204D2044921F8CD
:10B1580013000133F7E7FAF76DFEFEE7001A002047
:10B16800BE20002073B96AB9002908BF0028BCBFF7
:10B1780000204FF00041C4BF6FF000414FF0FF3096
:10B1880000F03CB882B0EC462DE9005000F006F81B
:10B19800DDF804E002B00CBC704700BF2DE9704335
:10B1A800069E14461D468046894600F029F804FB91
:10B1B80001F300FB0533A4FB00451D44B8EB040470
:10B1C80069EB0505C6E90045BDE870832DE97043C4
:10B1D800069E1446804689461D4600F05DF900FB30
:10B1E80005F504FB0153A0FB04451D44B8EB04041A
:10B1F80069EB0505C6E90045BDE87083704700BFE7
:10B2080000292DE9F00FC0F29F800024002BC0F226
:10B218009680154606460F46002B3ED18A4257D9DE
:10B22800B2FA82F34BB1C3F1200201FA03F720FA14
:10B2380002F29D40174300FA03F6290CB7FBF1F21E
:10B24800330C01FB127CA8B243EA0C4700FB02F363
:10B25800BB4209D97F1902F1FF3C80F00181BB4252
:10B2680040F2FE80023A2F44FF1AB7FBF1F3B6B260
:10B2780001FB137146EA014100FB03F0884208D93B
:10B28800491903F1FF3780F0ED80884240F2EA80E7
:10B29800023B43EA0242002303E08B420AD900231F
:10B2A8001A461046194614B1404261EB4101BDE807
:10B2B800F00F7047B3FA83F8B8F1000F40F08480BC
:10B2C8008B4202D3824200F2DE8000230122E8E7AB
:10B2D80012B90123B3FBF2F5B5FA85F2002A39D188
:10B2E8007F1B280C1FFA85FC0123B7FBF0F1320CF9
:10B2F80000FB117742EA07470CFB01F2BA4207D973
:10B308007F1901F1FF3802D2BA4200F2C1804146EA
:10B31800BF1AB7FBF0F2B6B200FB127046EA004063
:10B328000CFB02FC844507D9401902F1FF3702D211
:10B33800844500F2AB803A4642EA0142B1E7E44371
:10B34800524263EB430364E7404261EB41014FF033
:10B35800FF345BE79540C2F1200327FA03F1280C7C
:10B3680026FA03F39740B1FBF0F81F433B0C00FBB0
:10B3780018111FFA85FC43EA01410CFB08F38B42C4
:10B3880006FA02F608D9491908F1FF3279D28B4238
:10B3980077D9A8F102082944C91AB1FBF0F3BFB262
:10B3A80000FB131147EA01470CFB03F2BA4207D925
:10B3B8007F1903F1FF3160D2BA425ED9023B2F44B4
:10B3C800BF1A43EA084390E7C8F1200203FA08FCD1
:10B3D80025FA02F343EA0C0C4FEA1C4921FA02F35E
:10B3E80001FA08F720FA02F2B3FBF9F1174309FB57
:10B3F80011333A0C1FFA8CFB42EA03430BFB01FAA8
:10B408009A4505FA08F008D913EB0C0301F1FF324D
:10B4180035D29A4533D902396344CAEB0303B3FBE7
:10B42800F9F209FB1233BFB247EA03470BFB02F9F3
:10B43800B94508D917EB0C0702F1FF331BD2B94500
:10B4480019D9023A674442EA0145A5FB0001C9EB54
:10B4580007078F424FF000030AD305D02A4620E79A
:10B46800624601E73B4614E706FA08F68642F5D23B
:10B478006A1E002315E71A46E5E70B46A0E71146C2
:10B48800CBE7904688E7434642460AE7023A53E745
:10B4980002392F443CE700BF2DE9F00F144605465A
:10B4A8000E46002B43D18A4253D9B2FA82F757B1DC
:10B4B800C7F1200620FA06F601FA07F302FA07F4A4
:10B4C8001E4300FA07F5210CB6FBF1F22B0C01FB29
:10B4D8001267A0B243EA074600FB02F3B34209D958
:10B4E800361902F1FF3780F0F680B34240F2F3805C
:10B4F800023A2644F61AB6FBF1F3ADB201FB13612A
:10B5080045EA014100FB03F0884208D9091903F113
:10B51800FF3680F0E280884240F2DF80023B43EA57
:10B528000242002310461946BDE8F00F70478B42CF
:10B538004AD8B3FA83F6002E4DD18B4202D3824209
:10B5480000F2D6800023012210461946BDE8F00F0C
:10B55800704712B90124B4FBF2F4B4FA84F2002A59
:10B568007CD1091B260CA7B20123B1FBF6F02A0CEB
:10B5780006FB101142EA014107FB00F28A4207D993
:10B58800091900F1FF3C02D28A4200F2C3806046EA
:10B59800891AB1FBF6F2ADB206FB121145EA014574
:10B5A80007FB02F7AF4208D92C1902F1FF3180F0EE
:10B5B8009680A74240F29380023A42EA004210463F
:10B5C8001946BDE8F00F704700231A461046194681
:10B5D800BDE8F00F7047C6F1200522FA05F4B34024
:10B5E8001C434FEA144821FA05F301FA06F720FA3A
:10B5F80005F5B3FBF8FC2F4308FB1C333D0C1FFA81
:10B6080084FA45EA03430AFB0CF9994502FA06FB5A
:10B6180004D91B190CF1FF326DD39446C9EB03030F
:10B62800B3FBF8F508FB1533BFB247EA03470AFB3B
:10B6380005F8B84504D93F1905F1FF3361D31D4614
:10B6480045EA0C4CACFB0B23C8EB07079F424FF0B5
:10B65800000549D345D062462B4663E79440C2F1C2
:10B66800200321FA03FC260C20FA03F301FA02F561
:10B67800BCFBF6F843EA05010B0C06FB18CCA7B295
:10B6880043EA0C4C07FB08F3634500FA02F509D9B5
:10B698001CEB040C08F1FF323AD2634538D9A8F103
:10B6A8000208A444C3EB0C0CBCFBF6F389B206FBFE
:10B6B80013CC41EA0C4107FB03F28A4207D9091966
:10B6C80003F1FF3022D28A4220D9023B2144891A51
:10B6D80043EA084349E73A460CE733461FE70A4678
:10B6E8006BE7B0409042B6D20CF1FF32002319E765
:10B6F8003346324616E799458FD9ACF1020C2344FC
:10B708008CE7B8459BD9023D274499E70346DEE715
:10B718009046C7E7023821443AE700BF81F000416C
:10B7280002E000BF83F0004330B54FEA41044FEA1E
:10B73800430594EA050F08BF90EA020F1FBF54EAB9
:10B74800000C55EA020C7FEA645C7FEA655C00F055
:10B75800E2804FEA5454D4EB5555B8BF6D420CDD26
:10B768002C4480EA020281EA030382EA000083EAA9
:10B77800010180EA020281EA0303362D88BF30BD49
:10B7880011F0004F4FEA01314FF4801C4CEA11319F
:10B7980002D0404261EB410113F0004F4FEA0333FE
:10B7A8004CEA133302D0524263EB430394EA050F89
:10B7B80000F0A780A4F10104D5F1200E0DDB02FAF8
:10B7C8000EFC22FA05F2801841F1000103FA0EF28C
:10B7D800801843FA05F359410EE0A5F120050EF152
:10B7E800200E012A03FA0EFC28BF4CF0020C43FA83
:10B7F80005F3C01851EBE37101F0004507D54FF090
:10B80800000EDCF1000C7EEB00006EEB0101B1F5DF
:10B81800801F1BD3B1F5001F0CD349085FEA300025
:10B828004FEA3C0C04F101044FEA445212F5800F30
:10B8380080F09A80BCF1004F08BF5FEA500C50F1CD
:10B84800000041EB045141EA050130BD5FEA4C0CB0
:10B85800404141EB010111F4801FA4F10104E9D139
:10B8680091F0000F04BF01460020B1FA81F308BF30
:10B878002033A3F10B03B3F120020CDA0C3208DDFC
:10B8880002F1140CC2F10C0201FA0CF021FA02F1D7
:10B898000CE002F11402D8BFC2F1200C01FA02F147
:10B8A80020FA0CFCDCBF41EA0C019040E41AA2BF6C
:10B8B80001EB0451294330BD6FEA04041F3C1CDA34
:10B8C8000C340EDC04F11404C4F1200220FA04F054
:10B8D80001FA02F340EA030021FA04F345EA0301FE
:10B8E80030BDC4F10C04C4F1200220FA02F001FAC0
:10B8F80004F340EA0300294630BD21FA04F0294642
:10B9080030BD94F0000F83F4801306BF81F48011DA
:10B918000134013D4EE77FEA645C18BF7FEA655C4D
:10B9280029D094EA050F08BF90EA020F05D054EA1F
:10B93800000C04BF1946104630BD91EA030F1EBF24
:10B948000021002030BD5FEA545C05D14000494128
:10B9580028BF41F0004130BD14F580043CBF01F51B
:10B96800801130BD01F0004545F0FE4141F4700101
:10B978004FF0000030BD7FEA645C1ABF19461046DC
:10B988007FEA655C1CBF0B46024650EA013406BFDD
:10B9980052EA033591EA030F41F4002130BD00BF9C
:10B9A80090F0000F04BF0021704730B54FF4806459
:10B9B80004F132044FF000054FF0000150E700BFDA
:10B9C80090F0000F04BF0021704730B54FF4806439
:10B9D80004F1320410F0004548BF40424FF0000126
:10B9E8003EE700BF42004FEAE2014FEA31014FEA69
:10B9F80002701FBF12F07F4393F07F4F81F06051B8
:10BA0800704792F0000F14BF93F07F4F704730B526
:10BA18004FF4607401F0004521F0004120E700BFB9
:10BA280050EA010208BF704730B54FF000050AE040
:10BA380050EA010208BF704730B511F0004502D541
:10BA4800404261EB41014FF4806404F132045FEA43
:10BA5800915C3FF4DCAE4FF003025FEADC0C18BFE8
:10BA680003325FEADC0C18BF033202EBDC02C2F1DE
:10BA7800200300FA03FC20FA02F001FA03FE40EA70
:10BA88000E0021FA02F11444C1E600BF70B54FF070
:10BA9800FF0C4CF4E06C1CEA11541DBF1CEA135552
:10BAA80094EA0C0F95EA0C0F00F0DEF82C4481EABA
:10BAB800030621EA4C5123EA4C5350EA013518BFDA
:10BAC80052EA033541F4801143F4801338D0A0FBC7
:10BAD80002CE4FF00005E1FB02E506F00042E0FB74
:10BAE80003E54FF00006E1FB03569CF0000F18BF7A
:10BAF8004EF0010EA4F1FF04B6F5007F64F5407422
:10BB080004D25FEA4E0E6D4146EB060642EAC621B4
:10BB180041EA55514FEAC52040EA5E504FEACE2E21
:10BB2800B4F1FD0C88BFBCF5E06F1ED8BEF1004F24
:10BB380008BF5FEA500E50F1000041EB045170BDA0
:10BB480006F0004646EA010140EA020081EA0301E4
:10BB5800B4EB5C04C2BFD4EB0C0541EA045170BDE0
:10BB680041F480114FF0000E013C00F3AB8014F15A
:10BB7800360FDEBF002001F0004170BDC4F10004A3
:10BB8800203C35DA0C341BDC04F11404C4F1200524
:10BB980000FA05F320FA04F001FA05F240EA02007F
:10BBA80001F0004221F0004110EBD37021FA04F6B5
:10BBB80042EB06015EEA430E08BF20EAD37070BD6F
:10BBC800C4F10C04C4F1200500FA04F320FA05F0CE
:10BBD80001FA04F240EA020001F0004110EBD370D0
:10BBE80041F100015EEA430E08BF20EAD37070BD40
:10BBF800C4F1200500FA05F24EEA020E20FA04F319
:10BC080001FA05F243EA020321FA04F001F00041C7
:10BC180021FA04F220EA020000EBD3705EEA430E38
:10BC280008BF20EAD37070BD94F0000F0FD101F067
:10BC38000046400041EB010111F4801F08BF013CA0
:10BC4800F7D041EA060195F0000F18BF704703F0DE
:10BC58000046520043EB030313F4801F08BF013D65
:10BC6800F7D043EA0603704794EA0C0F0CEA135521
:10BC780018BF95EA0C0F0CD050EA410618BF52EADB
:10BC88004306D1D181EA030101F000414FF00000E1
:10BC980070BD50EA410606BF1046194652EA4306EF
:10BCA80019D094EA0C0F02D150EA013613D195EA63
:10BCB8000C0F05D152EA03361CBF104619460AD1AB
:10BCC80081EA030101F0004141F0FE4141F47001B5
:10BCD8004FF0000070BD41F0FE4141F4780170BDA5
:10BCE80070B54FF0FF0C4CF4E06C1CEA11541DBF0A
:10BCF8001CEA135594EA0C0F95EA0C0F00F0A7F80C
:10BD0800A4EB050481EA030E52EA03354FEA013138
:10BD180000F088804FEA03334FF0805545EA13134B
:10BD280043EA12634FEA022245EA111545EA106513
:10BD38004FEA00260EF000419D4208BF964244F1AA
:10BD4800FD0404F5407402D25B084FEA3202B61AC9
:10BD580065EB03055B084FEA32024FF480104FF49D
:10BD6800002CB6EB020E75EB030E22BFB61A754611
:10BD780040EA0C005B084FEA3202B6EB020E75EBA4
:10BD8800030E22BFB61A754640EA5C005B084FEA0C
:10BD98003202B6EB020E75EB030E22BFB61A7546D9
:10BDA80040EA9C005B084FEA3202B6EB020E75EBE4
:10BDB800030E22BFB61A754640EADC0055EA060EA5
:10BDC80018D04FEA051545EA16754FEA06164FEAE8
:10BDD800C30343EA52734FEAC2025FEA1C1CC0D194
:10BDE80011F4801F0BD141EA00014FF000004FF021
:10BDF800004CB6E711F4801F04BF01430020B4F1E2
:10BE0800FD0C88BFBCF5E06F3FF6AFAEB5EB030C99
:10BE180004BFB6EB020C5FEA500C50F1000041EB96
:10BE2800045170BD0EF0004E4EEA113114EB5C0463
:10BE3800C2BFD4EB0C0541EA045170BD41F4801136
:10BE48004FF0000E013C90E645EA060E8DE60CEA3E
:10BE5800135594EA0C0F08BF95EA0C0F3FF43BAF5B
:10BE680094EA0C0F0AD150EA01347FF434AF95EA12
:10BE78000C0F7FF425AF104619462CE795EA0C0FF6
:10BE880006D152EA03353FF4FDAE1046194622E7C3
:10BE980050EA410618BF52EA43067FF4C5AE50EA9D
:10BEA80041047FF40DAF52EA43057FF4EBAE12E78D
:10BEB8004FF0FF3C06E000BF4FF0010C02E000BF6E
:10BEC8004FF0010C4DF804CD4FEA410C7FEA6C5C51
:10BED8004FEA430C18BF7FEA6C5C1BD001B050EAF4
:10BEE800410C0CBF52EA430C91EA030F02BF90EADF
:10BEF800020F0020704710F1000F91EA030F58BF9E
:10BF0800994208BF90422CBFD8176FEAE37040F0FF
:10BF1800010070474FEA410C7FEA6C5C02D150EA9D
:10BF2800013C07D14FEA430C7FEA6C5CD6D152EA58
:10BF3800033CD3D05DF8040B704700BF844610461D
:10BF480062468C461946634600E000BF01B5FFF71C
:10BF5800B7FF002848BF10F1000F01BD4DF808EDEC
:10BF6800FFF7F4FF0CBF012000205DF808FB00BFBD
:10BF78004DF808EDFFF7EAFF34BF012000205DF817
:10BF880008FB00BF4DF808EDFFF7E0FF94BF012064
:10BF980000205DF808FB00BF4DF808EDFFF7CEFF65
:10BFA80094BF012000205DF808FB00BF4DF808EDA4
:10BFB800FFF7C4FF34BF012000205DF808FB00BF75
:10BFC8004FEA4102B2F1E04324BFB3F5001CDCF1B3
:10BFD800FE5C0DD901F0004C4FEAC0024CEA5070EB
:10BFE800B2F1004F40EB830008BF20F0010070471A
:10BFF80011F0804F21D113F13872BCBF01F000401D
:10C00800704741F480114FEA5252C2F11802C2F14E
:10C01800200C10FA0CF320FA02F018BF40F00100CF
:10C028004FEAC1234FEAD32303FA0CFC40EA0C0081
:10C0380023FA02F34FEA4303CCE77FEA625307D1BE
:10C0480050EA01331EBF4FF0FE4040F440007047F5
:10C0580001F0004040F0FE4040F40000704700BF8F
:10C06800002100F004B80C4B5B58435004310B48D6
:10C078000B4B42189A42FFF4F6AF0A4A00F003B895
:10C08800002342F8043B084B9A42FFF4F9AFFCF74F
:10C0980099FE00F00DF87047C03401080000002038
:10C0A800E8010020E801002010210020FFF7FEBF72
:10C0B8002DE9804891B0F4F763F8BC4EBC4CB168E8
:10C0C800002311F0080F2370274600F0E88063680A
:10C0D8001B7A042B00F2E180DFE803F00303058AF2
:10C0E800B100237ADAE0627AB14B002A00F0D580F9
:10C0F80000225A7293F82020100700F1CE80D87AD7
:10C108009A7A00F0070542EA05225A621A7B02F081
:10C118003F056D0145EAD0009862587B800040EAEF
:10C1280092109A7B02F0010540EA8520D862D87BFC
:10C1380000F00F05ED0145EA52021A631A7C02F07D
:10C148007F052D0145EA10105863587C400040EAED
:10C15800D212987C00F0030542EA45229A63DA7C01
:10C1680002F01F05AD0145EA9000D863187DC000B4
:10C1780040EA5212987D1A645A7D00F0070542EA97
:10C1880005225A64DA7D02F03F056D0145EAD000C8
:10C198009864187E800040EA92105A7E02F00105E9
:10C1A80040EA8520D864987E00F00F05ED0145EA45
:10C1B80052021A65DA7E02F07F052D0145EA101059
:10C1C8005865187F400040EAD212587F00F00305F6
:10C1D80042EA45229A659A7F02F01F05AD0145EAB9
:10C1E8009000D865D87FC00040EA52121A6652E023
:10C1F80094F864206E4B002A4FD0002283F8642004
:10C2080093F86620012A48D193F88A20102A84BF1F
:10C21800102283F88A2094F88A00664A0023DDB247
:10C22800854202F1020236D212F8015C12F802ECE1
:10C2380045EA0E2E604D45F823E00133EFE794F808
:10C24800CC205B4B4AB3002283F8CC2093F8CD2056
:10C25800A82A22D193F8E030FBB907EB43029FEDFF
:10C26800577A92F8D00092F8D12002EB002207EE1C
:10C27800902AF8EEE77A524AC7EE877A9FED517A0C
:10C2880077EEC77AFCEEE77A17EE900A42F82300B9
:10C298000133082BE1D1012300E0002323704A0475
:10C2A80008D594F8043123B1414B002283F80421C6
:10C2B8000123237023783BB1CB0505D53C4BD3F83C
:10C2C80008311B681B6898473F4922780B6832B9C8
:10C2D800374AD2F80C219A1AD243D20F00E0012231
:10C2E80082B3F7F7B7FC94F81021314B002A00F01D
:10C2F800AC83D3F81421550740F1A783D3F818214C
:10C30800100706D4B3F81C2122F00802A3F81C2158
:10C318009BE3B3F81C1101F0080292B2002A40F026
:10C32800948341F00801A3F81C11D3F82411C3F831
:10C338002011B3F83011A3F82811C3F83421C3F839
:10C34800382182E3D4F83C21194D511C012AC4F844
:10C358003C1174D0022A00F05B82002A40F05D8212
:10C36800D5F81411490740F15882D5F84011591AE7
:10C378000029C0F25282C5F8403195F84431012BAA
:10C3880024D002D3022B39D047E2D5F85031984750
:10C39800D5F854319847012385F84431B5F84A2136
:10C3A800D5F840311344C5F8403136E2041A00206C
:10C3B800E80100205002002074020020CDCCCC40BF
:10C3C800CC0200200080BB43D8200020D5F858318B
:10C3D8009847D5F84C319847D5F84031B5F84821F9
:10C3E8001344C5F8403105F5B070D5F85C3105F552
:10C3F800B2719847022385F844310EE285F844214A
:10C40800D5F86C11D5F86801D5F86021D5F87051C8
:10C418002D784B1CAB4203D1012384F874310023DF
:10C4280007EB8101C4F86C31C1F8782107EB83016F
:10C438000244D1F87811521AC4F86821EDE1D5F810
:10C448001421500740F1E98195F87421002A00F081
:10C45800E481D5F83822C2EB030A46F2A7129245C6
:10C4680040F2DB81DFF8A493C5F83832B9F80080D0
:10C478009FEDD89ADFEDD88AB7EE008AB8F1000FA1
:10C488002DD0D5F87011D5F83C020A78D5F8681186
:10C49800DFEDD20A013A0823B1FBF2F190FBF3F287
:10C4A800801A0A1892FBF3F305EE903AB8EEE50A03
:10C4B800C5F83C2280EE090A01F02AFF08F1FF388E
:10C4C8000023A9F80080C5F84432C5F8483238EE90
:10C4D800400A20EE280ABDEEC00A85ED900AD4F87D
:10C4E8007081D4F8683198F80020DFEDBC0ABC4DA3
:10C4F800013AB3FBF2F306EE903AB8EE660A80EE24
:10C50800090A01F005FF38EE400A20EE280A01F07A
:10C5180017FED4F84032D8ED017AD4ED935AC01AF8
:10C5280006EE900AB8EEE60A78EE676AB8EEE57AA3
:10C5380020EE260AA7EE270A01F002FE0146A948C6
:10C5480003685A1EC62A05D8C91AC5F85012C5F874
:10C558004C3226E0D5F85022002BC2EB010202DC57
:10C56800C5F84C221DE0C3F5967107EE101ADFEDF1
:10C578009E7AB8EEC77A05EE903A87EE277A07EEEC
:10C58800902AB8EEE76AF7EE007A77EEC77AF8EE07
:10C59800E56A66EE277AE6EE877AFDEEE77AC5ED7C
:10C5A800937A924DD4ED976AD5ED005A94ED999A05
:10C5B8009FED8F6AD4F84C228949F8EE657AD4ED5C
:10C5C800985AF8EEE68AB8EEE57A27EE866AC8EE5B
:10C5D800878A0023C4F85432C4F85832C4F85C324D
:10C5E800C4F860322B60B9F8003094ED917AD8ED38
:10C5F800036A28EE899AF6EE005A29EE279A67EE22
:10C60800067A69EE255A37EE099AE5EE867A94EDB0
:10C61800926A84ED919A37EE866A07EE902AF8EED0
:10C62800E75A78EE667A65EEA77AE6EE267AC4EDE2
:10C63800927A002B40F0F18003689FED6E7A013BFF
:10C64800C62BD4F8683294BFC1F82421FDEEE77AEE
:10C65800C3EB020388BFC1ED497A07EE903A05EEB5
:10C6680090AAF8EEE77A40F2DC5367EE877AB8EEE4
:10C67800657A0A21C7EE877AC4F86822FDEEE77A60
:10C6880017EE900A9842A8BF1846A3F6B833984206
:10C69800B8BF1846F7F740F9D8ED027A06EE900AC7
:10C6A80038EE678AB8EEE60A20EE080AA9EE270AED
:10C6B80084ED910A01F044FD05218046F7F72CF935
:10C6C800B4F87432C4F86C0203F21F339BB240F220
:10C6D8003E62934294ED9C8A0AD8414BB3F8763275
:10C6E80003F21F339BB293428CBF0023012300E067
:10C6F8000023002B69D094F87832394D13BBD5F854
:10C708002431D5F820213C48D21AB2F5FA7FA8BFC7
:10C718004FF4FA728242A8BF10460A21F7F7FCF8D4
:10C72800D5F87C32DB788022584390FBF2F3B3F5DE
:10C73800967FA8BF4FF49673A2F5D6729342B8BFFE
:10C74800134601E02D4B1B68D4F87C22517AD57C26
:10C75800527F07EE902AC8EB030359432020F8EED6
:10C76800E77A38EE888A91FBF0F1D4F8340127EEA5
:10C77800888ADFED237A03FB0500224BB0F5C81F3A
:10C78800A8BF4FF4C81028EE278A9842B8BF1846A9
:10C798004FF40053C4F83401BDEEC88A90FBF3F09F
:10C7A800194BB1F5967FA8BF4FF496719942ACBF6B
:10C7B8004118C11818EE103A6FF09502962BA8BFD1
:10C7C80096239342B8BF1346CB1AC4F83831C4ED48
:10C7D8009C8A22E080E6C547D048874AB1DC423EC1
:10C7E800E80100204C0100200000C842E42000209D
:10C7F800BD378635002474490CFEFFFFEC2000206D
:10C808000000003B0000E7FFD4FEFFFFE02000200F
:10C81800B368990301D5FCF70DF8D4F83C31022B25
:10C8280003DDB64B0022C3F83C21B3681A0640F179
:10C838000C81D4F88032B3B994F88432013B042BCC
:10C8480000F20381DFE813F0160016001600EE0070
:10C85800C900AA4BD3F88002F6F770FDFDF750F82F
:10C8680008B1FAF7F5FCD7F88002F6F76CFD002856
:10C87800EFD1E1E7D4F8A422A04D92F80080B8F1F6
:10C88800000F03D0B8F1010F0ED0DEE0012B00F24B
:10C89800DC8095F885229A4BD5F8800203EB0213C9
:10C8A8005968F6F746FD4FE0D5F88002F6F73CFDEB
:10C8B800002800F0CA8095F88432022B34D0032B6C
:10C8C8003ED0012B40F0C1808E4BD5F89C221B68CE
:10C8D8009A1AC72A40F2B980D5F89812042921D8A3
:10C8E800874AD5F88082C5F89C3202EB0111D8F846
:10C8F800083049688B4203D04046F6F71AFDA4E099
:10C9080095F8853202EB0312956815F8011B19B1E9
:10C918004046F6F71DFDF8E7D4F898320133C4F81D
:10C92800983292E002208EE095F88522744BD5F873
:10C93800800203EB02135968F6F7FBFC032082E040
:10C94800D5F8A4329B780BB904207CE095F8A03286
:10C958000BB985F8A08294F8A032684D012B17D145
:10C96800D5F89832B22B0DD8654AD5F88002134411
:10C9780093F85010F6F7ECFCD5F898320133C5F867
:10C98800983205E00023C5F89832022385F8A032D2
:10C9980094F8A032594D022B1AD1D5F898320F2BA2
:10C9A80013D8D5F8A42256495278D5F8800202EB5C
:10C9B80002120A44134493F80411F6F7C9FCD5F897
:10C9C80098320133C5F8983202E0032385F8A03283
:10C9D80094F8A032022B38D9B6E7D4F88C22474B0A
:10C9E8000132C4F88C22D4F8A422D2785AB193F830
:10C9F80085220132D2B20521B2FBF1F101EB8101AE
:10CA0800521A83F885223F4B1B68C4F890320023E2
:10CA180084F8A83294F8A93223F0020384F8A932E2
:10CA2800012010E0374BD4F890221968334B8A1A4A
:10CA380040F6C4118A4208D9D3F8142122F0200202
:10CA4800C3F814210520FDF77BFCF6F729FC2E49D5
:10CA5800B38908602BB1D4F8AC22821A002AFFF6F9
:10CA68002CABDFF89880D4F8B052DFF8A0B01844A7
:10CA78007379C4F8AC02049308F53170D4F8B8326D
:10CA8800984708F53170014694F8CA22F8F76EFB0A
:10CA9800BBF80030002B00F0A380D8F8CC321B780C
:10CAA8004FF0000A08EE103A08F53478D1461748D6
:10CAB800174A0388B3F57A7F04D1002142F80A1097
:10CAC800C8F81010134852F80A1030F909E07144F8
:10CAD80042F80A10D8F8102005EE90EA0132012A2F
:10CAE800F8EEE57AC8F8102016D10022C8ED017AD0
:10CAF800C8ED007AC8F8082028E000BFE801002047
:10CB08000C000108001A0020D8200020E82000208E
:10CB1800F4040020AC04002098ED006A05EE902A89
:10CB280077EEC66AB8EEE57A86EE877A36EE077A49
:10CB380037EEC76AD8ED027A88ED017AE6EE867A92
:10CB480088ED007AC8ED037AC8ED027ACF4A002151
:10CB5800012B20F8091029F8021034D1D8F8101048
:10CB6800012909DD013900EE101AD8ED037AB8EE73
:10CB7800C00A87EE800A01E09FEDC50A039202937E
:10CB880001F06AFD18EE100A039A029B48B1F8EE0C
:10CB9800C87AB4EEE70AF1EE10FA02DD4FF47A73C0
:10CBA8001CE0BC495AF801104FF47A7001F5FA718B
:10CBB80091FBF0F122F809100A200F2101220293BB
:10CBC800FDF738F9029B09F10209B9F1060F0AF1DC
:10CBD800040A08F114087FF46AAF013BABF800308F
:10CBE8000023DFF8B4A20AF531780AF5467233F863
:10CBF80008109A5A8A1A23F808200233062BF0D113
:10CC0800DAF8143113F0020300F0D182DAF8243391
:10CC18000AF54B7098470AF54B7001469AF832238B
:10CC2800F8F7A4FABAF834330AF54B79002B4AD04E
:10CC38000022DAF838E31346B7F83413DFF868C28D
:10CC48009548B1F5C87F04BF00214CF8031000F5E2
:10CC58004B7A5CF8031032F90AB059444CF80310C7
:10CC6800043300210C2B22F80A102EF8021002F1CE
:10CC78000202E1D1B0F83433012B1FD1D0F83C3394
:10CC88004FF4C872C83393FBF2F3AEF80030D0F813
:10CC98004033C83393FBF2F3AEF80230D0F8443394
:10CCA800C83393FBF2F27D4B1B88D21AAEF80420EE
:10CCB800A5F85410A5F85610FAF752F9B4F8343319
:10CCC800013BA4F83433B3685B0740F18580B4F8BE
:10CCD8004823714B322A13D1D3F838231188A3F88B
:10CCE8004A1351889288A3F84E23B5F85420A3F824
:10CCF8005023B5F85620A3F84C13A3F8522301E0AB
:10CD0800002A44D00020D4F838E30246B7F8483364
:10CD1800DFF898C1322B04BF00234CF802305E4B79
:10CD28005CF8021003F54B7A30F90AB059444CF814
:10CD38000210043200210C2A20F80A102EF80010E4
:10CD480000F10200E2D1B3F84823012A1AD183F88E
:10CD58006123052283F86223B3F84A2383F860131A
:10CD6800AEF80020B3F84C23AEF80220B3F84E23F7
:10CD7800AEF80420B3F85023B3F85233A5F8542082
:10CD8800A5F85630B4F84833013BA4F8483394F872
:10CD98006323414B02B3D3F85413D3F838034FF04D
:10CDA800320E002291FBFEF183F863230180D3F851
:10CDB800581391FBFEF14180D3F85C3393FBFEFEE0
:10CDC800364B1B88C3EB0E0EA0F804E0A5F85420E0
:10CDD800A5F85620FAF7C4F8D4F83833B4F82C1369
:10CDE8001A888A1AA4F82C235A88B4F82E138A1A97
:10CDF800A4F82E239B88B4F83023D31AA4F8303330
:10CE0800F6F74EFAD4F8643394EDDA6AD4F86C5332
:10CE1800234A95F800C0C4F86403C3EB000B05EE81
:10CE280090BAB8EE659A002329EE066A194638F9D1
:10CE380003E007EE90EAF8EEE77A0DF11C0A67EED8
:10CE4800867A0AEB4300C0ED007ABCF1000F2FD0C0
:10CE580005EE90CAB8EEE57AF7EE006A86EE877AB4
:10CE680039F9030007EE900AF8EEE77A0D4867EE05
:10CE7800877A36EEC77AD2ED006AE6EE877AC2ED97
:10CE8800007AFDEEE77A17EE90EA16E0000500203A
:10CE980000000000F4040020E80100200000002049
:10CEA8005805002064050020240500203C050020CA
:10CEB800D048A0F1500E33F80EE023F800E0CD483A
:10CEC80033F800E00233062B1EFB0E1102F10402B8
:10CED8008246ACD1DFF83083B8F800304FF06409EF
:10CEE80009FB01F15B4391FBF3F9A9F1490908300A
:10CEF80007A91FFA89F9F6F7F7FAB9F13B0F95ED8B
:10CF0800017A12D9B4F99013D4EDE30ABA4B94F824
:10CF1800A92207EE901AF8EEE77AF4EEE70AF1EEA6
:10CF280010FA1DDD42F008021CE0F7EE007A37EE39
:10CF3800276A0AF1080287EE866A00233AF903E0B5
:10CF48000233062B07EE90EAD2ED006AF8EEE77A94
:10CF5800E6EE877A67EE866AE2EC016AEED1D1E7FF
:10CF680022F0080294EDE20A83F8A92201F0CEF932
:10CF780094EDE37AD4EDE27A84EDE50AF0EE408AA6
:10CF880027EE070A94EDE18ADFED9C9AA7EEA70A3F
:10CF980001F062FBB1EE488AF0EE400AB0EE480AB2
:10CFA80001F0B4F9B0EE408A84EDE60A28EEA90A49
:10CFB80001F0C6F828EE290AA4F8740201F0C0F8B6
:10CFC800D4F81431A4F8760218071CD58C4807A9A0
:10CFD800F6F78AFA95ED027A894BF7EE007A37EE82
:10CFE800276A03F10C0287EE866AD3ED006ADFED4B
:10CFF800857AE6EE877A67EE866AE3EC016A934201
:10D00800F3D17F482CE0804B0293181D07A9F6F74F
:10D018006BFA98ED020A98ED017AD8ED037A20EEC2
:10D02800000AA7EE070AA7EEA70A01F015FBB5EE5E
:10D03800400AF1EE10FA029B11D093ED017A87EEC7
:10D04800007A83ED017A93ED027A87EE007A83ED18
:10D05800027A93ED037AC7EE007AC3ED037A6B4840
:10D06800F6F7ACFAA4F8A803B4F9A803DFED687AD8
:10D078009FED687AB4F97C13B4F97E23B4F9803350
:10D08800DFF8749129EE279A07EE900AF8EEE77A0E
:10D09800F1EE688A67EEC77AB1EE488ACDED0C7A70
:10D0A80007EE901AF8EEE77A0DA8CDED0D7A07EEA7
:10D0B800902AF8EEE77A0AA9CDED0E7A07EE903AB3
:10D0C800F8EEE77ACDED0A8ACDED0F7A8DED0B8A71
:10D0D800F6F70AFA6B78DDED0F7A012B1DD14E4B6E
:10D0E8001B7859070FD4D9F8AC33402293FBF2F2DE
:10D0F8009A1A07EE102AB8EEC77A37EE277ABDEEED
:10D10800C77A89EDEB7AD4F8AC33402293FBF2F37B
:10D1180005EE903AB8EEE57A05E0B8F8008007EE3B
:10D12800108AB8EEC77A77EEC77A94EDEC8ACDED1F
:10D138000F7AD4EDED7A9DED0D0AD4F8548279EE8C
:10D14800277A89EE279ADDED0F7A77EEC87AA9EE6D
:10D15800278A84EDEC8A00F0F3FFD4F8B8532978D5
:10D16800F6F7DAFB9DED0E0A4044C4F85402D4F8F1
:10D17800588200F0E5FF2978F6F7CEFBB0EE480AB2
:10D188004044C4F85802D4F85C8200F0D9FF6978AA
:10D19800F6F7C2FB214B1A685A441A60D4F8603279
:10D1A80040440133C4F85C02C4F8603205E0AAF8D0
:10D1B8002C33AAF82E33AAF830330498B4F8C422D2
:10D1C800A4F8BC230128B4F8C6220B4BA4F8BE234C
:10D1D80026D1B3F8C203B3F9C812022210FB021217
:10D1E800032192FBF1F292B2A3F8C023A3F8C22361
:10D1F8001AE000BF64050020E80100204C3D0F4400
:10D208008405002000000000000000200400002029
:10D21800BD37863535FA8E3CF0200020E42000200A
:10D22800B3F8C822A3F8C023F6F73AF8D4F8C833FD
:10D23800C549C4F8C803C31AA4F8C4330860F4F78E
:10D24800C7F8D4F81481C14D012318F0140F84F8DD
:10D2580010317CD0B5F81C2102F40272002A76D075
:10D2680095F8A92202F0100202F0FF0052B1B5F8B9
:10D278002C2196F92711D5F8383101FB0323A5F89D
:10D288002C3164E0D5F8CC23D178927879B3B5F80D
:10D2980030C1B5F928110FFA8CFEC1EB0E09B9F1AE
:10D2A800000FB8BFC9F1000991450EDD8E45C8BF12
:10D2B80052421FFA8CFCC8BF92B26244C5F83401CE
:10D2C80085F8D033A4F8302141E095F8D0332BB15C
:10D2D800D5F82431C5F8203185F8D003D4F8383191
:10D2E800D4F8D423194413885288994228E0B5F910
:10D2F8002801B5F930E1C0EB0E0E8EEAEE7CACEBFE
:10D30800EE7C944509DD0221914A85F878329EFB2E
:10D31800F1F1116085F8D0330AE095F8D0333BB1CC
:10D32800D5F82431C5F8203185F8781285F8D0135E
:10D33800D4F8D413D4F838210B88498802449A4287
:10D3480003DB8A42B4BF13460B46A4F83031D4F845
:10D35800B0927E4D99F864B1BBF1000F41D0B5F899
:10D368001C319A073DD095EDE20AD5EDE17A95EDAD
:10D37800E38AB5F830A120EE000AA7EEA70AA8EEC6
:10D38800080A01F069F988EE000ADFED727AB4EE56
:10D39800E70AF1EE10FA20D900F05AFFD5EDF67A37
:10D3A80020EE270A00F0CCFEB0F5617FA8BF4FF44D
:10D3B800617005EE900ADFED687AB8EEE50A80EE56
:10D3C800270A00F007FF06EE90BAF8EEE67A27EE95
:10D3D800800A00F0B5FE80B200E000205044A4F8B6
:10D3E800300118F0200F00F08780B4F81C31574D39
:10D3F80003F03003002B7FD095F8A932DB077BD5EB
:10D40800B5F9A803DFED557ADFF8588108EE100A60
:10D41800B8EEC88A28EE278AB0EE480A00F0DAFE8D
:10D42800F0EE408AB0EE480A00F04EFED5F8DC3344
:10D43800B5F9E60393F803A0B0EE409AB2EE048A79
:10D44800BAF1000F36D0B5F8E2331FFA83FB1BB2EE
:10D45800C01AF6F74FFBCAF10005A84203DB504596
:10D46800A8BF504600E02846B4F8E0338344B4F936
:10D47800E4039AB21BB21FFA8BFBC01A0392A4F8FA
:10D48800E2B3F6F737FBA842039A03DB5045B4BF73
:10D49800054655461544ADB2A4F8E0530FFA8BFB88
:10D4A8002DB205EE90BA07EE905AB8EEE57AF8EE8E
:10D4B800E76A09E0B5F9E45305EE900A06EE905ADA
:10D4C800B8EEE57AF8EEE66A68EEE67AE7EE097A0B
:10D4D80026EE899AC7EE887AA7EE289AFDEEE77AB3
:10D4E80089EE089A17EE903ABDEEC99AA8F800306E
:10D4F80019EE103AA8F80230194BD4F8E813D3F80B
:10D5080000C0B6F8F620114D09F1040009F15403E2
:10D51800DFF85490E04799F80010032926D9B5F9A7
:10D528002E01B5F9F0230028B8BF40426FF063031D
:10D538001B1A9A4204DB00F164039342A8BF134606
:10D54800A4F8F03332E000BFD8200020E801002022
:10D55800EC2000208FC2753CEFB6B04435FA8E3C03
:10D5680048010020DC200020BC20002001291DD813
:10D5780094F8F233C04D013B142B00F20282DFE82D
:10D5880013F08900000200025B009900000200020B
:10D59800470100020002000200020002BC00000273
:10D5A8000002000200020002B501D301B4F8300104
:10D5B800B4F8EE53B4F8ECE3D4F8F4C3B4F9F08358
:10D5C800AE4B00228A4203F11003D1D29CF900A08D
:10D5D80013ED027ACAF1000A08FB0AFA05EE90AACE
:10D5E8000FFA8EFA06EE10AA0FFA80FAF8EEE56A3C
:10D5F80005EE90AA0FFA85FA07EE90AAF8EEE77AF8
:10D60800F8EEE55A67EE877A13ED047ADFF874A22C
:10D61800E5EE877AB8EEC66A13ED037AE6EE077A86
:10D6280013ED017AE6EE877AFDEEE77A17EE90BA07
:10D638002AF812B00132C5E702210420F5F72AFFC3
:10D64800B4F8F0A300FB0AF01FFA80FB01210420C4
:10D65800F5F720FFB4F8EE8300FB08B01FFA80FB53
:10D668000420F5F725FF5844288102210520F5F705
:10D6780011FF00FB0AF01FFA80FA01210520F5F7D7
:10D6880009FF00FB08A01FFA80FA0520F5F710FF34
:10D6980050440DE005200121F5F7FCFEB4F8F083B5
:10D6A80000FB08F01FFA80F80520F5F701FF404459
:10D6B800688166E1D4F8B8A4B4F876829AF806B01E
:10D6C8000020F5F7F5FE4FFA8BFB1BFB08FB4FF02C
:10D6D80032089BFBF8FB584428809AF80EB0B4F83F
:10D6E80074A20120F5F7E4FE4FFA8BFB1BFB0AFA44
:10D6F8009AFBF8F84044688043E1614B1B7858076F
:10D7080003D4D4F8BC349B880BE0D4F8BC14B4F927
:10D7180030210B8849889A4203DB9142B4BF0B46FB
:10D728001346EB81574BEA891A80D4F8C03493F832
:10D738000080B8F1000F2ED00220F5F7B9FE524B49
:10D74800D3F8B834B3F91020598A904203DB0AB2EF
:10D758009042B8BF0246D4F8C4144B484989C2EB7A
:10D76800010EB4F8C8240FFA8EFE0FFA82FCF445B5
:10D7780001DA904402E003DDC8EB0208A0F8C8848F
:10D78800B4F8C82493F9163013FB02F3642293FB10
:10D79800F2F31944A980B4F81C213B4BD10510D5EC
:10D7A800B3F82A21EA802A81B3F82E21B3F82C3164
:10D7B8006A81AB81DFF8C0A0D4F8B8344FF0030811
:10D7C80009E0B3F8EC23EA802A81B3F8F0236A81F0
:10D7D800B3F8EE33EDE703EBC801BAF8062091F988
:10D7E80006B01BFB02FB64229BFBF2FBAAF806B007
:10D7F80040460293F5F75CFE08F101085844B8F179
:10D80800070FAAF80600029B0AF1020AE3D1B8E062
:10D818001B4B1B785A0703D4D4F8BC349B880BE005
:10D82800D4F8BC14B4F930210B8849889A4203DB38
:10D838009142B4BF0B461346EB81124BEA891A801A
:10D84800B4F81C31DFF83080DFF83CA0DB054FF07E
:10D8580003004FF0010119D5F5F71CFEBAF82CB1F9
:10D8680000FB0BF083B2022103200293F5F712FEAE
:10D87800BAF82AA118E000BF38010020E00500200E
:10D88800F0200020BE200020E8010020F5F702FE6D
:10D89800BAF8EEB300FB0BF083B202210320029327
:10D8A800F5F7F8FDBAF8ECA3029B00FB0A30A8F8DC
:10D8B800060001210420F5F7EDFD00FB0BF0022125
:10D8C8001FFA80FB0420F5F7E5FD00FB0AB0A8F875
:10D8D80008000320F5F7ECFDEB881844E8800420E5
:10D8E800F5F7E6FD2B89184428814AE00121042038
:10D8F800F5F7D0FDB4F8EE8300FB08F01FFA80F8C6
:10D908000420A5F80880F5F7D3FD404428810121BB
:10D918000520F5F7BFFDB4F8EC8300FB08F01FFA0B
:10D9280080F8A5F80A80BFE6B4F8F0B34FF0030812
:10D9380040460221F5F7AEFD00FB0BF01FFA80FA16
:10D9480001214046F5F7A6FDC8F1060323F00103BF
:10D958003B44B3F8EC3300FB03A01FFA80FA25F828
:10D9680018A04046F5F7A4FD504425F8180008F122
:10D978000108B8F1070FDBD1AC4BB3F83021AC4B41
:10D988001A80B368980637D50020F5F791FD2880EE
:10D9980082460120F5F78CFDD4F81821DFF89C8227
:10D9A80068801106A14B27D5D3F8CC24127812F041
:10D9B800020FB3F8742223D0D3F8B8E4B3F976325F
:10D9C8009EF90E109EF906E011FB02F2CEF1000E50
:10D9D800322103FB0EF392FBF1F26FF0310E92B29B
:10D9E80093FBFEFE964493FBF1F1F2440A44A8F837
:10D9F80000A01044A8F80200D4F8B814002319E0D5
:10DA0800D3F8B814B3F8763291F906E01EFB03FE9A
:10DA180032239EFBF3FEF244A8F800A091F90E1001
:10DA280011FB02F292FBF3F31844E3E7EA520233E4
:10DA3800102B0ED0E85E31F9232001EB830E9042C3
:10DA4800BEF802E0F2DB0FFA8EF28242A8BF02466D
:10DA5800ECE7D4F8CC341B785A0705D4744A99F803
:10DA680000001188012323E0704B93F8D0A4AAF199
:10DA7800040A5FFA8AFA5FFA8AFB4FF00008042367
:10DA880048FA8BF2002A0DDB5A1C07EB43030AEB1A
:10DA98000800D2B2B3F8D2140392C0B2F6F7AEF8C7
:10DAA800039A134608F10108B8F1040FE8D1D5E745
:10DAB800834208D232F9137009B28F42A8BF39469F
:10DAC80089B20133F4E7B368B4F9D8A4CDF804A057
:10DAD80003F4805603F0100A564BD4F8BC241B7884
:10DAE800D4F8C474D4F8F8E4059603F00403DBB260
:10DAF80004934FEA400900234B454ED0B2F8028008
:10DB080008B240454A4806DD30F803C0C1EB0808B2
:10DB1800C44420F803C0059EC6B1B7F80AC0019EE8
:10DB280030F903806645CBBFBEF802009088B2F892
:10DB380002B0BEF800B0DFF8F8C0804503DBD84576
:10DB4800B4BF404658462CF803001CE030F903C027
:10DB58001088B2F80280844503DBC445B4BF604630
:10DB68004046DFF8CC80019E23F80800B889864239
:10DB780003EB080C07DABAF1000F01D1108800E0B6
:10DB88009088ACF80000049828B92B4833F800C0F6
:10DB9800274823F800C00233AEE7D4F81435002B29
:10DBA80054D0224B93F8F233013B142B48D8DFE8CA
:10DBB80003F00B4747264B47471F47474747472D23
:10DBC8004747474747262D00D4F8F4335B782BB1F5
:10DBD8001A4B59890020F6F711F837E0154B1B78D6
:10DBE80003F0040303F0FF00002BF1D10146F2E734
:10DBF8000020E988F6F702F801202989EBE70020E0
:10DC08002989F5F7FBFF01206989E4E70020E98805
:10DC1800F5F7F4FF01202989F5F7F0FF022069895B
:10DC2800F5F7ECFF0320A989D5E700BFE80100203C
:10DC3800BE200020F0200020E4060020380100204B
:10DC4800044B9B689B0601D5F5F7E4FFF8F7F2F85B
:10DC5800FEF733BA041A002010B50023934203D00C
:10DC6800CC5CC4540133F9E710BD02440346934227
:10DC780002D003F8011BFAE7704700000D4B70B59E
:10DC88001D680022845C2B195B7803F00303012BC9
:10DC98008B5C05EB030608BF2034767806F0030694
:10DCA800012E08BF2033E41A02D10132002BE9D13A
:10DCB800204670BD7C01002010B504462246013480
:10DCC8001378002BFAD1CC5CD4540133002CFAD150
:10DCD80010BDC9B2024610F8013B1BB18B42F9D105
:10DCE800104670470029FBD018467047034613F8C2
:10DCF800012B002AFBD1181A013870470F4BF0B5D9
:10DD08001E680023934216D0C55C7419647804F029
:10DD18000304012CCC5C06EB040708BF20357F7890
:10DD280007F00307012F08BF20342D1B04D101334E
:10DD3800002CE7D100E000252846F0BD7C0100203A
:10DD480010B5034632B111F8014B03F8014B013A03
:10DD5800002CF7D11A44934203D0002103F8011B89
:10DD6800F9E710BD30B503780BB1044604E00B7831
:10DD7800002B18BF002030BD22460134107838B17E
:10DD88000023C85C28B1D55C8542F5D10133F8E79A
:10DD980030BD104630BD00210A2200F001B92DE93E
:10DDA800F04E82468B461F46144612B90020BDE845
:10DDB800F08E002BFAD00026A642F7D2A5196D08DE
:10DDC80007FB05B950464946089B9847002802DBDF
:10DDD80003D06E1C25462C46EEE74846BDE8F08E7B
:10DDE800174B2DE9F0411D68AC6D06460F46FCB98E
:10DDF800502000F0E3F8A8658460AB6D04604460CF
:10DE08001C61DC60AB6D9C615C61AB6DDC629C622B
:10DE1800AB6D5C631C63AB6DDC639C63AB6D5C6476
:10DE28001C64AB6DDC649C64AB6D1C77AB6D5C6291
:10DE380030463946AA6D0123BDE8F04100F002B82A
:10DE4800E0010020F0B508B9106828B304460F4671
:10DE580014F8015B17F8016B3EB1B542FAD10BB16A
:10DE68002046F3E714600370F0BD4DB915602846ED
:10DE7800F0BD17F8016BAE4207D0002EF9D11C4651
:10DE880023460F4613F8015BF3E715B10021217013
:10DE980000E02B461360F0BDF0BD000084463F480B
:10DEA8002DE9F04FD0F800800E46344614F8015B97
:10DEB80008EB0500407800F0080000F0FF0708B103
:10DEC8002646F2E72D2D03D1B41C7578012703E00F
:10DED8002B2D04BF7578B41C33F010000DD1302DF4
:10DEE80008D1207800F0DF00582851D16578102338
:10DEF800023402E0002B08BF0A23002F0CBF6FF08A
:10DF0800004A4FF0004ABAFBF3F9002603FB19AAAE
:10DF1800304608EB050B9BF801B01BF0040F01D04D
:10DF2800303D0BE01BF0030B1BD0BBF1010F14BFFE
:10DF38004FF0570B4FF0370BCBEB05059D4210DA2E
:10DF4800B6F1FF3F0AD0484506D801D1554503DC54
:10DF580003FB0050012601E04FF0FF3614F8015B87
:10DF6800D7E7731C0CD1002F4FF022030CBF6FF0C2
:10DF780000404FF00040CCF800302AB9BDE8F08FDF
:10DF880007B1404242B106B1611E1160BDE8F08F91
:10DF9800002B08BF0823B0E7BDE8F08F7C01002004
:10DFA80030B51346044A05460C46106829462246F1
:10DFB800BDE83040FFF772BFE0010020024B014688
:10DFC800186800F003B800BFE001002070B5CD1C50
:10DFD80025F0030508350C2D38BF0C25002D064605
:10DFE8003FDB8D423DD3214B1C6818462146A1B129
:10DFF8000B685B1B0ED40B2B03D90B60CC18CD50D0
:10E008001FE08C4202D1626802601AE04B686360CC
:10E018000C4616E00C464968E9E7154C23681BB91D
:10E02800304600F027F820602946304600F022F8F4
:10E03800431C014615D0C41C24F0030484420AD1B1
:10E04800256004F10B00231D20F00700C31A0BD034
:10E058005A42E25070BD3046611A00F00BF80130A8
:10E06800EED10C233360002070BD00BF04210020D6
:10E078000021002038B5064C0023054608462360D9
:10E0880000F008F8431C02D1236803B12B6038BDA7
:10E098000C210020094A136863B118446946884274
:10E0A80002D8106018467047054B0C221A604FF0D2
:10E0B800FF307047034B1360EFE700BF08210020D3
:10E0C8000C2100201021002000B510EE103A1A4A49
:10E0D80023F00043934283B019DDB3F1FF4F04DB13
:10E0E80030EE400A03B05DF804FB684600F0CCFF50
:10E0F80000F0030001289DED000ADDED010A12D0B1
:10E1080002280BD0A0B1012001F0BEFCEAE7DFED48
:10E118000B0A01F051F903B05DF804FB01F04CF96A
:10E12800B1EE400ADEE701F0AFFCB1EE400AD9E7F4
:10E1380001F042F9D6E700BFD80F493F00000000C0
:10E1480010B410EE100AC0F3C751A1F17F031E2BC3
:10E1580083B028DC5C1C21DB162B4FEAD0740BDD66
:10E16800C0F3160040F400009639884004B14042DC
:10E1780003B05DF8044B7047154B03EB8403D3EDF4
:10E18800007A37EE807A8DED017A9DED017A37EECF
:10E19800677A17EE103A23F0004262B9002003B004
:10E1A8005DF8044B7047FDEEC07A17EE900A03B095
:10E1B8005DF8044B7047C3F31600C3F3C75340F42C
:10E1C8000000C3F19603D840002CD1D0CFE700BFA0
:10E1D8008030010800B510EE103A1B4A23F00043C6
:10E1E800934283B01ADDB3F1FF4F04DB30EE400AEF
:10E1F80003B05DF804FB684600F046FF00F003003A
:10E2080001289DED000ADDED010A15D002280DD088
:10E21800A8B101F0D1F8B1EE400AE9E7DFED0B0A49
:10E22800002001F031FC03B05DF804FB012001F08F
:10E238002BFCB1EE400ADBE701F0BEF8D8E701207D
:10E2480001F022FCD4E700BFD80F493F00000000CE
:10E2580010B52DED028B2A4C8AB0B0EE408A00F042
:10E2680057FA94F900300133F0EE408A04D0B0EE4A
:10E27800480A01F027FE28B9B0EE680A0AB0BDECDA
:10E28800028B10BDB0EE480A01F0BAFDF7EE007A35
:10E29800B4EEE70AF1EE10FAEEDD0123194A009315
:10E2A80018EE100A002301920893FDF79BFB024623
:10E2B8000B461548CDE90423CDE9022301F030FCD3
:10E2C80094F90030022B8DED060B0FD0684601F053
:10E2D80023FC58B1089B73B9DDE90601FDF770FE10
:10E2E80000EE100A0AB0BDEC028B10BD01F084FEEE
:10E2F80021230360EEE701F07FFE089B0360EBE754
:10E30800E4010020883001089430010800F026BBA1
:10E3180070B52DED048BA84E8AB0B0EE409AB0EEE1
:10E32800608A00F0CDFB96F900300133F0EE408AA8
:10E3380004D0B0EE480A01F0C5FD28B9B0EE680A6D
:10E348000AB0BDEC048B70BDB0EE490A01F0BAFD0D
:10E35800002835D1B5EE408AF1EE10FAEED1974B90
:10E368000890012219EE100A8DE80C00FDF73AFB1F
:10E37800CDE9020118EE100AFDF734FB904B96F92F
:10E3880000400022CDE90623631CCDE904010DD02D
:10E39800022C0BD0684601F0BFFB002800F0A480D7
:10E3A800089B1BB101F028FE089B0360DDE906010C
:10E3B800FDF706FE00EE100A0AB0BDEC048B70BD36
:10E3C800B5EE409AF1EE10FA23D1B5EE408AF1EE9F
:10E3D80010FA5CD10123794A009319EE100A002340
:10E3E80001920893FDF7FEFACDE9020118EE100A32
:10E3F800FDF7F8FA96F9004000220023CDE9040160
:10E40800CDE90623002CC5D06D4B0022CDE90623AB
:10E41800CCE7B0EE680A01F0FBFC0446002868D09F
:10E42800F5EE408AF1EE10FA88D1B0EE490A01F013
:10E43800EFFC002882D0B0EE480A01F0E9FC002881
:10E448003FF47CAF04235D4A009319EE100A0023C1
:10E4580001920893FDF7C6FACDE9020118EE100AF9
:10E46800FDF7C0FA96F9004000220023022CCDE9FE
:10E478000401CDE9062300F08E80684601F04CFBCC
:10E48800002800F08880089B002B8FD08AE7B0EE28
:10E49800480A01F0BDFC00283FF450AFB5EEC08A31
:10E4A800F1EE10FA7FF54AAF0123444A009319EEC2
:10E4B800100A002301920893FDF794FACDE90201AE
:10E4C80018EE100AFDF78EFA3478CDE9040100221F
:10E4D800002C34D03B4B022CCDE9062332D101F07D
:10E4E8008BFD21230360CEE701F086FD2123036025
:10E4F80056E7B0EE490A01F08BFC002890D0B0EE48
:10E50800480A01F085FC00288AD0B0EE680A01F0BC
:10E51800D9FCE8B9294B0890012219EE100A8DE8B8
:10E528000C00FDF75FFACDE9020118EE100AFDF7BD
:10E5380059FA3478CDE90401002C31D100220023A6
:10E54800CDE90623684601F0E7FA00289BD1C6E723
:10E558001A4B0894032219EE100A8DE80C00FDF7F7
:10E5680041FACDE9020118EE100AFDF73BFA96F9D7
:10E578000030CDE904014BBB134BB5EEC09A4FF008
:10E588006042F1EE10FACDE9062343D496F9003043
:10E59800022B7FF472AF01F02FFD2223036072E794
:10E5A8000020002102460B46FDF79AFB022CCDE91C
:10E5B800060194D0C6E700BFE401002090300108AE
:10E5C8000000F03F0000F0FFFFFFEF471F4BB5EEE4
:10E5D800C09A0022F1EE10FACDE90623D6D5F6EE60
:10E5E800007A68EE277A17EE900AFDF7FBF90446E1
:10E5F8000D4645EC104B01F09BFA2046294653EC9A
:10E60800102BFDF7ABFC0028C0D1114B0022CDE93F
:10E618000623BBE7F6EE007A68EE277A17EE900A33
:10E62800FDF7E0F904460D4645EC104B01F080FA81
:10E638002046294653EC102BFDF790FC0028A5D165
:10E64800044B4FF06042CDE906239FE70000F07FBE
:10E658000000F0FFFFFFEFC710B52DED028B2A4C2D
:10E668008AB0B0EE408A00F055FE94F900300133CC
:10E67800F0EE408A09D0B0EE480A01F023FC20B140
:10E68800B5EEC08AF1EE10FA05D4B0EE680A0AB009
:10E69800BDEC028B10BD01231C4A009318EE100A32
:10E6A800002301920893FDF79DF92478CDE9040130
:10E6B800CDE902019CB900220023CDE90623684672
:10E6C80001F02AFAA8B1089BC3B9DDE90601FDF7F4
:10E6D80077FC00EE100A0AB0BDEC028B10BD0020DA
:10E6E800002102460B46FDF7FBFA022CCDE9060194
:10E6F800E5D101F081FC21230360E4E701F07CFC13
:10E70800089B0360E1E700BFE4010020983001089E
:10E7180008B510EE102A22F00043B3F17E5F2DED0C
:10E72800028B16D00CDCB3F17C5F1FDAB3F10C5FFF
:10E7380070DCBDEC028BDFED787AB0EE670A08BDBD
:10E7480030EE400AC0EE007ABDEC028BB0EE670AEC
:10E7580008BDBDEC028B9FED710ADFED717A002ACE
:10E76800D8BFF0EE407AB0EE670A08BD002AC0F2C2
:10E778008E80F7EE008A38EEC00AF6EE007A20EEB8
:10E78800278AB0EE480A00F0C5FD9FED667ADFEDF6
:10E79800663ADFED664A9FED663A9FED664ADFED21
:10E7A800665A9FED665ADFED667A9FED666ADFED81
:10E7B800666AE8EE073AA8EE034AE3EE884AA4EE52
:10E7C800085AE4EE885A10EE103AE5EE887A23F4F7
:10E7D8007F6323F00F03A5EE086A07EE103AE7EE11
:10E7E800886AE6EE088AB0EE486AA7EE476A26EE1F
:10E7F800888A70EE077AC8EE288AC6EE277AE8EE8D
:10E80800807ABDEC028B77EE277A77EEA77AB0EEA6
:10E81800670A08BD20EE007ADFED421ADFED422AD2
:10E82800DFED423A9FED422A9FED423A9FED426A60
:10E838009FED424ADFED424A9FED425ADFED425AD0
:10E84800DFED426ADFED427AE7EE212ABDEC028B6A
:10E85800E2EE873AA7EE023AA3EE876AA3EE074AEA
:10E86800E6EE074AA4EE075AE4EE875AB7EE006AC6
:10E87800A5EE076A25EE877A87EE066AE0EE466A15
:10E8880030EE660A77EEC07AB0EE670A08BDB7EEDA
:10E89800003A30EE030AF6EE007A60EE277A9FED32
:10E8A800212ADFED213ADFED214ADFED212A9FED14
:10E8B800214ADFED215A9FED215ADFED216A9FEDB4
:10E8C800216A9FED217AE7EE823AA7EEA24AE3EEAB
:10E8D800A74AA4EE275AE4EEA75AA5EE276AE5EE62
:10E8E800A76AB0EE438AA6EEA77AA6EE278A67EE55
:10E8F800278AB0EE670A00F00DFD88EE888A9FED42
:10E90800157ADFED157AA8EE007AF0EE006A37EE98
:10E91800000AE0EE667A17E7DB0FC93FDB0F4940D4
:10E928000000000008EF1138047F4F3A461124BD5B
:10E938002EC69D3D613330BFA80A4E3E2D5701407B
:10E9480090B0A6BE39D119C0ABAA2A3E6821A2331D
:10E95800DA0FC93F6821A2B3DA0F494010EE902AB6
:10E9680022F00041B1F1FF4F38B5F0EE407A18DCE3
:10E9780010EE104A24F00040B0F1FF4F11DCB2F164
:10E988007E5F46D0951705F0020545EAD47568B94B
:10E99800022D3BD09FED3F0A032D18BFB0EE670A4A
:10E9A80038BD07EE102A37EE270A38BD11B3B1F18A
:10E9B800FF4F32D0B0F1FF4F1CD0411AC9153C2986
:10E9C80021DC002A49DB07EE102A87EE870A01F0CE
:10E9D80017FA01F03DF9012D38D0022D2DD0002D68
:10E9E80040D09FED2D7ADFED2D7A30EE070A30EE1C
:10E9F800670A38BDDFED2A7A9FED2A0A002CA8BFE6
:10EA0800B0EE670A38BD9FED260AE4E79FED230ABA
:10EA180038BDBDE8384001F01BB9B0F1FF4F22D036
:10EA2800022DF3D0032D2BD0DFED1F7A9FED1F0AA7
:10EA3800012D18BFB0EE670A38BD9FED177ADFEDDC
:10EA4800177A30EE070A37EEC00A38BD10EE103AD2
:10EA580003F1004300EE103A38BD3C31B3DA9FEDC4
:10EA6800120AB8E738BD022D10D0032D0BD0DFED08
:10EA7800107A9FED100A012D18BFB0EE670A38BD55
:10EA88009FED040A38BD9FED0C0A38BD9FED0B0AB7
:10EA980038BD00BFDB0F49C02EBDBB33DB0F49407B
:10EAA800DB0FC93FDB0FC9BF00000000000000807A
:10EAB800DB0F493FDB0F49BFE4CB16C0E4CB164060
:10EAC8002DE9F04710EE905A35F000472DED028BF6
:10EAD80010EE904A10EE106A13D026F00048B8F1F4
:10EAE800FF4F10EE109A06DDBDEC028B5048BDE8D2
:10EAF800F04701F003BAB7F1FF4F08DDB8F17E5FC8
:10EB0800F2D1B7EE000ABDEC028BBDE8F087002E0B
:10EB180051DB4FF0000AB7F1FF4F43D0B7F17E5FEA
:10EB28005CD0B4F1804F68D0B4F17C5F00EE106A1D
:10EB38001CD001F065F9B8F1000F20D029F040434E
:10EB4800B3F17E5F1BD04FEAD973013B5AEA030049
:10EB580066D0B7F19A4F73DD364A904500F3CC8101
:10EB6800002CC0F2CF819FED340ACCE7B9F1000F39
:10EB7800DFDBBDEC028BBDE8F04700F0CBBB002C1F
:10EB8800BCBFF7EE007A87EE800AB9F1000FBADA57
:10EB9800A8F17E585AEA08083BD130EE400A80EEC8
:10EBA800000AB0E7B8F17E5FABD01FDD002CDADBDE
:10EBB80000EE105AA7E7B7F1974F14DAB7F17E5F66
:10EBC80009DBFB15C3F1960347FA03F202FA03F3D4
:10EBD800BB4200F087814FF0000A9FE7002C11DB51
:10EBE80000EE106A8FE74FF0020A94E7002CBADAB9
:10EBF80002EE105AB1EE420A85E706EE106A26EEDA
:10EC0800060A80E705EE906AB7EE000A80EE250A4C
:10EC180079E7BAF1010F7FF476AFB1EE400A72E7F7
:10EC280002EE106A32EE420A80EE000A6BE700BF7D
:10EC380094300108F7FF7F3F000000000000804B80
:10EC4800B8F5000F80F256815FED047A60EE277AFE
:10EC58006FF0170117EE908AEC4A4FEAE856C8F3AE
:10EC680016087F3E90450E4448F07E5140F33F81A0
:10EC7800E74A904540F3948100200136A1F5000150
:10EC88000246DFF8FC839FEDE36A9FEDE33ADFED90
:10EC9800E33A9FEDE34A9FEDE35ADFEDE34ADFF8FD
:10ECA800E4C3E24FDFEDE20A9FEDE21ADFEDE22A6C
:10ECB8009200904407EE901A98ED007A77EE876AF2
:10ECC800B7EE002A82EE262A491041F0005101F5DC
:10ECD8008021014477EEC75A01EE901A65EE826AE8
:10ECE80031EEC77A16EE900A37EEC70A26EEA67AF4
:10ECF80020F47F60A7EE063A20F00F000CEB02012B
:10ED080007EE900AE3EE073A3A44B1EE676AA3EEDB
:10ED1800874AE6EE215AA4EE075AE6EE005AE5EED7
:10ED2800074A65EE823A76EEA75A27EE077A65EE2D
:10ED3800A35AB0EE085AE7EE245AB0EE457AA7EE89
:10ED4800A77AD2ED004A91ED003A37EE257A02EE25
:10ED5800106A17EE100A20F47F6020F00F0207EE09
:10ED6800102A37EE455AB8EEC24AA6EE275A75EE73
:10ED7800C55A65EEA66AE3EE876AB0EE662AA7EE84
:10ED8800872A12EE100A20F47F6020F00F0202EEAC
:10ED9800102AA6EE072A07EE902A76EEC26A66EED9
:10EDA800A06AE7EE816A76EE836AB0EE667AA7EE2D
:10EDB800A27A37EE247A37EE047A17EE102A22F474
:10EDC8007F6222F00F0205EE902A35EEC47A37EE04
:10EDD800647AA7EEE27A76EEC77A24F47F6424F0A8
:10EDE8000F0406EE105A07EE104A02EE102A76EECD
:10EDF800476A66EE277A22EE077AE6EE827A0AF109
:10EE0800FF3A5AEA030AB7EE008A77EE876ABFEE3E
:10EE1800006A16EE903A08BFB0EE468A002B23F03F
:10EE2800004240F3AA80B2F1864F7BDC6FD0B2F18A
:10EE38007C5F7EDC0022104623F47F6323F00F03FF
:10EE480006EE903A9FED7D6A9FED7D2ADFED7D3AD3
:10EE5800DFED7D2A9FED7D4ADFED7D4A9FED7D5AEE
:10EE6800DFED7D5A36EEC77A26EE866A77EEC77AE8
:10EE7800B0EE003AA7EE826AB7EE000AF0EE467AE4
:10EE8800E6EEA37A27EEA77AB0EE672AA7EE224A23
:10EE9800A6EEE32AE4EE074A76EE426AA4EE875A23
:10EEA800B0EE676AE5EE075AE7EEA66AA5EEC76A0E
:10EEB800B0EE467A37EE437A27EE866A86EE077A10
:10EEC80077EE666A76EEE77A30EE670A10EE103A69
:10EED8001344B3F5000FC0F2968000EE103A28EE06
:10EEE800000A10E602F00102C2F1020A16E600204A
:10EEF8000246C6E60021AFE6584A904554DD002C8C
:10EF08007FF731AE9FED560A20EE000AFBE59FED34
:10EF1800556A76EEC76A37EE866AB4EEE66AF1EEAF
:10EF280010FA06DDDFED4E7A28EE270A20EE270AD2
:10EF3800E9E5D2154FF400017E3A41FA02F21A448B
:10EF4800C2F3C751484DA1F17F0445FA04F4C2F356
:10EF5800160022EA040205EE902A37EE657AC1F11E
:10EF6800960140F400000841002B37EE876AB8BFCD
:10EF78004042C20516EE103A5EE73C498A4208DC78
:10EF88007FF455AF76EEC76AF4EEE67AF1EE10FA42
:10EF9800CFD8DFED377A28EE270A20EE270AB2E528
:10EFA8004FF4001001226CE6F7EE007A30EE670AA3
:10EFB800DFED1B6ADFED2F7A9FED2F5A9FED2F6A49
:10EFC800F1EE405AB5EE007AE5EE876AB6EE007AC1
:10EFD800A6EEC07A60EE006A26EE877A67EEC77AF8
:10EFE800E0EE057AF0EE676AE0EE066A16EE902A21
:10EFF80022F47F6222F00F0207EE102AA5EE867A2D
:10F0080077EEC77AE9E600F07FFF68E771C41C0075
:10F01800D6B35D0042F1533E55326C3E05A38B3E9C
:10F02800ABAAAA3EB76DDB3E9A99193FA0300108FA
:10F038004F38763FA0C39D360038763F8CBEBF352B
:10F048001872313F0072313F4CBB31330EEADDB5E7
:10F0580055B38A38610B36BBABAA2A3E0700803FFE
:10F06800CAF249713CAA3833FFFF7F0000001643FB
:10F078006042A20D3BAAB83F70A5EC3600AAB83F83
:10F08800B0300108A830010870B510EE103A934A64
:10F0980023F00044944286B010EE106A054666DDFF
:10F0A8008F4A94421ADC002BDFED8E7A8E4A24F0C8
:10F0B8000F0440F3DB80944270EE677A66D09FEDD0
:10F0C8008B7A77EEC76A012077EEE67AC5ED006A9B
:10F0D80037EEC77A85ED017A06B070BD844A94424E
:10F0E80066DDB4F1FF4F49DAE215863AA4EBC25463
:10F0F80007EE104AFDEEC77ADFED7E6AF8EEE77A92
:10F1080037EE677ACDED037A27EE267AFDEEC77AD9
:10F11800F8EEE77A37EE677ACDED047A27EE267AAD
:10F12800B5EE407AF1EE10FA8DED057A40F0B18037
:10F13800F5EE407AF1EE10FA0CBF012302236E4976
:10F1480002208DE8030003A8294600F0B7F9002E35
:10F1580012DA95ED007AD5ED017AB1EE477AF1EE43
:10F16800677A404285ED007AC5ED017A04E0002215
:10F1780085ED000A4260002006B070BD70EE407A4E
:10F188000020C5ED017AC5ED007AF5E7DFED5B6A91
:10F198009FED5B7A77EEE67A012077EEC76A77EE25
:10F1A800E67AC5ED006A37EEC77A85ED017AE3E7BE
:10F1B80000F026FEDFED536ADFED4A5ADFED4B7AA9
:10F1C800B6EE007AA0EE267ABDEEC77AF8EEC76AE8
:10F1D80017EE100AB1EE666A1F28A6EE250A66EE3B
:10F1E800A77A1DDC484B411E24F0FF0253F821305A
:10F1F8009A4215D030EE677A85ED007A30EE470AEC
:10F20800002E70EE677AC5ED017AB5DAB1EE477A6D
:10F21800F1EE677A85ED007AC5ED017A4042ABE7F9
:10F2280030EE677AE41517EE102AC2F3C753E31AD3
:10F23800082BE1DD9FED317A9FED315AF0EE405A0F
:10F24800E6EE075A70EE657AE6EE077AD6EE857A2C
:10F2580035EEE77A17EE102AC2F3C753E41A192CD1
:10F268002CDC85ED007AB0EE650AC7E7944270EEB3
:10F27800277A10D09FED1D7A77EE876A4FF0FF301E
:10F2880077EEE67AC5ED006A37EE877A85ED017A82
:10F2980072E7032353E7DFED196A9FED197A77EEDA
:10F2A800A67A4FF0FF3077EE876A77EEE67AC5EDFB
:10F2B800006A37EE877A85ED017A5DE79FED137A6C
:10F2C8009FED135AB0EE650AA6EE070A75EEC07AEE
:10F2D800E6EE077AD6EE857A8CE700BFD80F493F6D
:10F2E800E3CB1640800FC93FD00FC93F43443537A1
:10F2F800800F494300008043383101080044353706
:10F3080008A3852E84F9223FB830010800A3852E72
:10F3180032318D2410EE103A23F00042B2F1FF4F43
:10F3280070B430D26AB3002B3DDBB2F5000F4FEA60
:10F33800E3512CD3A1F17F02C3F31603D10743F4A1
:10F34800000348BF5B00002556105B002C461921BE
:10F358004FF08072A018984202DC1B1A84181544DA
:10F3680001394FEA43034FEA5202F3D113B105F0D2
:10F3780001031D446D1005F17C5505EBC65500EEE3
:10F38800105A70BC7047A0EE000A70BC704713F4A6
:10F3980000020DD15B00180202F10102FAD5C2F198
:10F3A80001021144C6E730EE400A80EE000AE8E7A1
:10F3B80001221144BEE700BF10EE103A23F00043CB
:10F3C800B3F1485F2CDAFDEEC07A17EE903A002BC5
:10F3D80060D060EE007ADFED314A9FED315ADFED03
:10F3E800315A9FED316ADFED316A9FED317AA7EE30
:10F3F800A45AE5EE275AA5EEA76AE6EE276AA6EE16
:10F40800A77A27EE277A20EEC00AF6EE006AA7EE62
:10F41800870AB7EE007A97EEA60A37EE400A7047D9
:10F4280060EE007ADFED1D4A9FED1D5ADFED1D5A93
:10F438009FED1D6ADFED1D6A9FED1D7A1D4AA7EE3F
:10F44800A45A9342E5EE275AA5EEA76AE6EE276A84
:10F45800A6EEA77A27EE277AD5DD174A934214DC61
:10F4680003F17F4306EE903AF7EE005A75EEE65A3E
:10F4780060EEC00AB6EE006AE7EE870AD7EE866A43
:10F4880076EEE00A35EEE00A7047F6EE075AF5EE3A
:10F49800026AEDE7B7EE000A704700BF4ED747ADE6
:10F4A800F6740F317CF293B4010DD037610BB6BA04
:10F4B800ABAA2A3D9999993E0000483F2DE9F04FA3
:10F4C8002DED048BD7B0A54C649D039103F1FF3952
:10F4D80054F825801D46D31E48BF131DDB1023EAB0
:10F4E800E3730493049EDB4302EBC303824619EBE8
:10F4F80008000293C9EB060318D4659E184401302E
:10F508001AA906EB83040022002BAABFA658DFED38
:10F51800947A07EE106A03F10103A8BFF8EEC77AE0
:10F528008342E1EC017A02F10402EDD1B8F1000F57
:10F538004FEA880B1DDB1AA843AE00EB85045E4436
:10F5480042A8B9F1000FC0F2AE81DFED857A5146CD
:10F5580022460023F1EC016A32ED017A0133AB4215
:10F56800E6EE877AF6D1E0EC017AB04204F10404C1
:10F57800E7D10DF1180C4446CDF81480DFED7A8AF6
:10F588009FED788ADDF80880E344A60056AB334443
:10F59800002C13ED140A1BDDACF1040142AA32441D
:10F5A800314405AB60EE287AB0EE407AFDEEE77A9A
:10F5B80072ED016AF8EEE77AA7EEC87A37EEA60A86
:10F5C800BDEEC77A17EE100A43F8040F8B42E9D153
:10F5D8004046CDF800C000F097FCB0EE409AB4EE7B
:10F5E800000A29EE000A00F01DFCF2EE007AA0EEF7
:10F5F800679AB8F1000FDDF800C0FDEEC99AF8EE81
:10F60800E97A39EE679A40F3A180611EC8F10800D3
:10F618005CF8213043FA00F202FA00F01B1A4CF8A9
:10F62800213019EE901AC8F10700114443FA00F08E
:10F6380009EE901A0190019B002B2DDD19EE902AFE
:10F64800002C02F1010209EE902A40F34081634642
:10F658000CEB0607002153F8042BC2F1FF0011B987
:10F66800C2F5807012B143F8040C0121BB42F2D1FB
:10F67800B8F1000F0DDDB8F1010F00F00281B8F10B
:10F68800020F06D1621E5CF8223003F03F034CF8EB
:10F698002230019B022B69D0B5EE409AF1EE10FAA8
:10F6A80078D10599671EB9420ADC6644002356F8EA
:10F6B800042D5E4543EA0203F9D1002B40F0B181E5
:10F6C800059A531E5CF82320002A40F0A7810CEB12
:10F6D80083034FF0010E53F8042D0EF1010E002A9A
:10F6E800F9D0A644661C76452EDC0498049F204475
:10F6F800659C09EB06031AA904EB800001EB83045F
:10F70800659B774442AA02EB860603EB870750F80D
:10F71800041F07EE901AF8EEE77AB9F1000FE4EC4F
:10F72800017ADFED0F7A0BDB514622460023F1EC1C
:10F73800016A32ED017A0133AB42E6EE877AF6D1FF
:10F74800B842E6EC017AE2D174461EE740F0A180A7
:10F75800631E5CF823301B1201936CE750340108D8
:10F7680000000000000080430000803BB7EE000A64
:10F7780030EE499A00298FD04046CDF800C000F0FD
:10F78800C3FB39EE409ADDF800C0B5EE409AF1EEC1
:10F7980010FA86D0029BCDF800C0B0EE490A584254
:10F7A800DDF8148000F0B0FB5FED127ADDF800C0E0
:10F7B800B4EEE70AF1EE10FAC0F254811FED167AA2
:10F7C800029A20EE077A671CBDEEC77A0832B8EEB7
:10F7D800C77A0292A7EE670ABDEEC77ABDEEC00AE5
:10F7E80010EE103A4CF8243017EE104A4CF8274027
:10F7F8000298CDF800C0B7EE000A00F085FB002F94
:10F80800DDF800C036DB7D1CAA0042AE1FED2A7A67
:10F818000CEB0203324473ED017AF8EEE77A6345A4
:10F8280067EE807A20EE070A62ED017AF3D142A8EA
:10F8380000EB87040020B8F1000FC0F2E98090497E
:10F84800DFED907A2246002301E0834208DCF1ECE8
:10F85800016AB2EC017A01339845E6EE877AF4DA68
:10F8680056A901EB800301308542A4F1040443ED5D
:10F87800287AE0D1649C032C7FD8DFE804F0B387B2
:10F88800872A621E5CF8223003F07F034CF822308E
:10F89800FFE6F6EE007AB4EEE79AF1EE10FA0CDA2B
:10F8A80000220192F8E6DFED777AE0EC017AB042C7
:10F8B80004F104047FF445AE5BE619EE902A0221B8
:10F8C8000132002C019109EE902A3FF7C0AE0021C9
:10F8D800CEE6002F40F3B980B90056AB7A1C2EAEA5
:10F8E8000B4406EB820253ED287A2FA8134653EDFA
:10F8F800026A36EEA77A76EEC76A76EEA76AF0EE67
:10F90800477A63ED016A834203ED017AEFD1012F53
:10F9180040F39B8056A8014451ED287A134630A93C
:10F9280053ED026A36EEA77A76EEC76A76EEA76AD4
:10F93800F0EE477A63ED016A8B4203ED017AEFD16D
:10F94800DFED507A134633ED017A994277EE877AE4
:10F95800F9D1019C002C7DD0DDED2E6A9DED2F7A2A
:10F96800039EF1EE677AF1EE666AB1EE477AC6ED6C
:10F97800027AC6ED006A86ED017A19EE901A01F056
:10F98800070057B0BDEC048BBDE8F08F002F74DB87
:10F998002EAA7B1CDFED3B7A02EB830333ED017A61
:10F9A800934277EE877AF9D1019AA2B3B1EE677ADA
:10F9B800DDED2E6A039B002F83ED007A76EEE77A61
:10F9C80008DD2FAB03EB8707B3EC017ABB4277EE78
:10F9D800877AF9D1019C0CB1F1EE677A039DC5EDE8
:10F9E800017ACAE7002F45DB7B1C2EAADFED257ABA
:10F9F80002EB830333ED017A934277EE877AF9D1EC
:10FA0800019E0EB1F1EE677A0399C1ED007AB4E771
:10FA1800DFED1C7A24E7B0EE677AC9E74FF0010EF4
:10FA28005FE6029A5CF82730DDF81480083A029203
:10FA3800002B7FF4DDAE0CEB870353F8041D013F68
:10FA4800083A0029F9D00292D2E6019CDFED0D7A3E
:10FA5800002C81D1039D2E9A2F9BC5ED027A2A6036
:10FA68006B608AE7BDEEC00A274610EE105A4CF8C4
:10FA78002450BDE6DFED037AC2E7DFED027A93E7B3
:10FA88005C3401080000000010EE103A23F0004337
:10FA9800B3F1485F04DAFDEEC07A17EE903A23B36B
:10FAA80060EE007A9FED155A9FED156ADFED156A35
:10FAB8009FED157ADFED155AA7EE856A27EE805A75
:10FAC800E6EE276AA6EEA77AE7EE275A70B165EE4A
:10FAD800C55AB6EE007AE0EE875A9FED0D7AD5EE5C
:10FAE800A70AE5EE070A30EE600A70479FED097A2B
:10FAF800A7EEA57AA7EE050A704700BFD3C92E2F37
:10FB0800342FD7B21BEF3836010D50B98988083C1D
:10FB1800ABAA2A3EABAA2ABE00207047000000000C
:10FB28009FED010B704700BF000000000000F87F48
:10FB3800F0B553EC102BC3F30A50A0F2FF31132990
:10FB480083B09C4610EE107A4FEAD37631DC002958
:10FB58004FDB3D48084100EA0304144327D040081E
:10FB680000EA030717430CD04FF4802C132923EA2B
:10FB780000004CFA01F140EA010C14BF00274FF0D5
:10FB88000047324B03EBC6063C46D6E9006763469E
:10FB9800224630463946FBF7C7FDCDE9000132461B
:10FBA8003B46DDE90001FBF7BDFD41EC100B03B05E
:10FBB800F0BD33290ADDB1F5806FF8D151EC100B97
:10FBC8000B46FBF7B1FD41EC100BF0E7A0F2134038
:10FBD8004FF0FF31C1401142E9D049081142D0D05D
:10FBE8004FF0804722EA010147FA00F041EA000796
:10FBF800C7E723F000411143D9D0C3F313010A43E7
:10FC0800544214431148590C240B490404F40024A9
:10FC180000EBC60053EC102B44EA0103D0E9004581
:10FC280020462946FBF780FDCDE900012B462246F8
:10FC3800DDE90001FBF776FD21F0004343EAC671D8
:10FC480041EC100BB3E700BFFFFF0F008834010839
:10FC580038B510EE105A25F00044B4F1A14FF0EE7B
:10FC6800407A0BDBB4F1FF4F56DCDFED527A9FEDA3
:10FC7800520A002DC8BFB0EE670A38BD4F4B9C42F0
:10FC880059DCB4F1445F4ADB4FF0FF3367EEA76AF3
:10FC98009FED4B1A9FED4B2A9FED4B3ADFED4B1A28
:10FCA800DFED4B2A9FED4B4ADFED4B3A9FED4B5A68
:10FCB800DFED4B4A9FED4B6ADFED4B5A26EEA67AF5
:10FCC8005A1CA7EE012AE7EE212AA2EE073AE2EE35
:10FCD800873AA3EE074AE3EE874AA4EE075AE4EE12
:10FCE800875AA5EE076A25EE877A66EE266A3AD025
:10FCF8003E493F4A9B00194436EE877A91ED005AF7
:10FD080097EE275A1344002D93ED000A75EE677A93
:10FD180030EE670A24DB38BD30EE000A38BDDFED6F
:10FD2800356A70EE266AB7EE007AF4EEC76AF1EE2D
:10FD380010FAA9DD38BD00F063F82F4B9C4219DC9E
:10FD4800A3F5D0039C422ADCF0EE007ABFEE007ADD
:10FD5800A0EE277A002370EE277AC7EE277A95E778
:10FD6800B1EE400A38BD36EE877AB0EE670AA7EEE4
:10FD7800670A38BD214B9C420BDCF7EE087AB7EED8
:10FD8800007AA0EE277A022370EE677AC7EE877AA8
:10FD98007CE7FFEE007AC7EE807A032376E7B7EEBA
:10FDA800007A70EE477A30EE077A0123C7EE877A39
:10FDB8006CE700BFDB0FC93FDB0FC9BFFFFFDF3EAA
:10FDC800D769853C59DA4B3D356B883D21A215BD75
:10FDD8006BF16EBD6E2EBA3D95879DBD2549123ECD
:10FDE800388EE3BDABAAAA3ECDCC4CBE98340108F0
:10FDF800A8340108CAF24971FFFF973FFFFF1B4073
:10FE080010EE102A22F0004300EE103A704700BFAF
:10FE180010EE103A23F00040B0F1FF4FACBF0020C5
:10FE28000120704710EE103A23F00040C10D7F39D1
:10FE3800162910B418DC00291C4622DB1E4808418C
:10FE4800184214D0DFED1D7A70EE277AF5EEC07AED
:10FE5800F1EE10FA0BDD002B21DB24EA000000EEA6
:10FE6800100A5DF8044B7047B0F1FF4F04D200EE62
:10FE7800103A5DF8044B704730EE000A5DF8044B09
:10FE88007047DFED0E7A70EE277AF5EEC07AF1EE64
:10FE980010FAECDD002B08DB9FED090AE9E74FF4C7
:10FEA800000343FA01F10C44D7E70028BFEE000A2B
:10FEB80008BF00EE103ADCE7FFFF7F00CAF2497185
:10FEC8000000000010EE103A33F0004001D102208B
:10FED8007047A0F50003B3F1FE4F01D2042070472C
:10FEE800054B421E9A4201D803207047B0F1FF43E8
:10FEF80058425841704700BFFEFF7F009FED010A3E
:10FF0800704700BF0000C07F08B510EE103A33F00C
:10FF180000412DED028B10EE102A11D0B1F1FF4FE8
:10FF280011D2B1F5000F13D3C90D0144FE2930DCFD
:10FF380000291CDD22F0FF4242EAC15200EE102ADD
:10FF4800BDEC028B08BDBDEC028B30EE000A08BD8B
:10FF5800DFED1E7A1E4A20EE277A904217EE103AFD
:10FF680022DBC3F3C75117EE102A1939DDE711F167
:10FF7800160F1EDA4CF2503290420ADC9FED158AB9
:10FF880000EE903AB0EE480A00F02AF820EE080A8F
:10FF9800D6E79FED118A00EE903AB0EE480A00F0DD
:10FFA8001FF820EE080ACBE79FED0A0A27EE000AA1
:10FFB800C6E7193122F0FF4242EAC152DFED077A63
:10FFC80007EE102A27EE270ABAE700BF0000004C08
:10FFD800B03CFFFF6042A20DCAF249710000003335
:10FFE80010EE101A21F0004210EE901A01F00043B2
:08FFF800134300EE103A7047BC
:020000040801F1
:10000000014B1868704700BFE001002000000000AD
:1000100000C20100081A01082B1A010801000000A3
:1000200000E10000401A0108621A01080200000005
:1000300000960000761A0108981A010803000000D3
:10004000004B0000AC1A0108CE1A010804000000A1
:1000500080250000E21A01081F220108B56206246B
:100060002400FFFF0303000000001027000005002C
:10007000FA00FA0064002C01003C00000000C800F7
:1000800000000000000017C2B56206010300F00581
:1000900000FF19B56206010300F00300FD15B5620B
:1000A00006010300F00100FB11B56206010300F038
:1000B0000000FA0FB56206010300F00200FC13B560
:1000C0006206010300F00400FE17B562060103009A
:1000D0000102010E47B562060103000103010F4949
:1000E000B56206010300010601124FB56206010365
:1000F0000001300540A7B562060103000112011E90
:1001000067B56206080600C80001000100DE6A004B
:10011000B56206160800030703000000000031E581
:1001200001B5620616080003070300510800008AA3
:100130004102B562061608000307030004E004004C
:10014000199D03B5620616080003070300000202AA
:100150000035EF04B56206160800030703008001AE
:100160000000B2E80004004810000102000400484A
:100170002000010200000000000000000301000058
:10018000DC060108040000009C06010804000000D1
:100190005C060108020100003C06010800010000A5
:1001A0000000000006000000DC0501080600000059
:1001B0007C050108010100000000000004000000AF
:1001C0003C05010806000000DC04010808000000EE
:1001D0005C04010808000000DC03010808000000BE
:1001E0005C030108010100000000000000010000A4
:1001F00000000000000100000000000004000000FA
:100200001C03010806000000BC02010800010000F8
:1002100000000000020100009C0201080101000032
:10022000000000000000000000000000840201083F
:100230006C0201086A02010868020108812C0008AA
:100240003D2C0008192C0008F12B0008E12B0008B8
:10025000913600086D2C0008912B0008612C0008D5
:10026000532C0008E8090020FFFFFFFF0A010003EC
:100270000103020303030403050306030703080342
:100280000903FFFF00030103020303030403050343
:100290000603070308030903FFFF00000000803F77
:1002A0000000000000000000000080BF0000803F50
:1002B00000000000000000000000803F0000803FC0
:1002C000000080BF0000803F000080BF0000803F32
:1002D000000080BF000080BF0000803F0000803F22
:1002E0000000803F0000803F0000803F0000803F12
:1002F0000000803F000080BF000080BF0000803F02
:100300000000000000000000000000000000803F2E
:100310000000000000000000000000000000803F1E
:10032000000000000000803F0000803F0000803F90
:10033000000080BF000080BF000000000000803F80
:10034000000000000000803F000080BF0000803FF0
:100350000000803F000080BF000000800000803F60
:100360000000803F000000BF0000803F0000803F91
:10037000000000BF000080BF0000803F0000803F01
:10038000000080BF0000003F0000803F0000803F71
:100390000000003F0000803F0000803F0000803FE1
:1003A0000000003F000080BF000080BF0000803FD1
:1003B000000080BF000000BF000080BF0000803F41
:1003C000000000BF0000803F000080BF0000803FB1
:1003D0000000803F0000003F000080BF0000803F21
:1003E000F704353FF70435BF0000803F0000803F31
:1003F000F70435BFF70435BF0000803F0000803FA1
:10040000F70435BFF704353F0000803F0000803F10
:10041000F704353FF704353F0000803F0000803F80
:1004200000000000000080BF000080BF0000803F8F
:10043000000080BF00000000000080BF0000803F7F
:10044000000000000000803F000080BF0000803FEF
:100450000000803F00000000000080BF0000803FDF
:10046000000080BF0000803F000080BF0000803F90
:10047000000080BF000080BF0000803F0000803F80
:100480000000803F0000803F0000803F0000803F70
:100490000000803F000080BF000080BF0000803F60
:1004A000000080BF0000803F0000803F0000803FD0
:1004B000000080BF000080BF000080BF0000803FC0
:1004C0000000803F0000803F000080BF0000803FB0
:1004D0000000803F000080BF0000803F0000803FA0
:1004E000000000BFD0B35D3F0000803F0000803FB0
:1004F000000000BFD0B35DBF0000803F0000803F20
:100500000000003FD0B35D3F000080BF0000803F8F
:100510000000003FD0B35DBF000080BF0000803FFF
:10052000000080BF00000000000080BF0000803F8E
:100530000000803F000000000000803F0000803F7E
:10054000000000000000803F000080BF0000803FEE
:10055000000080BF000080BF000000000000803F5E
:10056000000000000000803F0000803F0000803F4E
:100570000000803F000080BF000000000000803FBE
:10058000D0B35DBF0000003F0000803F0000803F0F
:10059000D0B35DBF000000BF000080BF0000803FFF
:1005A000D0B35D3F0000003F0000803F0000803F6F
:1005B000D0B35D3F000000BF000080BF0000803F5F
:1005C00000000000000080BF0000803F0000803F6E
:1005D000000000000000803F000080BF0000803F5E
:1005E00000000000A8AAAA3F0000803F0000803F52
:1005F000000080BFB0AA2ABF000080BF0000803F7B
:100600000000803FB0AA2ABF000080BF0000803FEA
:1006100000000000A8AAAA3F000080BF0000803FA1
:10062000000080BFB0AA2ABF0000803F0000803FCA
:100630000000803FB0AA2ABF0000803F0000803F3A
:100640000000803F00000000000000000000803F2C
:10065000000080BF00000000000000000000803F9C
:10066000000080BF0000803F000080BF0000803F8E
:10067000000080BF000080BF0000803F0000803F7E
:100680000000803F0000803F0000803F0000803F6E
:100690000000803F000080BF000080BF0000803F5E
:1006A000000000000000803F000080BF0000803F8D
:1006B000000080BF000000000000803F0000803F7D
:1006C0000000803F000000000000803F0000803FED
:1006D00000000000000080BF000080BF0000803FDD
:1006E00000000000A8AAAA3F000000000000803F10
:1006F000000080BFB0AA2ABF000000000000803FB9
:100700000000803FB0AA2ABF0000000000A24A04F7
:10071000524F4C4C3B50495443483B5941573B4145
:100720004C543B506F733B506F73523B4E6176524B
:100730003B4C4556454C3B4D41473B56454C3B0099
:1007400000000000021C0108000000000100000081
:10075000071C010801000000020000000E1C010837
:100760000200000003000000171C01080300000045
:10077000040000001D1C0108050000000500000029
:10078000221C010806000000060000002C1C0108C5
:100790000700000007000000351C010808000000E9
:1007A000080000003E1C01080900000009000000CC
:1007B000471C01080A0000000A000000511C010843
:1007C0000B0000000B0000005B1C01080C00000087
:1007D0000C000000651C01080D0000000D00000069
:1007E0006D1C01080E0000000E000000751C0108C1
:1007F0000F0000000F0000007D1C01081000000029
:1008000010000000861C010811000000110000000B
:100810008D1C01081200000012000000971C010846
:1008200013000000130000009F1C010814000000CA
:1008300014000000AA1C01081500000015000000AB
:10084000B41C0108160000001600000000000000A3
:10085000FF000000F51B0108EC1B0108E01B01086C
:10086000000000008025000000C201000000000020
:10087000010000008025000000C201000600000009
:10088000020000008025000000C2010007000000F7
:10089000030000008025000000C2010007000000E6
:1008A000010001020001030001040001050001062E
:1008B00000010700010800010900010A00010B0006
:1008C000010C01039001C800C800C800C800C8009E
:1008D000C800C800C80064000000C800C800C80004
:1008E000C8003200020000008025000000C20100A4
:1008F00000000000200000008025000000C2010070
:1009000001000000400000008025000000C201003E
:1009100000000000010000008025000000C201006E
:1009200000000000100000008025000000C201004F
:10093000000300000400000080250000004B0000C0
:10094000000000000800000000E1000000E10000DD
:10095000000400003203530054004D003300320005
:1009600020005600690072007400750061006C0080
:10097000200043004F004D00200050006F00720027
:100980007400200020002603530054004D0069002D
:10099000630072006F0065006C0065006300740006
:1009A00072006F006E0069006300730004030904A5
:1009B0006F20010873200108792001087F200108B9
:1009C00082200108892001088C200108912001085B
:1009D0009D200108A0200108A6200108AD200108E3
:1009E000B7200108C1200108CA200108D820010849
:1009F000E4200108EB200108F1200108FE20010895
:100A00000921010816210108000000001E1E64646F
:100A10006464646409024300020100C032090400F6
:100A2000000102020100052400100105240100015B
:100A3000042402020524060001070582030800FFC2
:100A400009040100020A000000070503024000003B
:100A500007058102400000000000000000004F0078
:100A6000000007000700147F147F14242A7F2A1235
:100A70002313086462364955225000050300000024
:100A80001C2241000041221C0014083E08140808E2
:100A90003E080800503000000808080808006060A0
:100AA000000020100804023E5149453E00427F40AC
:100AB0000042615149462141454B311814127F10C3
:100AC00027454545393C4A494930017109050336F6
:100AD00049494936064949291E0036360000005664
:100AE000360000081422410014141414140041228A
:100AF00014080201510906324979413E7E11111153
:100B00007E7F494949363E414141227F4141221C75
:100B10007F494949417F090909013E4149497A7F95
:100B20000808087F00417F41002040413F017F08C5
:100B30001422417F404040407F020C027F7F040826
:100B4000107F3E4141413E7F090909063E41512146
:100B50005E7F09192946464949493101017F010152
:100B60003F4040403F1F2040201F3F4038403F63F0
:100B70001408146307087008076151494543007F52
:100B800041410002040810200041417F000402019D
:100B900002044040404040010204000020545454EC
:100BA000787F484444383844444420384444487F9B
:100BB0003854545418087E090102064949493F7FB8
:100BC0000804047800447D40002040443D007F102C
:100BD00028440000417F40007C0418047C7C080409
:100BE000047838444444387C141414080814141845
:100BF0007C7C080404084854545420043F4440209A
:100C00003C4040207C1C2040201C3C4030403C4468
:100C1000281028440C5050503C4464544C44000864
:100C200036410000007F000000413608000201024A
:100C300004023E55554122000000000000007900EA
:100C4000001824742E24487E4942405D2222225DF1
:100C500015167C161500007700000A55555528001A
:100C600001000100000A0D0A0408142A14220404D9
:100C700004041C000808080001010101010002052C
:100C8000020044445F444400000402017E2020101E
:100C90003E060F7F007F0018180000004050200023
:100CA000000A0D0A0022142A14081708342A7D1796
:100CB00008046A59304845402042004200427E42C2
:100CC0000042007E7E0042007E7E7E42007E7E7E6E
:100CD0007E007E7E7E7E7E5A0000005A5A40404052
:100CE0005A7A6060607A7A7070707A7A7878787AF6
:100CF0007A7C7C7C7A7A7E7E7E7A0506040203000A
:100D0000B9460008B94600087D790008B9460008D0
:100D1000B9460008B9460008B9460008E92E00089F
:100D2000B9460008B9460008B9460008B9460008A7
:100D3000B9460008B946000804010000672401080C
:100D40006C240108702401087F240108752401081F
:100D5000742301087B240108000000001F22010801
:100D60001B240108232401082B2401083324010833
:100D70003A240108452401084D240108552401089E
:100D80005D2401086224010800000000B15700083A
:100D9000392F0008092F000851A500085B2F000813
:100DA0004DA50008AD960008F52E0008255700084F
:100DB000072F0008012F0008052F00081225010841
:100DC0001B2501085F5800083F250108432501083D
:100DD00095590008592501085E250108D9680008C1
:100DE00077210108722501089D8300088F250108DD
:100DF00094250108CD6F0008C32501081F220108B2
:100E0000B9830008C8250108D025010801B00008F1
:100E1000E4250108E8250108F9A00008FB250108E0
:100E20000A26010811AF0008242601081F22010824
:100E300009650008292601082D2601080567000814
:100E40006C25010849260108356500085C26010863
:100E500062260108D16500082F2D01087D260108B2
:100E6000816F00088C2601087D260108AD7B0008F3
:100E7000982601089D260108E5830008F91E01084F
:100E8000AD26010859A10008DB260108CF2601087C
:100E900035970008F52A01081F220108D9640008C7
:100EA000482701084F270108542701086527010832
:100EB0006F2701087A270108852701087423010894
:100EC000902701087524010899270108A327010824
:100ED000B1270108B4270108C4270108CB2701085E
:100EE000D4270108DE270108E627010800000000DA
:100EF000F127010844000000101A00200000000043
:100F000028230000FA27010841000000121A0020DF
:100F10000000000001000000082801084400000053
:100F20001E1B0020B0040000A40600000F280108CA
:100F300044000000201B002000000000D00700003B
:100F40001928010844000000221B002000000000B6
:100F5000D00700002328010842000000241B0020C5
:100F600000000000120000003028010842000000CC
:100F7000251B002001000000FF0000003B280108A5
:100F800042000000261B00200000000001000000BD
:100F90005028010844000000D41A0020000000007E
:100FA000D00700005D28010844000000D61A002088
:100FB00000000000D00700006A280108440000007B
:100FC000D81A002000000000D00700007628010891
:100FD00044000000DA1A002000000000D0070000E2
:100FE0008628010844000000DC1A002000000000F0
:100FF000D00700009728010844000000DE1A0020F6
:1010000000000000D0070000A228010844000000F2
:10101000E01A002000000000D0070000B7280108F7
:1010200044000000E21A002032000000007D0000B1
:10103000C628010844000000E41A00203200000025
:10104000F2010000D528010841000000271B002004
:101050000000000001000000E2280108410000003B
:10106000281B00200000000001000000F5280108F6
:1010700041000000291B002000000000B400000017
:1010800001290108410000002A1B00200000000087
:10109000640000000D290108420000002B1B002005
:1010A000FFFFFFFF010000002329010841000000AD
:1010B000301B002000000000090000003A29010850
:1010C00041000000311B002000000000090000006A
:1010D0005129010841000000321B002000000000DF
:1010E000090000006829010841000000331B0020AE
:1010F00000000000090000007F29010841000000F5
:10110000441B0020300000007E00000090290108F0
:1011100050000000341B0020B004000000C2010099
:101120009D29010850000000381B0020B004000079
:1011300000C20100AA290108500000003C1B002049
:101140000000000000C20100B729010850000000A3
:10115000401B0020B004000000C20100D02901089B
:10116000410000002C1B00200000000001000000D6
:10117000DD290108410000002D1B002000000000B7
:1011800004000000EB290108410000002E1B002094
:101190000000000001000000FB29010841000000E0
:1011A0002F1B00200000000001000000092A010898
:1011B00081000000601B002000000000C80000004B
:1011C000132A0108810000006A1B002000000000B3
:1011D000C80000001D2A010881000000741B0020C7
:1011E00000000000C8000000272A0108810000005C
:1011F000611B002000000000C8000000322A010826
:10120000810000006B1B002000000000C8000000EF
:101210003D2A010881000000751B0020000000002D
:10122000C8000000482A010881000000621B00205D
:1012300000000000C8000000522A010881000000E0
:101240006C1B002000000000C80000005C2A0108A0
:1012500081000000761B002000000000C800000094
:10126000662A0108840000000A1D0020000000001A
:10127000D0070000742A0108810000000E1D002024
:101280000000000001000000892A0108840000001D
:10129000101D00200A000000D0070000972A010856
:1012A00084000000121D00200A000000D00700008A
:1012B000A52A0108810000000D1D0020000000008B
:1012C00064000000B32A0108410000001C1B00203C
:1012D0000000000003000000C52A010841000000D2
:1012E000481B00200000000003000000D82A01086D
:1012F00041000000491B0020000000000100000028
:10130000E92A0108410000004A1B002000000000FB
:1013100001000000FD2A0108600000004C1B0020B5
:10132000A6FFFFFF5A000000152B01086000000017
:10133000501B00204CFFFFFFB40000002D2B0108C4
:1013400041000000541B00200000000001000000CC
:10135000462B010841000000551B00200000000042
:1013600001000000512B010844000000121B002066
:1013700000000000204E0000622B01084100000028
:10138000081B002000000000FF0000006D2B01087A
:1013900041000000091B00200A000000320000008C
:1013A000832B0108410000000A1B00200A000000F6
:1013B00032000000992B0108440000000C1B0020A3
:1013C0000100000010270000AD2B010844000000C0
:1013D0000E1B00200000000072060000C22B010856
:1013E00041000000101B0020000000000100000070
:1013F000E02B010841000000E61A00200000000078
:1014000008000000EB2B010841000000E71A002053
:101410000000000008000000F52B0108410000005A
:10142000E81A00200000000008000000FF2B01085F
:1014300048000000EA1A00204CFFFFFF680100008E
:10144000102C010848000000EC1A00204CFFFFFFA0
:1014500068010000222C010848000000EE1A00205C
:101460004CFFFFFF68010000322C0108440000001F
:10147000FA1A00206400000084030000482C0108D0
:1014800044000000F21A00200000000000010000EB
:10149000512C010841000000F81A00200000000053
:1014A00080000000612C010844000000F41A0020B4
:1014B00064000000E8030000722C010844000000F2
:1014C000F61A002064000000E8030000842C0108E4
:1014D00081000000B71C002001000000FA0000009D
:1014E000962C010881000000B81C002000000000BC
:1014F000010000008D2C010881000000B51C0020B7
:101500000000000020000000AB2C0108810000005A
:10151000B61C00200000000064000000B82C010888
:1015200081000000BC1C00200000000096000000AC
:10153000D22C010884000000BA1C00200100000029
:1015400084030000EC2C010842000000F01A002087
:10155000FFFFFFFF01000000022D010882000000D4
:10156000061D0020FFFFFFFF01000000102D0108F5
:1015700082000000071D00200000000001000000A4
:10158000222D010881000000A81B0020000000009F
:1015900002000000372D0108010100009A20002000
:1015A00000000000FA0000003F2D010801010000CA
:1015B0009B2000200000000064000000472D01086F
:1015C000010100009C2000200000000064000000D9
:1015D0004F2D0108010100009D20002000000000A7
:1015E00064000000582D0108010100009E20002029
:1015F0000000000064000000682D010801010000E7
:101600009F2000200000000064000000712D0108F0
:1016100001010000A0200020000000006400000084
:101620007A2D010804010000A2200020E803000038
:10163000D0070000892D010881000000FE1C002059
:1016400000000000C8000000982D01088100000083
:10165000FF1C002000000000C8000000AB2D0108A6
:1016600084000000001D0020E8030000D0070000F7
:10167000BD2D010884000000021D00206400000050
:10168000D0070000CF2D010884000000041D0020B9
:1016900064000000B80B0000E12D0108810000008B
:1016A000081D002000000000FF000000EE2D0108D2
:1016B00041000000F11A0020000000000A000000B4
:1016C000FB2D010881000000B01B0020000000007D
:1016D000FA0000000A2E010881000000B81B00205B
:1016E0000000000064000000192E010881000000C5
:1016F000B91B00200000000064000000272E010834
:10170000A0000000B41B0020010000001400000035
:10171000372E010881000000CC1B002000000000D3
:1017200001000000462E010888000000AE1B0020CA
:10173000D4FEFFFF2C010000552E01088800000098
:10174000AC1B0020D4FEFFFF2C010000632E01081B
:1017500081000000BC1B00200000000030000000E1
:10176000712E0108A0000000C01B00200000000036
:1017700001000000802E0108A0000000C41B002012
:1017800000000000010000008C2E0108A0000000F5
:10179000C81B00200000000001000000982E010876
:1017A00088000000AA1B0020B0B9FFFF50460000CF
:1017B000A82E010881000000581B00200000000036
:1017C00002000000B72E0108810000005D1B002010
:1017D00000000000C8000000BF2E010881000000CA
:1017E000671B002000000000C80000001A2C010840
:1017F00081000000711B002000000000C8000000F4
:10180000C72E0108810000005C1B002000000000C2
:10181000C8000000CE2E010881000000661B0020D9
:1018200000000000C8000000092C01088100000031
:10183000701B002000000000C8000000D52E010829
:10184000810000005E1B002000000000C8000000B6
:10185000DB2E010881000000681B00200000000052
:10186000C80000002C2C010881000000721B002021
:1018700000000000C8000000E12E0108A0000000E8
:10188000801B00200000000064000000EA2E010818
:10189000A00000008C1B002000000000640000007D
:1018A000F32E0108A0000000981B0020000000009B
:1018B00064000000FC2E0108A00000007C1B00203A
:1018C0000000000064000000042F0108A0000000D8
:1018D000881B002000000000640000000C2F01089D
:1018E000A0000000941B0020000000006400000025
:1018F000142F0108A0000000841B0020000000003D
:10190000640000001B2F0108A0000000901B0020B5
:101910000000000064000000222F0108A000000069
:101920009C1B00200000000064000000292F01081B
:10193000A0000000A41B0020000000000A0000001E
:10194000372F0108A0000000A01B002000000000AD
:101950000A000000432F0108810000005F1B0020E7
:1019600000000000C8000000492F010881000000AD
:10197000691B002000000000C80000004F2F010874
:1019800081000000731B002000000000C800000060
:10199000552F010881000000631B0020000000009B
:1019A000C80000005D2F0108810000006D1B0020B1
:1019B00000000000C8000000652F01088100000041
:1019C000771B002000000000C80000006D2F0108F8
:1019D00081000000651B002000000000C80000001E
:1019E000732F0108810000006F1B00200000000021
:1019F000C8000000792F010881000000791B002039
:101A000000000000C800000024505542582C34311A
:101A10002C312C303030332C303030312C313135CA
:101A20003230302C302A31450D0A0024504D544BB1
:101A30003235312C3131353230302A31460D0A0001
:101A400024505542582C34312C312C303030332C2A
:101A5000303030312C35373630302C302A32440D8E
:101A60000A0024504D544B3235312C353736303046
:101A70002A32430D0A0024505542582C34312C315F
:101A80002C303030332C303030312C33383430304F
:101A90002C302A32360D0A0024504D544B32353149
:101AA0002C33383430302A32370D0A002450554256
:101AB000582C34312C312C303030332C3030303104
:101AC0002C31393230302C302A32330D0A00245078
:101AD0004D544B3235312C31393230302A32320DBF
:101AE0000A0024505542582C34312C312C303030DF
:101AF000332C303030312C393630302C302A3136DE
:101B00000D0A000000400140000400480080000071
:101B1000041801020F0100000040014000040048C9
:101B200000400000001801020E010000002C0140DE
:101B30000000004800010000001B01020806000030
:101B4000000400400004004801000000081D0002DD
:101B500000020000000400400000004840000000B7
:101B6000001D0002060200000000004000000048C6
:101B700004000000081C00020201000000040040F4
:101B800000040048020000000C1D000201020000D9
:101B9000004801400000004880000000001A0102D7
:101BA0000701000000040040000000481000000091
:101BB000041D000204020000000000400000004874
:101BC00002000000041C00020101000000000040AF
:101BD00000000048080000000C1C000A030100007F
:101BE00044656320313420323031340032333A35A9
:101BF000363A313800633539356266380053504B18
